:020000040001F9
:109000003890002031BC0200AB320200E73302008E
:1090100023340200473402002B3502000000000018
:109020000000000000000000000000007337020094
:10903000B737020000000000434D0200A34E0200BB
:10904000BB510200F75A0200BD51020095570200C1
:109050009B570200275C02007F8A0200E57A02002B
:10906000B75A0200BF5A0200C75A02009B5D0200B5
:109070007B6C0200C5740200E7AD0200CBB00200B9
:109080007FB20200A36A0200F3B30200FFB702003E
:10909000E5B902009BBA0200DF110200A7BA020084
:1090A00033BB02000FBC020077BD0200B5BD020059
:1090B0004B780200B7BD0200000000000000000075
:1090C000B9BD0200BBBD0200BDBD0200DD2402002F
:1090D000BFBD0200C1BD0200C3BD02000000000010
:1090E0000000000000000000000000000000000080
:1090F0000000000000000000000000000000000070
:10910000000000000000000000000000000000005F
:10911000000000000000000000000000000000004F
:10912000000000000000000000000000000000003F
:10913000000000000000000000000000000000002F
:10914000000000000000000000000000000000001F
:10915000000000000000000000000000000000000F
:1091600000000000000000000000000000000000FF
:1091700000000000000000000000000000000000EF
:1091800000000000000000000000000000000000DF
:1091900000000000000000000000000000000000CF
:1091A00000000000000000000000000000000000BF
:1091B00000000000000000000000000000000000AF
:1091C000000000000000000000000000000000009F
:1091D000000000000000000000000000000000008F
:1091E000000000000000000000000000000000007F
:1091F000000000000000000000000000000000006F
:1092000081B000F5E0700268914203D343681A44CC
:10921000914202D380680028F5D101B07047DFF891
:109220006817086890B94FF4805048604FF4803256
:109230004FF0FF308A60C86008610420DFF84C27D7
:10924000DFF84C374861C2F8BC010B600120704761
:1092500001F1080313F0070F0EBF0023C3F1080349
:1092600003F007031944D21A8161C26042F001037E
:109270004B60091D28238B50DFF80C170A69C26167
:1092800070472DE9FC4B074601F1080010F0070F6D
:109290000FBF8946C0F1080000F0070001EB00098C
:1092A00002F1080111F0070F06D002F10800C0F129
:1092B000080000F0070002441546A5EB090009EB81
:1092C0000306A0EB030B43F00303C9F80430AE42DE
:1092D00028BF01F0FFF92879C10758BF01F0FAF95A
:1092E000BBF1100F38BF01F0F5F9B869854207D11D
:1092F000F8685844F860BE6140F00100706050E1C9
:10930000786985420AD1B8688344C7F808B07E619D
:109310004BF00100706046F80BB042E1686800F065
:109320000301012940F0AB80C008C0000190C008D3
:109330001F2839D8AC68D5F80C800090454508BF87
:1093400001F0C8F9A54208BF01F0C4F968680099A6
:10935000C008C000B0EBC10F18BF01F0BBF9009905
:1093600007F1280000EBC100844206D03A6994421C
:10937000C0F08080E168A9427CD1A04506D1009868
:109380003968012282409143396075E0804506D0FA
:10939000386980456ED3D8F80800A8426AD1C4F86D
:1093A0000C80C8F8084067E0EC68D5F81880AC423B
:1093B0000CD0A8683969884222D3C168A94204BF89
:1093C000A168A9421CD1C460A0601BE005F1140291
:1093D000146834B905F1100214689CB101E01A4612
:1093E000146804F114031968002902BF04F1100382
:1093F00018680028F3D139698A4228BF106001D269
:1094000001F068F9B8F1000F36D0E96907F59870F6
:1094100000EB81000268954208D10460A4B9E869B4
:109420007968012282409143796025E0386980455E
:1094300008D3D8F81000A84214BFC8F81440C8F8E0
:10944000104001E001F046F9B4B139698C4211D302
:10945000C4F81880286928B1884226BF2061846139
:1094600001F038F9686938B13969884202D360611E
:10947000846101E001F02EF901982D188344686899
:109480004008400068604BF0010171604FEADB0466
:1094900046F80BB01F2C23D807F1280000EBC408B6
:1094A0004546BBF1100F38BF01F014F9386820FAB7
:1094B00004F1C90705D4012101FA04F404433C6016
:1094C00007E0D8F80800396988422CBF054601F04A
:1094D00001F9C8F80860EE60B560C6F80C8060E07D
:1094E0005FEA1B2008BF002123D0B0F5803F28BFD2
:1094F0001F211ED2A0F58072120C02F008029040CB
:10950000A0F58051090C01F004018840A0F58043CA
:109510001B0CC2F10E0203F00203521AD21A984039
:1095200002EBD032D01D2BFA00F101F0010101EB6A
:10953000420107F5987202EB8100F161002272612D
:1095400032617A6822FA01F3DB0707D4012303FAB8
:1095500001F1114379600660B0611DE002681F29C6
:109560001DBF4908C1F119010BFA01F1594600E08C
:1095700002465068C008C000584516D002F11003DA
:10958000CC0F03EB8403490018680028F0D1386938
:10959000834204D31E60B261F660B66001E001F060
:1095A00099F809F10800BDE8F68B396990688A429C
:1095B00028BF8842F3D3C6609660B060F260002096
:1095C000B061EEE72DE9FE4F04468B46A5692E46B5
:1095D000904699463146FFF713FEA8F1280201682C
:1095E000406801EB000AAAF1270111F007000EBF45
:1095F0000021C1F1080101F007010AEB0100A0F10F
:109600002F0706F11000874238BF374607F11800D0
:1096100001905946002000902046FFF719FE07F1FF
:10962000080010F0070F18BF01F054F81B207860F5
:1096300007F1080104F5E07090E80C5081E80C5047
:10964000C0F800B0C0F80480C0F80C9081600198A8
:10965000009900E0001D07224260491C00F1080249
:109660005245F7D30129D8BF01F034F8B74200F0D2
:109670009580BF1B301D311DC05940084000C851A6
:1096800047F0010171604FEAD70BF751BBF11F0F93
:1096900021D804EBCB0000F12805A846102F38BFD5
:1096A00001F018F8206820FA0BF1C90705D4012150
:1096B00001FA0BF10843206006E0A868216988429E
:1096C0002CBF804601F006F8AE60C8F80C60C6F802
:1096D0000880F5606FE0380A08BF002123D0B0F59C
:1096E000803F28BF1F211ED2A0F58072120C02F00D
:1096F00008029040A0F58051090C01F00401884057
:10970000A0F580431B0CC2F10E0203F00203521AB3
:10971000D21A984002EBD032D01D27FA00F101F0A6
:10972000010101EB420104EB8102002302F5987074
:10973000F16173613361626822FA01F3DB0707D4D8
:10974000012303FA01F1114361600660B0611DE07D
:1097500002681F291DBF4908C1F1190107FA01F16B
:10976000394600E002465068C008C000B84216D032
:1097700002F11003C80F03EB8003490018680028AA
:10978000F0D12069834204D31E60B261F660B560F7
:1097900011E003B0BDE8F04F00F09CBF0BE0216981
:1097A00090688A4228BF8842F3D3C6609560B06053
:1097B000F2600020B06103B0BDE8F08F2DE9F04108
:1097C000714F05463868884608B9FFF728FDB96823
:1097D00001EB08002F30491E20EA010188457DD2A7
:1097E00005F5D876B06828B1326889188A4275D2F2
:1097F000884273D300F0AEFF01001CBF0C6811F16A
:10980000010F6BD03068201805F5D87230605368AE
:10981000984238BF18467060A86960BB286908B1D3
:10982000814200D22961316174610020F06105F14B
:109830002802386868624FF0FF3028620020D2604A
:10984000926002F1080353611361801C10322028DA
:10985000F5D34E48854208BFA4F1280228D055F818
:10986000040CC00805EBC002A2F108000A19121A84
:10987000283A01461CE005F5E070024600E09268D7
:109880007AB3136857683B449942F8D1137B1F079A
:1098900027D4AB691768BB4223D3D2F804C067440E
:1098A000BB421ED2A444C2F804C0E868A9692218C9
:1098B0002846FFF7CDFC1FE08068C0B103689342E3
:1098C000FAD1027B130712D4026801604368E418DE
:1098D000446043462846BDE8F041D2E40020BDE89C
:1098E000F0812A69914238BF29610A19E5E700230E
:1098F00022462846FFF766FEE8688045EED2A0EBD8
:109900000800A969E86001EB0802AA6140F00100C3
:10991000506048F00300486001F10800BDE8F081A4
:1099200038B4194B1A6882B94FF480525A604FF418
:1099300080344FF0FF329C60DA601A610422134CCD
:10994000134D5A61C4F8BC211D6011F1400F17D2AC
:109950008269AAB1C368283199420BD200F5E0713F
:109960000C68A24203D34D682C44A24202D38968FA
:109970000029F5D1C16999423CBF4FF0FF31C16167
:1099800032BC002070470000E85E0020AC5500208B
:109990006859883C2DE9F84F00258946090AC9F124
:1099A000000B08BF002323D0B1F5803F28BF1F2341
:1099B0001ED2A1F58072120C02F008029140A1F5AE
:1099C00080531B0C03F004039940A1F58044240C40
:1099D000C2F10E0204F00204D21A121BA14002EBE3
:1099E000D132D11D29FA01F303F0010303EB420345
:1099F000074607F5987858F8230030B31F2B0FBFA0
:109A00004C465C08C4F1190409FA04F4AC46594602
:109A100000E064004268D208D200A2EB09028A4248
:109A200003D21100054600F06881426910304FEA08
:109A3000D47B50F82B00002A1CBF82429446002899
:109A4000E7D18B466046B0BBBDBB012000FA03F3F3
:109A50005B00584203437868034000F04D81584250
:109A600003405B1E180B00F01000C340590901F0C1
:109A70000801CB409A0802F00402D3405C0804F0CD
:109A800002040818E3401018C3F3400620183044BD
:109A9000F3401B1858F823000DE008464168C90838
:109AA000C900A1EB090159453CBF8B460546016938
:109AB0000029F2D140690028F0D1002D00F01C816E
:109AC000B868A0EB0900834580F0168138698542AB
:109AD000C0F010816868C008C00009EB0B01884223
:109AE00018BF00F0F7FD05EB0906B54280F00281D2
:109AF000EC68D5F818A0AC420CD0A8683969884247
:109B000022D3C168A94204BFA168A9421CD1C46084
:109B1000A0601BE005F11402146834B905F11002CD
:109B200014689CB101E01A46146804F11403196822
:109B3000002902BF04F1100318680028F3D1396925
:109B40008A4228BF106001D200F0C4FDBAF1000FB4
:109B500036D0E96908EB81000268954209D10460BA
:109B6000200014D1E869796801228240914379602C
:109B700026E03869824508D3DAF81000A84214BFFD
:109B8000CAF81440CAF8104001E000F0A3FDBCB1CF
:109B90003869844212D3C4F818A0286930B13969F1
:109BA000884226BF2061846100F094FD686938B165
:109BB0003969884202D36061846101E000F08AFD66
:109BC000BBF1100F0CD2D94449F003006860291D85
:109BD000281D50F8090040F0010041F8090088E014
:109BE00049F0030068604BF0010070604FEADB0051
:109BF00046F80BB01F281DD807EBC00101F128045F
:109C0000396821FA00F2D207A34605D4012202FAEC
:109C100000F00843386006E0A068396988422CBF2C
:109C2000834600F057FDA660CBF80C60C6F808B07C
:109C3000F4605EE05FEA1B2008BF002123D0B0F58E
:109C4000803F28BF1F211ED2A0F58072120C02F0A7
:109C500008029040A0F58051090C01F004018840F1
:109C6000A0F580431B0CC2F10E0203F00203521A4E
:109C7000D21A984002EBD032D01D2BFA00F101F03D
:109C8000010101EB4201F16100227261326108EBD6
:109C900081007A6822FA01F3DB0707D4012303FA73
:109CA00001F1114379600660B0611DE002681F296F
:109CB0001DBF4908C1F119010BFA01F1594600E035
:109CC00002465068C008C000584518D002F1100381
:109CD000CC0F03EB8403490018680028F0D13869E1
:109CE000834204D31E60B261F660B66001E000F00A
:109CF000F1FC13E100F0EEFC0DE18B46A3E63969BF
:109D000090688A4228BF8842F1D3C6609660B060EE
:109D1000F2600020B061ECE72DE9F84F0646884676
:109D2000716848420140491E080B00F01000C14014
:109D30004A0902F00802D1408B0803F00403D9401D
:109D40004D0805F002051018E9401818C1F3400449
:109D5000281806F5987A2044E14009185AF821108D
:109D60004868C008C0000D46A0EB080909E001469C
:109D70004868C008C000A0EB080048453CBF8146C9
:109D80000D4608690028F2D149690029F0D13069EF
:109D90008542C0F0BE806868C00808EB090BC000AF
:109DA000584518BF00F096FC05EB0800854200906E
:109DB00080F0AF80EF68AC69AF420CD0A868316921
:109DC000884222D3C168A94204BFB968A9421CD104
:109DD000C760B8601BE005F11402176837B905F1D8
:109DE000100217689FB101E01A46176807F11403C3
:109DF0001968002902BF07F1100318680028F3D181
:109E000031698A4228BF106001D200F063FC002C47
:109E100031D0E9690AEB81000268954208D10760F8
:109E20008FB9E8697168012282409143716022E034
:109E30003069844205D32069A84214BF6761276155
:109E400001E000F047FCB7B13069874211D3BC6133
:109E5000286930B13169884226BF3861876100F0D6
:109E600039FC686938B13169884202D37861876109
:109E700001E000F02FFCB9F1100F0BD24BF0030002
:109E80006860291D281D50F80B0040F0010041F8C2
:109E90000B003DE048F00301696049F00100291D15
:109EA00041F80800009840F80990D6F808804FEA79
:109EB000D80BBBF1200F28BF00F00CFCB8F1000F4D
:109EC00022D006EBCB00776900F12804A246B8F156
:109ED000100F38BF00F0FEFB306820FA0BF1C90705
:109EE00005D4012101FA0BF10843306006E0A068B7
:109EF000316988422CBF824600F0ECFBA760CAF8AB
:109F00000C70C7F808A0FC60C6F808900098706153
:109F100004E000F0DFFB0020BDE8F28F05F108004F
:109F2000BDE8F28F2DE9FE4F0546AFF30080F52D19
:109F3000DFF89C6780F004810B2D31BF10250B35B5
:109F4000ED08ED003068EC08E04010F0030F46D05B
:109F5000C04300F00100041906F1280000EBC4081A
:109F6000E700D8F808506868C008C000B84218BFB9
:109F700000F0B0FBD5F80890454508BF00F0AAFBFB
:109F80004D4508BF00F0A6FB6868C008C000B84295
:109F900018BF00F09FFBC84507D13168012000FAC7
:109FA00004F421EA040434600DE03069814508D3EB
:109FB000D9F80C00A84204D1C8F80890C9F80C8060
:109FC00001E000F087FB47F003006860291D281DB1
:109FD00005F10804C05940F00100C851F8E0B1682B
:109FE000A94280F0BE80002800F0A1804FF0010857
:109FF00008FA04F1490000FA04F4484201430C4015
:10A0000060420440641E200B00F01000C44061094F
:10A0100001F00801CC40A20802F00402D440630819
:10A0200003F002030818DC401018C4F340071818A6
:10A030003818FC40241806F1280000EBC40AE70099
:10A04000DAF80890D9F80400C008C000B84218BF78
:10A0500000F040FBD9F808B0D14508BF00F03AFB4A
:10A06000D94508BF00F036FBD9F80400C008C0008D
:10A07000B84218BF00F02EFBDA4506D1316808FA65
:10A0800004F421EA040434600DE03069834508D308
:10A09000DBF80C00484504D1CAF808B0CBF80CA096
:10A0A00001E000F017FB45F00300C9F804007F1B36
:10A0B00009F1040147F00100485109EB0500019046
:10A0C000C751B4684FEAD40ABAF1200F28BF00F094
:10A0D00001FB34B3CDF800A006F12800756900EB50
:10A0E000CA0AD346102C38BF00F0F4FA3168009841
:10A0F00021FA00F2D30704D408FA00F008433060D4
:10A1000007E0DAF80800316988422CBF834600F086
:10A11000E1FACAF80850CBF80C50C5F808B0C5F8F9
:10A120000CA0B76009F108040198706150E07068F4
:10A13000C0B329463046FFF7EFFD040011D047E0D9
:10A1400015F1400F28BF4FF0FF350AD20B35ED084F
:10A150007068ED0028B129463046FFF71BFC04006B
:10A1600036D1B068A8421DD3411B726910290AD3A9
:10A1700050197061B16041F001034360415045F0F6
:10A18000030555600BE00021B1607161131D40F0C3
:10A1900003015160111D095841F00101195002F1EC
:10A1A000080415E0F06885420DD2401BB169F060EB
:10A1B0004A19B26140F00100506045F003054D605E
:10A1C00001F1080404E029463046FFF7F7FA044697
:10A1D000AFF300802046FFF7EEBA002800D17047A9
:10A1E0002DE9FC47A0F10805AFF30080DFF8E0643B
:10A1F00032699542C0F05982686800F00301012974
:10A2000000F05382C1084FEAC109C10705EB0908F4
:10A2100039D42C6810F0030F00F0498260420544E5
:10A220009542A144C0F041827069854200F0C78028
:10A23000E408202C5ED2D5F80CA0AF68554508BFC5
:10A2400000F048FABD4208BF00F044FA6868C00850
:10A25000C000B0EBC40F18BF00F03CFA06F12800B4
:10A2600000EBC400874205D031698F423FD3F968C3
:10A27000A9423CD1BA452CD13068012101FA04F43D
:10A2800020EA04043460454580F00F82D8F8044089
:10A29000E00740F10A82A00700F16881B0698045BB
:10A2A00040F0A080F068B5618144C6F80C9049F098
:10A2B000010068607069854202D100207061B06061
:10A2C000F069484580F0F38100213046FFF728FB14
:10A2D000EDE1824506D03069824508D3DAF80800FE
:10A2E000A84204D1C7F80CA0CAF80870CBE700F068
:10A2F000F1F9C8E7EC68AF69AC420BD0A8689042AE
:10A3000023D3C168A94204BFA168A9421DD1C4607A
:10A31000A0601CE005F114031C6834B905F11003BA
:10A320001C68A4B101E063461C6804F1140CDCF85D
:10A330000010002902BF04F1100CDCF80000002816
:10A34000F1D1934228BF196001D200F0C3F9002F68
:10A3500099D0E96906F5987000EB81000268954292
:10A3600009D10460200011D1E8697168012282409E
:10A370009143716087E73069874205D33869A84205
:10A3800014BF7C613C6101E000F0A4F9002C3FF4B3
:10A390007AAF31698C42AAD3A761286928B1884273
:10A3A00026BF2061846100F095F9686900283FF4B8
:10A3B0006AAF316988429AD36061846163E798F833
:10A3C000040000F0030003287FF45DAFC6F8089096
:10A3D00049F00101D8F8040040084000C8F8040022
:10A3E00069600AE0706980450AD1B068756181448E
:10A3F000C6F8089049F00100686045F8099056E1F8
:10A40000E408E400A144E408202C3AD2D8F80CA0D7
:10A41000D8F80870D04508BF00F05CF9B84508BF0F
:10A4200000F058F9D8F80400C008C000B0EBC40F21
:10A4300018BF00F04FF906F1280000EBC400874276
:10A4400007D031698F42C0F08480F968414540F0FF
:10A450008080BA4507D13068012101FA04F420EA6E
:10A460000404346077E0824506D031698A4570D3B0
:10A47000DAF8080040456CD1C7F80CA0CAF808709B
:10A4800069E0D8F80C40D8F8187044450DD0D8F8D9
:10A4900008003169884222D3C168414504BFA168E0
:10A4A00041451CD1C460A0601BE008F1140214688F
:10A4B00034B908F1100214689CB101E01A4614681E
:10A4C00004F114031968002902BF04F1100318688D
:10A4D0000028F3D131698A4228BF106001D200F010
:10A4E000F9F8002F37D0D8F81C1006F5987000EB5B
:10A4F0008100026890450AD10460200012D1D8F88A
:10A500001C007168012282409143716023E0306930
:10A51000874205D33869404514BF7C613C6101E046
:10A5200000F0D8F8BCB131698C4212D3A761D8F8D9
:10A53000100028B1884226BF2061846100F0CAF86B
:10A54000D8F8140038B13169884202D3606184615F
:10A5500001E000F0BFF849F00100686045F809909B
:10A56000706985420BD1C6F80890A0E064086400C9
:10A57000C8F8044049F00100686045F809904FEAC6
:10A58000D907202F22D206F1280000EBC704A046ED
:10A59000B9F1100F38BF00F09DF8306820FA07F1CC
:10A5A000C90705D4012101FA07F70743376006E020
:10A5B000A068316988422CBF804600F08BF8A56006
:10A5C000C8F80C50C5F80880EC6070E05FEA19200C
:10A5D00008BF002123D0B0F5803F28BF1F211ED225
:10A5E000A0F58072120C02F008029040A0F5805194
:10A5F000090C01F004018840A0F580431B0CC2F156
:10A600000E0203F00203521AD21A984002EBD03223
:10A61000D01D29FA00F101F0010101EB420106F51C
:10A62000987202EB810000226A612A61E961726816
:10A6300022FA01F3DB0707D4012303FA01F11143E6
:10A6400071600560A8611DE002681F291DBF4908EF
:10A65000C1F1190109FA01F1494600E002465068CA
:10A66000C008C000484526D002F11003CC0F03EB10
:10A670008403490018680028F0D13069834204D36C
:10A680001D60AA61ED60AD6001E000F023F8306A62
:10A69000401E30620BD1D6F8C80100E08068002867
:10A6A000FCD14FF0FF30306201E000F013F8AFF35F
:10A6B0000080BDE8F387316990688A4228BF8842EC
:10A6C000E3D3C5609560A860EA600020A861DEE77A
:10A6D000AC550020012000F053B8F0B402461068D9
:10A6E00095681318506803EB5004C00721D54D44FA
:10A6F0001FE0F0BC02F10C00704713F8017B05F875
:10A70000017B491EF9D1A0B1B60813F8011B06F070
:10A710000306032E08BF13F8016B01EB0621494223
:10A72000801C294405D011F8016B05F8016B401E0F
:10A73000F9D1A342DDD013F8016B16F0030104BF79
:10A7400013F8011BC91C30090F28DAD113F8010BCB
:10A750000F30D6E70749086808B10020704706485F
:10A76000C008C00008600549C908C900091A01608D
:10A77000704700BF1C6000203F90002038B00020D0
:10A780002021090326311820ABBEF9E700000000A4
:10A7900028B100BF02A1800141F0010108477047C4
:10A7A0000338FDD87047000010B5040005D04FF401
:10A7B0007A70FFF7EDFF641EF9D110BDF8B50446BD
:10A7C0000F461546002611E014F8010F70B1384607
:10A7D00001F044F802463946204601F05AF80028B4
:10A7E000F2D12070384601F039F80444207890B155
:10A7F000711C22280BD1601C45F826000E46222130
:10A8000001F078F8040006D000202070DCE745F85D
:10A8100026400E46D8E73046F2BD10B5044601F09A
:10A820001DF8401E06D4215C0D2912BF0A29002103
:10A830002154F6D0002010BD0CB410B5C0B00446B1
:10A840000A4642AB4FF48071684601F071F8014648
:10A850001CB9684601F020F908E0012C04D1002160
:10A86000684601F00DFC01E04FF0FF3040B010BC35
:10A870005DF80CFB012908BF0FF2100101D009B9E6
:10A8800006A1D9E74FF0FF30704700004F4B20255D
:10A8900073203A2025730D0A000000004552524FE4
:10A8A00052202573203A2025730D0A000A4600BF66
:10A8B00000A1C1E74552524F52202573203A20494A
:10A8C0006E76616C696420506172616D6574657249
:10A8D0000D0A00000A4600BF00A1ADE74552524FE5
:10A8E00052202573203A2046756E6374696F6E207E
:10A8F0004661696C7572650D0A00000080B518B973
:10A90000BDE8024001F0E1BD012908BF4FF0FF3072
:10A9100004D0022906D1506802F06AF8BDE802406E
:10A9200001F060BE4FF0FF3002BD000070B504467C
:10A9300002F09CF80546DFF8486B02F097F8401BE0
:10A94000B0F5FA6F06D296F8040118B16420FFF74B
:10A950002BFFF2E702F0A8F802A100F03DF9002079
:10A9600070BD0000646675206F6B0D0A000000006A
:10A9700070B501290446154602D102F0FFF852E0F5
:10A980000229AAA621D16868A9A102F01DF918B967
:10A99000204602F012FA46E06868314602F014F9E7
:10A9A00028B9204602F0F3F8012C3CD126E0686873
:10A9B00001783039042936D202F01AF8042832D24C
:10A9C0000146204602F0BAFA2DE003292BD168682F
:10A9D000314602F0F9F8A0B9A8681022002102F06F
:10A9E0000CF80446200403D0A1B2002002F039FA8A
:10A9F000240C03D02146012002F033FA02F08FFA32
:10AA000011E0012655F8260001783039042907D2D3
:10AA100001F0EEFF042803D20146204602F08EFA30
:10AA2000761C022EEEDD002070BD7CB500280D46A0
:10AA3000144630D1012DDFF8546A0DD13088F189E8
:10AA4000451CA942B8BFB589294602B0BDE870408F
:10AA50000246002002F070BC022D0BD1606801F0AC
:10AA6000C7FF0546B0898542A4BFF089A84263DBD1
:10AA70002846E9E7032D5FD1606801F0B9FF00F0D7
:10AA80001FFAB1898D42A2BFF289AA42884253DBE4
:10AA90008242D9DA50E0022D4EDB66680FF62C2197
:10AAA00000F012FAF8B9022D0DD0032D0FD1A468D1
:10AAB0000FF6102100F0C0F810B902F049FD04E0D3
:10AAC000204601F095FF02F027FD002076BD042D01
:10AAD00032D1E06801F08CFF00F0F2F92946BDE8C0
:10AAE0007C4002F0F8BC022D06D1304601F080FF18
:10AAF000BDE8764002F099BC032D08D1304601F044
:10AB000077FF00F0DDF94FF0FF3201460EE0042D33
:10AB100012D1304601F06CFF00F0D2F90646E06831
:10AB20001022002101F069FF02463146284602B09A
:10AB3000BDE8704002F00BBC4FF0FF3076BD38B579
:10AB400001290446154602D102F0CEFD42E0022959
:10AB500023D16D6837A100F039FB50B902F071FFC5
:10AB600000280CBF0FF66C110FF68C1100F034F8B2
:10AB700030E0287830380A282CD2284601F038FFF7
:10AB80000546002180B202F021FF00282A4614BFAA
:10AB90000FF6A4110FF67C1119E003291AD1686889
:10ABA000BEA102F011F8A8B9A868017830390A29C5
:10ABB00010D201F01DFF0546002180B202F022FFF5
:10ABC00000282A460CBF0FF68C110FF6AC11204658
:10ABD000FFF732FE002032BD20462DE61CB50129CC
:10ABE00005D102F081FD01F035FD002016BD0229DE
:10ABF00018D15468AAA100F01FF810B902F074FD32
:10AC0000F3E70FF6B00100F017F80028EBD0A5A18C
:10AC100000F012F830B902F067FD01F01BFD01F001
:10AC20001AFDE2E74FF0FF3016BD00002D6F000067
:10AC30002D6400002D630000204601F0C5BF2DE902
:10AC4000F8410F46012FA1B040F3EE801446804634
:10AC5000666895A100F038F9002842D1042F93A628
:10AC600038D1A06803236A4691A1FFF7A7FD032806
:10AC700040F0ED80009801F0BBFEB0F5FA6FA8BF80
:10AC8000A0F5FA600890019801F0B2FE401E07900E
:10AC9000029801F0ADFE06900323E0686A4685A1A4
:10ACA000FFF78CFD03286DD1009801F0A1FE0590FF
:10ACB000019801F09DFE0490029801F099FE039026
:10ACC00003A802F0DDFF002840F0E18003F052F914
:10ACD0000346D2E0022F55D103F030F80FF6B0034F
:10ACE000CBE075A100F0F0F80028DFF8A85735D1C7
:10ACF000032F72A646D1A468204600F0AFFD20289D
:10AD000046D22021684603F099F92146684603F0AF
:10AD1000A7F9694605F11B0003F0A2F9684601F0A6
:10AD200039FA03F0E2F90446012C08BF03F0D1F927
:10AD3000684601F0C3FC002806D46B463246012168
:10AD40004046FFF797FD03E031464046FFF7C2FD5E
:10AD5000012C02D1012003F0ADF99CE00FF25471F7
:10AD600000F0B2F830B901F03BFB0FF638030FF6F4
:10AD70002C0283E00FF6340100F0A6F878B9032F17
:10AD80000FF6300663D1A06801F032FE0328009070
:10AD90005DD201226946002001F0DCFC53E00FF691
:10ADA0001C0100F091F8F8B9032F0FF618064ED1E8
:10ADB000A06801F01DFE4FF0FF310091421F1A2ADA
:10ADC000694605D201236B76E8650093486006E08A
:10ADD00000283CD16876E865002200904A60022293
:10ADE000012001F0B7FC2EE00FF2E07100F06CF8EA
:10ADF000002831D1052F0FF2DC7628D1E0686946B2
:10AE000003F092F9206901A903F08EF90746002F9B
:10AE100006DD394601A803F0C4F90099814208D043
:10AE200031464046FFF742FD4FF0FF3022B0BDE80B
:10AE3000F081E06801F0DCFD00F042F83B4601AA39
:10AE4000294601F0C7FC002821D4A36815E031464B
:10AE50004046FFF72BFD1EE00FF2807100F034F842
:10AE60000028E1D1032F0FF27C760CD1A468204694
:10AE700001F0C7FC00280AD423463246012140468F
:10AE8000FFF7F8FC07E0022FCAD1B4A4EFE7314680
:10AE90004046FFF71FFD0020C8E700002D620000BC
:10AEA00065780000616C6C0072746300525443005A
:10AEB0002D0000003A0000006964000049440000D1
:10AEC0000546A06801F094BD304601F07DBE78B51E
:10AED0000229A1B0044633D155680FF21071DFF892
:10AEE000B46500F073F960BB19A801F0F7FB00210D
:10AEF00011A803F077F909A803F092F90322B1A190
:10AF000006A803F007FA07220FF2E86107A803F08A
:10AF100001FA03F02FF8034606A907A8049105904B
:10AF200009AD316EDFF8700502680391029211A934
:10AF30000091019519AA0FF2C4612046FFF77CFC2D
:10AF4000C4E0BAA100F042F928B903F013F80246B0
:10AF50000FF2C86170E0B6A100F038F980B9684618
:10AF600001F0BCFB0028EBD1B2A1684601F02CFE39
:10AF700010B9684603F054F96A460FF2B0619CE0DC
:10AF8000ADA100F023F938B90021684603F02AF991
:10AF90006A460FF2A86190E00FF2B06100F016F976
:10AFA00030B9684603F03CF96A460FF2A86184E0C4
:10AFB0000FF2B46100F00AF918B9204603F009FA5B
:10AFC00084E00FF2AC6100F001F918B9204600F0FE
:10AFD000D9FD7BE00FF2A06100F0F8F810B90FF294
:10AFE000A0615AE00FF2C45100F0F0F890B90122CC
:10AFF000694601F09DFB002809D4009810F1010F6B
:10B0000004BF01210091009A0FF2886114E00FF251
:10B01000A45158E000F0D8F8A8B9022269460120EE
:10B0200001F086FB00280BD4009901291CBF0022E7
:10B030000192019A0FF26C612046FFF7FDFB45E09B
:10B040000FF280513FE00FF26C6100F0BFF838B9A9
:10B05000307E002814BF0FF278610FF260611CE0AF
:10B06000C5A100F0B3F888B902A803F074FBBDF8DD
:10B070001400BDF8121001900091BDF81030029A32
:10B080000FF260612046FFF7D7FB1FE00FF26C6103
:10B0900000F09CF820B90FF27061FFF79DFD15E0FC
:10B0A0000FF2385100F092F880B9684601F0BAFB0F
:10B0B000002806D46A460FF264612046FFF7BCFB05
:10B0C00004E00FF220512046FFF704FC002022B0DC
:10B0D00070BD03F011BC38B50129144602D103F04C
:10B0E00007FD29E0022914D16068BEA101F06CFDC2
:10B0F00010B903F000FD1FE06068017834390229BF
:10B100001AD201F075FC011F022915D203F012FDBD
:10B1100012E0032910D1012554F8250001783439B3
:10B12000022906D201F064FC011F022938BF03F096
:10B1300001FD6D1C022DEFDD002032BDBFF34F8FEE
:10B14000DFF85813DFF858030A6802F4E06202439C
:10B150000A60BFF34F8F00BFFDE700000000000052
:10B1600080B5012002F0A6FF002002BDF8B502293B
:10B17000044624D155680FF2443100F027F8F0B1AD
:10B180000FF230510FF2AC56C24F00F01FF820B949
:10B19000387633460FF294520DE000F015F870B98E
:10B1A000012000900122694601F0D4FA012078764E
:10B1B00033460FF2104201212046FFF75BFB0020CF
:10B1C000F2BD0000344700000FF2F031284601F0D4
:10B1D000FBBCF8B50229044625D155680FF2DC21E5
:10B1E000FFF7F4FFF8B10FF2CC410FF25056A94F20
:10B1F000FFF7ECFF28B90120387633460FF22C52C6
:10B200000DE0FFF7E1FF70B90090012269460120CF
:10B2100001F0A0FA0020787633460FF2A83201211F
:10B220002046FFF727FB0020F2BD00007274630088
:10B2300069640000585858006370750070B504299F
:10B24000A0B014460FD1606801F0D2FBFFF738FEC2
:10B2500000EB0536E068694602F066FF82B2694697
:10B26000304602F014FC002020B070BD2DE9F04102
:10B270000129054602DC4FF0FF300DE0506801F077
:10B28000B7FB04000AD103F033FD22460FF2D04190
:10B290002846FFF7D1FA0020BDE8F081012C04D147
:10B2A00003F013FD03F016FDEFE7022C04D103F0C9
:10B2B0000CFD03F016FDE8E7032C41F2813641F264
:10B2C000941740F2A46817D103F0FFFC03F002FDCD
:10B2D0004046FFF75DFA03F0FFFC4FF44870FFF7BC
:10B2E00057FA03F0FEFC3846FFF752FA03F0F2FC7F
:10B2F0003046FFF759FAC6E7042C14D103F0E5FCF9
:10B3000003F0EFFC4046FFF743FA03F0ECFC4FF488
:10B310004870FFF73DFA03F0DDFC3846FFF738FAD6
:10B3200003F0DFFCE4E722460FF21C412846FFF75A
:10B3300083FAA0E780B500F021FF002002BD2DE9CF
:10B34000FC41054600240FF22848564E4DA70C201C
:10B35000604332584AB1002C12BF41463268394628
:10B360002846FFF769FA641CF1E747A12846FFF772
:10B3700063FA0020BDE8F681626174002DE9F843AC
:10B380000446894616469846002500E06D1C0C20B0
:10B39000684308EB00073968F9B1306801F014FC24
:10B3A0000028F3D16CB9387901280FD102F091FE51
:10B3B000BB68324649460020984733A000F05BFB4B
:10B3C00009E07879012808BF02F083FEBB683246A5
:10B3D000494620469847002001E04FF0FF30BDE885
:10B3E000F28300002D61000038B504468AB00D4696
:10B3F000012C01BF2878422869784D2904D12946BB
:10B40000012003F0F9FC39E02846FFF706FA002C8A
:10B4100029460CBF0FF260300FF2683000F02BFBB2
:10B420000A236A461AA12846FFF7C8F90546009A7A
:10B430000FF26030294600F01EFB002D1EDD194B77
:10B4400000F034F8002819D5174803681BB100F044
:10B450002DF8002812D5009800F000FA02280DD32C
:10B460000FF23C31FFF7B8FB009A0FF2883120460B
:10B47000FFF7E2F90FF29031FFF7AEFB0BB030BDF2
:10B480001C350020257300000D0A0000005F00201D
:10B490002000000044320020B02F00200CED00E01E
:10B4A0000400FA059C300020046000206A4629460A
:10B4B000204663E774646174610000007364617422
:10B4C0006100000064697361626C65007374726589
:10B4D000616D0000573235513235364A562C207393
:10B4E00075636365737366756C6C792065726173DF
:10B4F00065642E0D0A000000573235513235364A48
:10B50000562C206E6F74206572617365642E0D0A6F
:10B5100000000000536563746F722025642C207353
:10B5200075636365737366756C6C7920657261739E
:10B5300065642E0D0A000000536563746F72202548
:10B54000642C206E6F74206572617365642E0D0A21
:10B5500000000000426C6F636B2025642C20737523
:10B56000636365737366756C6C792065726173656E
:10B57000642E0D0A00000000426C6F636B2025648E
:10B580002C206E6F74206572617365642E0D0A0045
:10B59000436C65617265642E0000000054444154A0
:10B5A0004100000053617665640000006D6F6465C2
:10B5B000000000004D4F44450000000070617573AD
:10B5C0006500000050415553450000006463666704
:10B5D0000000000044434647000000006E616D65B6
:10B5E000000000004E414D4500000000696E666F8E
:10B5F000000000003530304450530000494E464FA3
:10B600002C25732C25732C25732C25732C25733A2C
:10B6100025732C25732C2573000000004F4B2052FE
:10B620005443203A2025730D0A0000004F4B204957
:10B6300044203A2025730D0A000000004F4B2043A0
:10B640005055203A2025730D0A0000006370755F85
:10B65000696400004F4B204350555F4944203A2015
:10B6600025730D0A000000006661756C740000000F
:10B67000756172740000000074696D6572000000ED
:10B680004F4B2054494D4552203A203130300D0A5D
:10B69000000000004F4B204D4F4445203A202564C8
:10B6A0000D0A00004F4B205041555345203A2025AC
:10B6B000640D0A0074726967676572004F4B20540D
:10B6C000495252474552203A204F4E0D0A00000081
:10B6D0004F4B2054524947474552203A204F464647
:10B6E0000D0A00004F4B20424154203A202564208F
:10B6F00025642025642025640D0A000061637475AB
:10B7000061746F72000000004F4B2041435455415B
:10B71000544F52203A2023310D0A00004F4B204E47
:10B72000414D45203A2025730D0A000054524947E7
:10B7300047455200454E41424C454400444953411F
:10B74000424C454400000000696E76616C696420DB
:10B75000666972655F6D6F646520282564290A003B
:10B7600066697265203A206F6B282564290A0000FB
:10B770002C202573000000003E3E2025730D0A0D8D
:10B780000A000000424C453E3E2025730D0A0D0A7A
:10B79000000000002564202D3E2025730D0A0000C6
:10B7A0000D0A2D2D2D2D2D2D2D2D2D2D2D2D2D2D0C
:10B7B0002D2D2D2D2D2D2D2D2D2D2D2D2D2D2D2DB9
:10B7C0002D2D2D2D2D2D2D2D2D2D2D2D2D2D2D2DA9
:10B7D0002D2D2D2D2D2D2D2D2D2D2D2D2D2D2D2D99
:10B7E0002D2D2D2D2D2D2D2D2D2D2D2D2D2D2D2D89
:10B7F0000D0A00002573203A206E6F742064656680
:10B80000696E65642E0D0A0023232323232323233B
:10B8100023232323232323232323232323232323F8
:10B8200023232323232323232323232323232323E8
:10B8300023232323232323232323232323232323D8
:10B8400023232323232323232323232323232323C8
:10B850002323232323230D0A0000000000F101030A
:10B86000810704D010F8011B89B18107FAD1026861
:10B87000B2F10131914311F0803F04BF50F8042F21
:10B88000F6E710F8011B11B110F8011BFBE7C01A15
:10B89000704704E010F8013B6BB1491C521E52B1D5
:10B8A0000B7890F800C09C45F4D002D24FF0FF30E6
:10B8B000704701207047002070470B78012B70B54E
:10B8C00005460C460AD140684E6803687168DB681B
:10B8D0009847686803683146DB68984700236868C2
:10B8E0006360C4E90433237003682146DB68BDE864
:10B8F000704018470278C9B28A421AB11CBF10F8CA
:10B90000012FF9E718BF0020704700F5805210B5ED
:10B910005368B3F5806F09DA946800EB8300214423
:10B920000133446091605360002010BD0120FCE7AA
:10B9300008B584B00023039300290EBF0193019042
:10B94000491E0291009301A904AB074878441830BE
:10B9500003F096FA019909B100220A70002858BF35
:10B96000039805B000BD00BF332A000000000000AE
:10B9700010B5040008D000BF99A14FF47A4041F0FF
:10B9800001018847641EF6D110BD38B50178884C96
:10B9900011B1022934D031BD684604F01CFB9DF87A
:10B9A000001082A000F067F8608882499DF80020AE
:10B9B000401C608001F5A1657F2A688802D150B3E0
:10B9C000401E1BE00D2A18BF0A2A0CD100220A547F
:10B9D0000120287004F07EFB00206880606C002845
:10B9E00019DD002116E0B0F5807FA4BF002068803B
:10B9F0006A889DF8000088546888401C688031BDC2
:10BA0000616C082907DA04EBC10200235360491C6A
:10BA100040689060616431BD38B58AB00DF11000A6
:10BA200071A1644C182202F075FC4FF480700190F3
:10BA300004F20C614FF480600291039004F20C5503
:10BA4000009507235C4A694604A804F065FA04F5EA
:10BA5000A06100220A720A604A6018B104F074FB07
:10BA60004FF0FF300BB030BD5248704751490020B5
:10BA700081F8080570470EB400B5C0B0024641AB6E
:10BA80004FF480716846FFF753FF0146684600F0A7
:10BA900003F840B05DF810FB2DE9F041444D064637
:10BAA000686C00288846C8BF002047DCEFF305809B
:10BAB000F8B14048002400F5A06105E0375D02447C
:10BAC000641C82F800714B6044450BDA4A680F68C9
:10BAD000531CB3F5806FA8BF0023BB42EED1A86C06
:10BAE000401CA864002CC4BF062004F0F3FA2046D2
:10BAF00024E02878012803D1A96C491CA9641BE023
:10BB000001202870002700E07F1C47450BDAF05D1C
:10BB100004F020FB0400F7D0A86C401CA86402E0ED
:10BB20000120FFF725FF04F0ADFA0028F8D000202F
:10BB300028700CB9404601E04FF0FF30BDE8F081BD
:10BB400038B51C4C04F5A06507E02868401C286047
:10BB5000B0F5806FA4BF002028602868696888421B
:10BB60000DD0204490F8000104F0F4FA0028ECD045
:10BB70000F48816C491C81644FF0FF3032BD0020BA
:10BB800032BD0000F8B504465FF000050BA6084F73
:10BB900008E007EBC5008368426831462046FEF79F
:10BBA0004BFE6D1C786C8542F3DBF1BD2563000014
:10BBB000945C0020A04700208BB9010055415254ED
:10BBC0005F4552524F52203A2025642C2025640DA7
:10BBD0000A0000000000000000000000000000005B
:10BBE0000338FDD870470000050000000400000085
:10BBF000FFFFFFFFFFFFFFFF0000000000E0D70195
:10BC000010B5040008D00FF2B8714FF47A4041F03B
:10BC100001018847641EF6D110BD00B5C1B01121E5
:10BC20008DF800100246BDA101A804F0A5FA01A8F4
:10BC3000FFF714FE1F28C8BF1F2082B201A9684663
:10BC40007CDF08B14FF0FF3041B000BDE0B5FFF739
:10BC5000E4FF0021CDE900110620ADF80410ADF895
:10BC60000000ADF802004FF4C871ADF80610684648
:10BC70007ADF08B104F0A0FA07BD04F09DBA7CB5E4
:10BC80000546287858BBAA8A1646012E27DDDFF81C
:10BC900040452969204602F02DFB0020A05504F5FF
:10BCA00080720120A98A50711160107990B92078B2
:10BCB00001231371422804BF62784D2A04D10FF288
:10BCC0004850FFF7D8FE05E00A4621460FF25050D3
:10BCD000FFF7D1FEBDE87640022004F0FBB973BD4A
:10BCE0001CB5DFF8F004DFF8F044019001A904F17D
:10BCF000280004F072FA08B104F05EFADFF8DC0400
:10BD00000090694604F10C0004F09EFB08B104F0B9
:10BD100053FA13BD007840B9DFF8BC2410883B21EA
:10BD200076DF002818BF04F047BA704704F044BA21
:10BD300000B587B01C21684602F080F90020009011
:10BD40004FF4A0314FF4F020029001910020032124
:10BD5000ADF80E008DF810008DF80C10DFF880049F
:10BD6000DFF8801405900691684604F06EFC08B177
:10BD700004F022FA07B000BD704730B5DFF8585420
:10BD8000ABB004466C60AC21684602F057F9022063
:10BD90008DF8000000218DF8021006208DF80300B8
:10BDA0000121ADF84C108DF87C1005F13400149091
:10BDB0001FA8DFF834140A78C460012A07BF0023E3
:10BDC000036100210161DFF82414DFF8244481625B
:10BDD0002046694604F01FFD08B104F0EDF9012189
:10BDE000204604F015FD2BB030BD80B50321DFF8EF
:10BDF000000404F085FD18B1BDE8024004F0DCB990
:10BE000001BD38B5DFF8D0530446218828881029B1
:10BE10000ED0112933D013296ED0212960D02229C8
:10BE20004ED03B2972D052296BD056296ED031BDED
:10BE3000DFF8C023116811B9072004F0BFFF0FF22B
:10BE4000F830FFF718FE0FF2805000F069F88FDF2E
:10BE5000010004D00FF2F430FFF70DFE03E00FF203
:10BE60001C40FFF708FEA188298005F1280004F096
:10BE7000C6F908B104F0A0F904F0FEFF31BD0120BD
:10BE800004F09CFF4FF6FF7028800FF21C40FFF774
:10BE9000F2FDDFF8640301686868A96040281CBFF0
:10BEA0004020FFF76AFF44F25061052005F039F8A1
:10BEB000DFF81C13002081F80401FFF796FF31BD65
:10BEC000627AA37AACA1B2A0022A0CBF02460A464B
:10BED000022B08BF01460FF2E830FFF7CCFD31BD61
:10BEE0000FF2E84000F01CF88FDFA8B101460FF216
:10BEF0000840FFF7C0FD31BD0023002285217FDF10
:10BF000007E0002300220021B1DF02E0A088132116
:10BF100076DF08B104F050F931BD00002573000050
:10BF20000188ADF800106946A088704780B505F01B
:10BF3000CDF808B104F040F90020009069460120D6
:10BF400005F062F908B104F037F9684605F0B5F973
:10BF500008B104F031F901BD9F484B8802889A422C
:10BF600002BF0A8840F677239A4202D18988CA1E06
:10BF70004280704710B5A14CA149204605F0F6F962
:10BF800008B104F019F9F721204605F005FA18B1B7
:10BF9000BDE8104004F010B910BD38B504468C4D12
:10BFA00005F23C521021C02005F0BCFA08B104F0A3
:10BFB00003F9FFF7BBFF2046FFF748FEFFF7DAFF64
:10BFC000FFF78EFE4020FFF7D8FEFFF7B1FE0A20F4
:10BFD000FFF716FE05F58270002101808170FFF7E2
:10BFE00004FF002032BD7A4870477948D0F800013C
:10BFF00070477749002081F805017047F0B5044685
:10C00000804815460278C1B00AB908202BE0807834
:10C01000012811D14FF4807301AA204605F0A4FA3B
:10C02000002807DD01AA0A211154401C01ACADF81B
:10C03000000003E000201AE0ADF800100026012DFA
:10C04000654F08D100F015F868B9BDF800000EE0A2
:10C050000120FFF7D5FD00F00CF81328F4D1761C71
:10C06000332EF5D30D2004F06FF84FF0FF3041B0C0
:10C07000F0BD3B886A46214607F10C0004F04DBA3A
:10C0800038B504460D46FFF7E9FB81B22A46204643
:10C09000BDE83840B2E70CB40A4610B54C49044636
:10C0A00091F80401C0B028B9082004F04DF84FF011
:10C0B000FF300EE042AB4FF480716846FFF738FC6A
:10C0C0000028D8BF002004DD81B222466846FFF771
:10C0D00095FF40B010BC5DF80CFB000010B50446A5
:10C0E00086B00020207004A86DDF10B14FF0FF3043
:10C0F00015E09DF811009DF81210039002919DF833
:10C1000013009DF814100190CDF800109DF8153023
:10C110009DF8162087A1204604F02EF8002006B0D6
:10C1200010BD000078B589B08AA02B4D90A6FFF70E
:10C13000A2FC00242246314601A804F01DF801A803
:10C14000FFF78CFBADF800006A462B8801A905F1CA
:10C150000C0004F0E2F948B9641C142CEADB00BFBF
:10C160008EA0FFF788FC00200AB070BD0246214671
:10C1700082A0FFF780FCF2E731000000164800883B
:10C180004FF6FF7290421CBF132176DF704700000C
:10C190003200000080B5FFF740FD002802D54FF0C7
:10C1A000FF3002BD4020FFF7E8FD002002BD084837
:10C1B00090F80411012900D1704780B590F85C0116
:10C1C00074DF4FF4C860FFF7D8FDBDE801400CE60E
:10C1D0001C3500207BBC0100C42F00207FBC010067
:10C1E00015BD01002DBD01003460002079BD0100A6
:10C1F000243600200860002044320020405F0020E8
:10C2000059BF010020360020424C455F4D45534741
:10C21000203A20424D20282564290D0A0000000004
:10C22000424C455F4D455347203A20257320282531
:10C2300064290D0A00000000424C453E3E20636F19
:10C240006E6E65637465642E0D0A00004552524F90
:10C25000523A206661696C656420746F2072657162
:10C260007565737420504859207570646174652831
:10C2700030782578292E0D0A000000005359535FAD
:10C28000424C45203A2050485920757064617465CD
:10C290002072657175657374656420746F20324D0A
:10C2A0006270732E0D0A0000424C453E3E206469C8
:10C2B00073636F6E6E65637465642E0D0A00000013
:10C2C0005359535F424C45203A20504859207570CD
:10C2D0006461746520636F6D706C657465202852AD
:10C2E000582025734D6270732C2054582025734DAF
:10C2F000627073290D0A00004552524F52203A20B5
:10C300006661696C656420746F2061636365707435
:10C3100020706565722773205048592075706461DC
:10C32000746520726571756573742028307825787E
:10C33000290D0A00253032583A253032583A253036
:10C3400032583A253032583A253032583A25303270
:10C35000580000007379735F626C655F7465737475
:10C360002829202D2073746172740D0A00000000CA
:10C37000746573742D25640D0A000000626C655F9E
:10C380006E75735F646174615F73656E64282564A4
:10C3900029202D3E2025640D0A0000007379735F6B
:10C3A000626C655F746573742829202D2073746F27
:10C3B000700D0A00000000000000000000000000F6
:10C3C0000338FDD87047000002020000020200009E
:10C3D00028B10FF2FC41800141F00101084770478C
:10C3E0002DE9F047DFF87C54DFF87C246968D2F847
:10C3F00000900024002990B00DD529682861491CBF
:10C4000029606C60D9F8080032309628E86058D36B
:10C410009638E86055E006D10120686001210E20C1
:10C4200001F0D4FA19E04A1E0B2A02D2491C6960B5
:10C4300047E04FF0FF3712D10D20686005F02FF96B
:10C44000009001F0A7FC0190039710222869029048
:10C4500069464FF4604001F01AFB044631E00D29B3
:10C4600003D103264EF2100804E04DF6C040042626
:10C4700000EB8118A24610E0EC6809F110001022D0
:10C4800050F824100DEB0A1001F034FF641C962CB8
:10C4900028BF0024EC600AF1010AB245ECDB32014E
:10C4A0006946404601F0F3FA04466868401C3328A8
:10C4B000686006DBA8686F60002848BF2F6005F041
:10C4C0002BFA204610B0BDE8F0872DE9F04F8BB075
:10C4D0000446102206A94FF4604001F002FA002839
:10C4E0002BD406AD4EF2100B686801F03DFD0346FB
:10C4F0000898069A0FF28031009088A62046FEF731
:10C500009BF94620FFF764FF0A9485A70FF21428D1
:10C510000FF214290FF2142A9624102206A9584665
:10C5200001F0DFF9002808D4BDF9180010F4704FAD
:10C530000FD0010404D552460CE04FF0FF302AE042
:10C54000410448BF4A4605D4810454BF3A46424696
:10C5500000E03246B5F90C00BDF918300FF23C315D
:10C560000590C3F30B03B5F90A00049003900BF197
:10C57000100BB5F906000290B5F904000190B5F969
:10C58000020000900A98FEF757F94620FFF720FFB7
:10C59000641EC2D100200BB0BDE8F08F18B5A1B069
:10C5A00044F25441C301ADF80010ADF8020003F5A8
:10C5B00060431228B9BF802284247022742401A908
:10C5C000184601F08EF9002806D40122214668465B
:10C5D000FFF714FD002802D54FF0FF3000E00020E7
:10C5E00022B010BD38B500282CD501F07EFD012801
:10C5F00018D19C4CA068002805D52068401C00215B
:10C600002060A1601CE0FFF7C9FFA068401C132850
:10C61000A06015DB61684FF0FF300029A0600FD5E6
:10C6200020600DE000252846FFF7B8FF32244FF4C4
:10C630007A70FFF7CDFE641EF9D16D1C132DF2DB6D
:10C64000002032BD132802D34FF0FF3032BDBDE8C9
:10C650003240A3E700E000BF4FF0FF30704780B5E5
:10C6600001464FF400724FF4704001F073FA002855
:10C6700000D580E0BDE8044000210F2001F0A6B9FC
:10C6800070B5ADF5007D04460D4616466846FFF7C9
:10C69000E6FF002848BF4FF0FF300CD43246294651
:10C6A0000DEB040001F026FE4FF4007269464FF4D2
:10C6B000704001F069FA0DF5007D70BD10B50446BB
:10C6C000FFF7CCF8202800D395E02046FFF7C6F806
:10C6D0002146BDE81040421C0020D1E710B500F013
:10C6E000C5F84FF4704001F0FCF8002800D585E053
:10C6F0002078FF2804BF6178FF290BD1A078FF289C
:10C7000004BFE178FF2905D154A00168216005200C
:10C7100003F01AFD002010BD000000000000000022
:10C72000490000004C0000005300000054000000CD
:10C7300080B510283EBF13185B1E102B00D317E0E6
:10C740004FF2200303EB8000BDE808409204120C76
:10C7500001F0C7B880B510283EBF13185B1E102B20
:10C7600000D305E0BDE8084080009200203087E754
:10C77000072003F0E9FC4FF0FF3002BD38B5034657
:10C780001546032B38BF412DA0B00C4603D307201C
:10C7900003F0DAFC13E04FF260008022694600EB00
:10C7A000C31001F0D7F9002809D40098854206D1BA
:10C7B000294602A801F0F5FC0199884202D04FF009
:10C7C000FF3005E02A4602A9204601F093FD002033
:10C7D00021B030BD10B50C4611461A4603283CBFA7
:10C7E0001319412B00D306E004EBC01404F16000E0
:10C7F000BDE8104044E7072003F0A6FC4FF0FF30EF
:10C8000010BD10B50446FFF729F8202800D3F2E741
:10C810002046FFF723F82146BDE81040421C4FF4A4
:10C82000F0702DE710B500F021F84FF2E01001F0A4
:10C8300058F8002800D5E1E72078FF2804BF617888
:10C84000FF2908D1A078FF2804BFE178FF2902D191
:10C8500003A001782170002010BD00005858580036
:10C86000000000009C2F0020B03200200446002071
:10C870002070202221467047426174746572793DB0
:10C8800025640D0A54696D653D25730D0A5472695E
:10C89000676765723D25640D0A00000025732564F5
:10C8A0002C25642C25642C25642C25642C25642CD3
:10C8B00025640D0A000000000000000000000000D8
:10C8C0000000000000000000000000000000000068
:10C8D0000338FDD8704700002DE9FC4F83B00E46A9
:10C8E00017460BB100221A608046444600E0641CE3
:10C8F000207805F045F80028F9D120782D2816BFBA
:10C900002B2814F801BB4FF02B0B002F019603D4FA
:10C91000012F01D0252F04DB002E47D0C6F8008060
:10C9200044E0002F0ADD102F04BF2078302802BF1A
:10C93000617841F0200178290ED10AE02078302872
:10C9400018BF0A2708D1607840F02000782802D16B
:10C950001027A41C00E00827029400E0641C207843
:10C960003028FBD04FF0000925A02646CA468DF896
:10C97000000007E09DF80050451BCA46EDB207FBDA
:10C980000959641C207805F005F800BF1CA3014676
:10C990003A46184605F008F80028EBD10299A14262
:10C9A000484605D1019808B1C0F8008000201CE07D
:10C9B0001DA1A61BC95D761A002E0FD405DC451BF0
:10C9C00003D3B5FBF7F1514508D005F019F80498E9
:10C9D00008B1012101604FF0FF3003E0BBF12D0FE2
:10C9E00008BF4042019901B10C6005B0BDE8F08F6D
:10C9F000FFE700230A2200216EE700BF00236BE758
:10CA000030313233343536373839616263646566C4
:10CA10006768696A6B6C6D6E6F707172737475762E
:10CA20007778797A0000000000002115110E0D0CB6
:10CA30000B0B0A0A09090909090808080808080867
:10CA4000070707070707070707070707070000008B
:10CA50001149124A0120086001211148416081609A
:10CA60002021116001220260002070470D480068FB
:10CA70007047884201D3401A7047C1F18071401855
:10CA8000704708490968814201D3081A7047C0F10C
:10CA90008070081870470000080000400815014029
:10CAA000001001400415014011DF0849B120086061
:10CAB000BFF34F8F064907480A6802F4E062024359
:10CAC0000A60BFF34F8F00BFFDE700BF1C050040A9
:10CAD0000CED00E00400FA05E0B50020082101900B
:10CAE00000914FF4807300220021364805F0D6F8FB
:10CAF0000EBD2DE9FE43334D6F88AC88EE8881462C
:10CB00004FF00608761E06D51F26641E03D50F2497
:10CB10007F1E48BF0127200200EB0730082269462C
:10CB200000EBC60000F0DDFE009911F1010F06D008
:10CB30009DF90400012806D0B8F10108E2D10020D7
:10CB40006861BDE8F783D9F800100098091A696197
:10CB5000F7E71C484069704738B504460D4694F91C
:10CB6000040010B92046FFF7C4FF2B46214601B050
:10CB7000BDE830400822134805F0C4B8114949887F
:10CB800000F0DCB90F484088112100F0F2B938B547
:10CB90000C4D04466888411E8941C90F204600F0AB
:10CBA000CDF9002802D54FF0FF3032BD698820460C
:10CBB00000F0C4F90546012C08BF00F0B0F9284682
:10CBC00032BD0000A05E002081EA00039B0717D160
:10CBD000820707D010F8012B11F8013BBAB19A4235
:10CBE000F6D014E002680B689A42A2F1013301BF4B
:10CBF000934313F0803F50F8042F51F8043FF3D0D3
:10CC000010F8012B11F8013B0AB19A42F8D0D01A62
:10CC1000704700000000000000000000000000005D
:10CC200028B10FF23C41800141F0010108477047F3
:10CC300010B5044601F0AEF820600020207104F029
:10CC400031FD6071DFF8B4030188E18010BD90F917
:10CC500004100329BCBF41796529BEBFC08840F2DA
:10CC6000FF11884201DB00207047012070473EB56C
:10CC70000546FFF7ECFF012833D06946DFF8800353
:10CC800000F061FD00F02FF81024BDF8040000282A
:10CC900004BFBDF8060000281DD000F071F800F0B8
:10CCA00022F8BDF80200BDF80030000300EB03409D
:10CCB000BDF8043000EB0320BDF8063008222946F9
:10CCC00000EBC30000F00DFE2846FFF7C0FF01286F
:10CCD00007D0641ED9D14FF6FF70E8804FF0FF30C7
:10CCE0003EBD00203EBD012300222021684600F009
:10CCF0000EBD38B584B00546FFF7EEFE002848BFEC
:10CD00004FF0FF303AD402A80821019000914FF46F
:10CD1000007302220021BA4804F0C0FF04002DD4A1
:10CD200002A8FFF7A4FF002C0CBFBDF80E000020E6
:10CD300000F0B0F974B99DF90C0010F1010F09D0A1
:10CD400000218DF80C10012D04BF02A8FFF704FF8D
:10CD500000F016F802A8FFF76BFF0120012D8DF8F7
:10CD60000C000AD1002102A8FFF7F6FE00F008F837
:10CD7000002000F007F800F003F8002005B030BDF7
:10CD800046204DE71CB504466846FFF751FF234691
:10CD9000082269469A4804F0B5FF16BD1CB5044642
:10CDA0006846FFF745FF02218DF80410ADF80640F4
:10CDB00000216846FFF7D0FE16BD38B5904D0446F9
:10CDC000688802280CBF03210221204600F0B6F833
:10CDD000002802D54FF0FF3032BD69882046BDE8FB
:10CDE0003440ABE00000000070B5064686B00C464B
:10CDF000154668090002EB0000EB043003F0F8036D
:10CE0000082204A9181800F06CFDFFF7B9FF9DF97E
:10CE1000140010F1010F21D0022804980CD101F068
:10CE2000A3F8BDF816109DF815200291019200900C
:10CE30002B46224674A10EE001F096F8BDF81610BC
:10CE40009DF815200190039102922B469DF9140044
:10CE500076A1009022463046FDF7EEFC002006B099
:10CE600070BD2DE9F84FA2B08B46050345F2444151
:10CE70000228ADF804104FF001094FF0FF3A4BD2F1
:10CE80000001002700904FF6FF7801AE1BEA090F62
:10CE90004FEA4A0A36D0009838187080802202A9DA
:10CEA000284600F01EFD002836D40A244FF47A707C
:10CEB000FFF7B6FE641EF9D1002101A800EBC10006
:10CEC0008288424504BFC088404502D0491C1029D1
:10CED000F3DB102903DA708840F4404070801BEACD
:10CEE0000A0F03D1708840F400407080C900091D0A
:10CEF000002289B201A8FFF781F800280CD47088BD
:10CF0000010405D480357F1C102F4FEA4909BDDB91
:10CF1000002023B0BDE8F08F4FF0FF30F9E780B577
:10CF200045F244404FF6FF71ADF80000ADF8021035
:10CF3000002204216846FFF761F802BD70B50C4677
:10CF400088B9012C8CBF4FF400754FF48075002612
:10CF500005E0324621460020FFF746FF761CAE4230
:10CF6000F7D3002070BD2046BDE870404FF6FF713A
:10CF700077E72DE9F8430446022C0D464FF400797B
:10CF800023D2204841888288C08802EBC10200EB8E
:10CF900042177F1BC84648BF07F500774FF48079DA
:10CFA0000026AE4227DA97FBF9F109FB1172002047
:10CFB000FFF71AFF7F1C474505DB022C2CBFA7F5A6
:10CFC0008067A7EB0807761CEBE7042C10D20C480F
:10CFD00041888288C08802EB011200EB42177F1B58
:10CFE000B7F5806FB8BF07F580674FF40068D7E7E3
:10CFF0004FF0FF3000E00020BDE8F283005F00202A
:10D00000185F0020A05E00202564253033642020B6
:10D0100074696D655B545D203A20202573202533AB
:10D02000642020543A25640D0A0000002564253050
:10D030003364202074696D655B25645D203A20208F
:10D040002573202533642020423A25640D0A000010
:10D0500000000000000000000000000000000000D0
:10D060000338FDD8704700000000000000000000F9
:10D0700028B10FF26C61800141F00101084770474F
:10D0800010B5040005D04FF47A70FFF7F1FF641E6D
:10D09000F9D110BD1CB5411C88B240F2FF1290427C
:10D0A00000DA00B901214FF4FF7000900123DFF88E
:10D0B000B844102289B2204604F0ACFF2188DFF882
:10D0C000AC24916516BD38B50146DFF89C5480222A
:10D0D000284604F0C4FF040004BF288900280BD1AF
:10D0E000A98A2888814207D004F016FC29880FF20B
:10D0F0009040A982FEF7BFFC204632BD2DE9F04FDB
:10D10000DFF864348BB09C89A142A1BF0A92DB890D
:10D110000A9A934205DA072003F016F84FF0FF3021
:10D1200084E08146002500248A4601E00AF1010AD4
:10D13000DFF83404C189491C8A4508BFB0F80CA047
:10D140000FF2504152464846FDF776FB0026002775
:10D15000300300EB0A404FF0000B00EB07281022D1
:10D1600006A908EB0B1000F0BCFBBDF9182012F16A
:10D17000010F04BFBDF91A0010F1010F24D1BDF950
:10D180001C0010F1010F04BFBDF91E0010F1010FCA
:10D190001AD1BDF9200010F1010F01BFBDF9220025
:10D1A00010F1010FBDF9240010F1010F0CD1641C26
:10D1B000022C26DD11271026002D28DD0FF2E0318C
:10D1C0004846FDF739FB22E0BDF92430BDF92600C1
:10D1D0000FF2204104930590002CBDF92030BDF9D9
:10D1E000220002930390C8BF0024BDF91C30BDF992
:10D1F0001E00009301904846BDF91A30FDF71CFB54
:10D200006D1C0BF1010BBBF1100FA8DB7F1C102F65
:10D210009EDB761C102E9ADB0A98824586D12A4620
:10D220000FF2F8314846FDF707FB00200BB0BDE8D0
:10D23000F08F38B5FFF71AFC044640F6B83502E027
:10D24000FFF714FC04462046FFF71BFCA8420AD255
:10D2500002F05CFF0021012004F0B9FF0128EFD0AB
:10D2600000F0E1F8EFE731BD2DE9FE4FBE4DA88992
:10D270000F468742A2BF0292E989914206DA07204F
:10D2800002F062FF4FF0FF304FE07F1CE989B8B237
:10D29000491C88420FF2DC3008BFAF891FFA87F9BA
:10D2A0004946FEF7E8FB0026ADF80070B046ADF841
:10D2B0000280002400E014B901F0F9FC03E0032C23
:10D2C00008BF01F0F6FCADF804404FF0000A02F090
:10D2D0001DFF0021012004F07AFF0AEBCA00ADF81F
:10D2E000060000230122B1B2684604F02AFF8346FB
:10D2F0004620FFF7BDFE761CBBF1840F17D30AF161
:10D30000010ABAF1010FE2DD641CA4B2102CD2DBD9
:10D3100008F101081FFA88F01028C8DB029881453F
:10D32000B3D1002004F080FF0020BDE8FE8FFFF79E
:10D3300080FF1024A046E7E7002808BFFFF7DEBE05
:10D34000012808BFFFF790BF4FF0FF3070472DE96D
:10D35000F04DA2B00C4644F25341ADF80010904697
:10D360006101ADF80410ADF8020021034FF0010B8C
:10D370000025002601EB004A18EA0B0F32D006EB1D
:10D38000D6704010F3010AEB002003F080038022E6
:10D390000DF10601181800F0A4FABDF80600F0B16E
:10D3A00000274FF6FF720DF106003901405A9042F6
:10D3B00002D07F1C082FF6DB082F03DB0F2C08BFE1
:10D3C0001F2E05D100F080F8012501E000F02BF8B8
:10D3D000380100F073F80028F8D46DB902E0462057
:10D3E000FFF746FEBDF80400761C401C1F2EADF86A
:10D3F00004004FEA4B0BBFDD8DB900F065F8BDF8B6
:10D40000040040F40040ADF8040001E000F00BF827
:10D41000002206216846FEF7F1FD0028F6D4002020
:10D4200022B0BDE8F08D01202AE62DE9F041A2B03E
:10D43000044644F25340ADF80000ADF8024000202D
:10D44000ADF8040000262404002740F2FF188022D3
:10D450000DF10601204600F044FABDF80600E8B1DF
:10D4600000254FF6FF720DF106002901405A904247
:10D4700002D06D1C082DF6DB082D01DB474505D1D8
:10D4800000F022F8012601E0FFF7CDFF280100F0AF
:10D4900015F80028F8D430000CD102E04620FFF740
:10D4A000E7FDBDF8040080347F1C401C4745ADF803
:10D4B0000400CCDD002022B0BDE8F081801D81B2E7
:10D4C00000226846FEF79ABDBDF8020040F4004015
:10D4D000ADF80200704780B5A2B00B4644F253414C
:10D4E000ADF80430ADF80010ADF80200DB01802289
:10D4F0000DF1060103EB004000F0F3F9BDF8060062
:10D5000010B94FF0FF3004E0002286216846FEF794
:10D5100075FD23B000BD000010B504464FEA0401BC
:10D5200059A0FEF7A8FA1148114A016811600CB918
:10D53000846D05E04FF6FF70844204BF0A480488FA
:10D540000C490D480D4A0C6000210160117010BD9E
:10D5500007490A4A4FF0FF30086000211170014668
:10D5600052A0FEF788BA0000005F0020443200207D
:10D5700030320020283200202C32002020320020BF
:10D5800073646174615F626C6F636B203A20256421
:10D590000D0A0000626C6F636B2025640D0A0000A9
:10D5A00053545245414D5F454E44212121212121B3
:10D5B000212121212121212121212121212121215B
:10D5C000212121212121212121212121212121214B
:10D5D000212121212121212121212121212121213B
:10D5E0002121212121212121212121212121210D3F
:10D5F0000A000000253032642C253032642C25309E
:10D6000032642C253032642C253032642C253032A3
:10D61000642C253032642C25640D0A00454E4421CB
:10D6200021212121212121212121212121212121EA
:10D6300021212121212121212121212121212121DA
:10D6400021212121212121212121212121212121CA
:10D6500021212121212121212121212121212121BA
:10D6600021212121212121212121282564290D0A7F
:10D670000000000073656E7420626C6F636B203A6B
:10D680002025640D0A000000656E61626C655F74A0
:10D6900072616E736665725F73656E736F725F64DD
:10D6A000617461282564290D0A00000064697361B2
:10D6B000626C655F7472616E736665725F73656ECE
:10D6C000736F725F646174612825303858290D0AC0
:10D6D000000000000000000000000000000000004A
:10D6E0000338FDD87047000038B500241BA5002181
:10D6F000A0B200F06BF921462846FEF7BCF9641C85
:10D700000E2CF4DB1AA0BDE83240FEF7B4B910B518
:10D71000C4880CB1641E14E04C1E818811B1491EEE
:10D7200081800EE00F218180418811B1491E418026
:10D7300007E00F21418001888A4234BF491E591EEB
:10D740000180C48010BD02880A8042884A80828895
:10D750008A80C088C88070470000000045726173ED
:10D76000652025645F736563746F720D0A000000A5
:10D77000457261736520646F6E650D0A00000000DC
:10D7800028B10FF23C41800141F001010847704788
:10D790001FB5069C009101920293039400226946F2
:10D7A000001D04F034FE04B010BDF8B511F1010FF6
:10D7B0000CBF531C531D092B01DB0720F1E0C3F103
:10D7C0000805DFF86443261DEFB26D1CF05511F11A
:10D7D000010F0FD0EFB2080EF0556D1CEFB2080C20
:10D7E000F0556D1CEFB2080AF0556D1C201DEEB20D
:10D7F0006D1C8155100006D0211DEEB200206D1C5D
:10D800008855521EF8D11846F2BD1CB50A460021B3
:10D8100000911218DFF810434042204400F10C013F
:10D820000023D2B2DFF80403FFF7B2FF18B102F011
:10D830008BFC4FF0FF3016BDF8B51D46144602466E
:10D8400008182918C9B2DFF8E06200915242B718EF
:10D85000C2B207F1940307F10C01DFF8D002FFF721
:10D8600097FF00B19DE02CB12A4606F194012046B5
:10D8700000F040FD0020F2BD10B5DFF8AC4266209C
:10D88000A07200219920E0720220FFF7BEFFB0B91C
:10D8900000F0F3F8204600F072F880B9A078C107D4
:10D8A0000ED400F083F850B900F0E7F8204600F0FD
:10D8B00066F800F0E2F8A078C10701D40320E1E0A7
:10D8C000002010BD10B5044603224FF0FF31902018
:10D8D000FFF76BFF2246BDE8104002230021C0B2D3
:10D8E000AAE770B50C46154640F201118D42064676
:10D8F00005DA06F0FF01C1F58071914201D20720DF
:10D900000AE0802D12DD00F018F880232246002165
:10D91000C0B2FFF791FF20B102F016FC4FF0FF30CC
:10D9200070BD00F0AAF88034803D803600F005F824
:10D93000EBB22246BDE87040D0E70022314613200A
:10D9400033E779490620FFE7C872002101205CE730
:10D950000A4680B5411E03290BD2754B7249184403
:10D96000012310F8010CC8720021BDE8005001200D
:10D9700062E7072002F0E8FB4FF0FF3002BDF8B588
:10D9800004460025684E6A4F785DF07201236219E3
:10D9900000210120FFF750FF18B96D1C032DF3DBA8
:10D9A000F2BD02F0D1FB4FF0FF30F2BD5E49B7206F
:10D9B000CAE780B569460120FFF7CAFF002806BF05
:10D9C0009DF8000010F00100012002BD38B50446AA
:10D9D000B4F5005F0D46A8BF07200CDAFFF7B1FFD2
:10D9E00048B900F04AF8002221032120FFF7DDFEAC
:10D9F00000F045F800B100E01AE002F0A5FB4FF09E
:10DA0000FF3032BD38B50446B4F5007F0D46A8BFDF
:10DA100007200CDAFFF795FF48B900F02EF8002236
:10DA20002104DC20FFF7C1FE00F029F800B1E4E793
:10DA30002DB900F022F8FFF7BCFF0128F9D0002033
:10DA400032BD10B50446FFF77CFF50B900F015F861
:10DA500000224FF0FF31C720FFF7A7FE00F00FF8BC
:10DA600000B10FE02CB900F008F8FFF7A2FF012881
:10DA7000F9D0002010BDB8B20544462080E6002150
:10DA8000C0B2C2E602F060FB4FF0FF3010BD2DE9DE
:10DA9000F0410646154640F2011085420C4605DA73
:10DAA00006F0FF00C0F58070A84201D207202CE0EC
:10DAB000FFF747FF002828D1FFF7DFFF802DDFF8B1
:10DAC000688017DD00F02CF80746802200F023F86C
:10DAD0008021F8B2FFF799FEB8B9FFF7CEFFFFF744
:10DAE00068FF0028F9D1FFF72CFFFFF7C6FF80344D
:10DAF000803D803600F014F80646AAB200F00BF81C
:10DB0000E9B2F0B2FFF781FE18B102F01DFB4FF051
:10DB1000FF30BDE8F081214608F10C0000F0EABBBF
:10DB200000223146122040E60859002034320020FD
:10DB30001034002080B500224FF0FF31B920FFE7FC
:10DB4000FFF733FEFFF79BFF18B102F0FDFA4FF02D
:10DB5000FF3002BDF8B504460D46164604E0FFF757
:10DB60008AFFF61B14FA87F4B0B260B18128ACBF0B
:10DB700080273746BAB229462046FFF7B2FE002872
:10DB8000EDD54FF0FF30F2BDF8B504460D46164610
:10DB900004E0FFF770FFF61B14FA87F4B0B260B12F
:10DBA0008128ACBF80273746BAB229462046FFF706
:10DBB0006EFF0028EDD54FF0FF30F2BD00000000F1
:10DBC0000338FDD870470000002101E0491C0A38E5
:10DBD0000A28FBDA40EA0110C0B2704701090A22A4
:10DBE00000F00F0012FB01007047C5E030B585B0B2
:10DBF0000446002008218DF80800019103AD00952E
:10DC000000F096F860B10020206118210120E0604A
:10DC100061610020A060606020604FF0FF302DE067
:10DC2000687800F07F00FFF7D9FF20609DF80E00B4
:10DC300000F07F00FFF7D2FF60609DF80F0000F05A
:10DC40003F00FFF7CBFFA060287900F03F00FFF70F
:10DC5000C5FFE0609DF81100FFF7C0FF00F007006E
:10DC6000A0619DF8120000F01F00FFF7B7FF401EF3
:10DC70002061E879FFF7B2FF6061002005B030BD98
:10DC800030B585B0044600208DF808008DF80C00F2
:10DC900003AD2068FFF798FF68706068FFF794FF96
:10DCA0008DF80E00A068FFF78FFF8DF80F00E06879
:10DCB000FFF78AFF2871A069FFF786FF8DF8110032
:10DCC0002069401CFFF780FF8DF812006069FFF7A4
:10DCD0007BFF8DF8130003A9082000F03FF880B9FE
:10DCE000A52000F02BF800280BD4204901208876CD
:10DCF0001F480168CA0544BF81F48071016000209B
:10DD000001E04FF0FF3005B030BD00B585B02C20EC
:10DD1000012103AA8DF808000191009200F008F893
:10DD200000280CBF9DF80C004FF0FF3005B000BD7F
:10DD3000012302AA51210F4804F040BC00B585B070
:10DD40002C218DF808108DF80C0003A9012000F09B
:10DD500005F808B14FF0FF3005B000BD019000910B
:10DD6000012302AA5121034804F03DBC44320020A3
:10DD7000086000207433002080B5FFF7C6FF00283C
:10DD800002D54FF0FF3002BDA52801D1012002BD10
:10DD9000002002BD00B58BB06846FFF727FF68463C
:10DDA00000F002F80BB000BDF8B505468CB02F6945
:10DDB000EE686C6986A16846302200F0ABFA04F583
:10DDC000FA64611E40F26D13880803FB01036420AE
:10DDD000B1FBF0F29A1A4FF4C873B1FBF3F15DF89E
:10DDE00027008A188218012F11D914F0030F06D1C9
:10DDF0006420B4FBF0F0642101FB104030B9B4FBA7
:10DE0000F3F34FF4C87000FB134404B9521CB61866
:10DE100051496C68AB688E193C204FF461614443F2
:10DE200028684E4A01FB0343C31802FB06363046FE
:10DE30000DB0F0BD10F0030F14D16421B0FBF1F16F
:10DE4000642202FB110159B94FF4C873B0FBF3F31C
:10DE50004FF4C87101FB1300401E8041C00F704792
:10DE600001207047002070472DE9F0413B493C4EAE
:10DE7000B0FBF1F501FB15003C22B0FBF2F23C21B6
:10DE800001FB1202B2614FF46161B0FBF1F201FBE0
:10DE900012003C23B0FBF3F0F0610721281DB0FB1A
:10DEA000F1F1C1EBC101401A3262306340F2B27746
:10DEB00040F26D144FF4B77809E0854225D300F0A5
:10DEC00033F8012814BF204640462D1A7F1C00F06D
:10DED0002BF801280CBF40462046EEE7B46A3044D8
:10DEE000005D854218D300F01FF8012814BF002000
:10DEF0000C203044005D641C2D1AB46200F014F84C
:10DF000001280CBF0C200020E8E7A7F5FA60F062BA
:10DF100075630020B062F1E700206D1CB06375628C
:10DF200006F11800BDE8F081384683E71FB50168A7
:10DF30000C4C03914168029181680191C168009184
:10DF4000036942692EA15B1C02F5FA62204602F0C9
:10DF500013F9204604B010BDC506F5FF805101003D
:10DF6000442B0020645E002080B5FFF77DFFBDE8F4
:10DF70000240DBE700B58BB06846FFF737FE684626
:10DF8000FFF7D4FF0BB000BD1CB50C464FF4616128
:10DF9000B0FBF1F14FF4616202FB11003C2290FBF7
:10DFA000F2F3182902FB13000ADB0190182291FBFF
:10DFB000F2F20093182000FB12110B4618A102E0A8
:10DFC0000A4600901AA1204602F0D6F8204616BD57
:10DFD000000000001F0000003B0000005A0000008D
:10DFE0007800000097000000B5000000D400000099
:10DFF000F300000011010000300100004E0100009C
:10E00000253034642D253032642D253032642025AE
:10E010003032643A253032643A25303264000000F0
:10E0200025646425646825646D2564730000000020
:10E0300025646825646D256473000000002204F0E7
:10E0400007BBB1F5807F02D34FF0FF3070470170FE
:10E05000012070470078401E8041C043C00F7047C8
:10E060005FEA000C80EA01039B0715D1830706D005
:10E0700011F8013B00F8013BB3B18307F8D10A68FE
:10E08000B2F1013323EA020313F0803F02BF40F8EC
:10E09000042B51F8042FF3E711F8013B00F8013B82
:10E0A00013B111F8013BF9E76046704780B504F001
:10E0B000FBFA14E080B5002807BF00230C490023B9
:10E0C0000C4942F21072012004F008FB0A4A0121B7
:10E0D00004E080B504F046FB074A0021117018B136
:10E0E00002F032F84FF0FF3002BD0348007870476D
:10E0F000BDB10200CB17020035600020A0F1300254
:10E100000A2A81B038BF30380CD3A0F14103062B66
:10E1100038BF373806D3A0F16101062934BF57381C
:10E120004FF0FF3001B07047F8B504460D460026A9
:10E13000207870B1617861B1FFF7E0FF0746607841
:10E14000FFF7DCFF00EB071005F8010BA41C761CA1
:10E15000EEE73046F2BD00290ADB00F580535B682C
:10E160008B4205DD00EB810043681360002070479F
:10E170000120704718B50021174A0B4608205C089B
:10E18000DB07234644BF154C6340401EF7D142F8DD
:10E190002130491CB1F5807FEFD31149012008607F
:10E1A00011BD70B50D460E49044608684FF0FF36A4
:10E1B00008B9FFF7DFFF0020074908E0225C724042
:10E1C00002F0FF0251F8223083EA1626401CA842D2
:10E1D000F4D3F04370BD0000AC5100202083B8EDB3
:10E1E000F85F00201FB50C4638494A68029220B1FA
:10E1F000D1F8002037A101F0BFFF6CB19DF80800F5
:10E200009DF80910019000919DF80A309DF80B20AF
:10E2100032A1204601F0B0FF002004B010BD000084
:10E2200080B52B490A684B682FA101F0A5FF00209B
:10E2300002BD1A2838BF413006D3342838BF4730D2
:10E2400002D33E2802D2001FC0B2704701D1402045
:10E250007047232070472DE9FC411D490A68009250
:10E26000002749680191DDE900480B260546204654
:10E2700041463E22002304F08FFA1046FFF7D9FFF3
:10E28000E855414620463E2200237F1C04F084FAD4
:10E29000761E04468846EAD104F095FB0A2404F071
:10E2A0009AFB10F1010F03D1641EF8D1FFF772FD44
:10E2B0003E22B0FBF2F23E2101FB1200FFF7B9FF54
:10E2C000E855E91900204870BDE8F681000100100A
:10E2D000600000106E52462578000000256325631B
:10E2E0002563256300000000253038582530385854
:10E2F0000000000062B38B0708D0521E11F8013BEA
:10E3000000F8013B00F024808B07F6D1830740F032
:10E31000208000BF103A07D330B4B1E83810103A6B
:10E32000A0E83810F9D230BC530724BFB1E8081078
:10E33000A0E8081044BF51F8043B40F8043BD20762
:10E3400024BF31F8022B20F8022B44BF0B78037056
:10E350007047121F17D35B0009D151F8043B20F816
:10E36000023B1B0C121F20F8023BF6D20BE051F8C7
:10E37000043B00F8013B1B0A20F8023B1B0C121F58
:10E3800000F8013BF3D238BF121D521E24BF11F812
:10E39000013B00F8013BF8D870478268521C82604C
:10E3A000426832B10268531C036011704168491E13
:10E3B0004160704730B5134B1C68202C08DA0C25DF
:10E3C00065431D44641C1C6045F8040F6960AA6025
:10E3D00030BD2DE9FC410B4D0FF22C0804462E1DDB
:10E3E000002709E0B06800904146736856F80C2B8E
:10E3F0002046FCF721FA7F1C28688742F2DB0020C8
:10E40000BDE8F681845700206661756C74203A205F
:10E4100025642C2025642C2025640D0A00000000B2
:10E4200028B10FF27C31800141F0010108477047AB
:10E430000168CE4A914206D2408940F6AD518842E9
:10E4400001DA012070470020704738B50C46002CD7
:10E450001546194605D44FF47F6292FBF5F29442BB
:10E4600002DB4FF0FF3032BDAAB2000304FB05000F
:10E47000BDE838401030FFF734BA2DE9F84F541A90
:10E4800086B004EBD47401EB64094FF0FF3A0591B8
:10E490000492002580460E4617469B465446B81BFC
:10E4A00003281BDB1AF1010F0AD100F078F800F005
:10E4B0006AF822D000F071F84FF0000A00B96D1C24
:10E4C0006B465A4649464046FFF7BFFF00F05BF8EF
:10E4D00015D14F4624E000F060F8761CB74228DBE7
:10E4E00000F05DF800F04FF8F5D1109B5A46711E10
:10E4F0004046FFF7AAFF304642E0002040E000F02F
:10E500004CF800B96D1C14F1010F0DD16B465A4641
:10E5100039464046FFF799FF00F035F81CD14E46CA
:10E5200000F035F8012402E04E4600F030F8032DEB
:10E53000B5DB049C109E059F00E0641EBC4217DB07
:10E5400033465A4621464046FFF77FFF3046FFF7E5
:10E550006FFF0128F1D111E000F01FF80028E8D08A
:10E5600010985A466946FFF7D5FE0498401C07E00C
:10E57000002000210022002386E80F004FF0FF302A
:10E5800007B0BDE8F08F009810F1010F7047B81B7D
:10E5900000EBD07006EB60097047684648E76B46B1
:10E5A0005A463146404650E738B515460C4629686C
:10E5B000401828602889401C28816889201A1F2853
:10E5C00005DBFFF7E7FB6860A889401CA8816C8128
:10E5D00031BD2DE9FC4104461D460E46174628462E
:10E5E000FFF726FF40B9062C0CBF601C601E2B46AF
:10E5F0001022FE21FFF729FF00212046FFF7E6F950
:10E6000000F0A7F85A485B49009001914FEA04389E
:10E61000082269464046FFF73AFA00F09AF8284681
:10E62000FFF706FF012805D12A4639463046FFF795
:10E63000BBFF07E02E60FFF7ADFB68606F81012034
:10E640002881A8811022294608F11000FFF71FFA3F
:10E6500000F07FF848480021048041800020BDE898
:10E66000F68100002DE9F84F84B080464148404EC5
:10E6700003908B469246002501AFAC1D4FEA04394A
:10E68000082201A94846FFF72CF900284FF0FF3077
:10E6900057D4CAF800000198B04202BF78680399C5
:10E6A000884251D1CDF800A01023FE22002120463F
:10E6B000FFF7E3FE002847D4FE2819DD6D1C012D6D
:10E6C000DBDD042201A946F21400FFF70AF900F08D
:10E6D00040F8042202A947F21400FFF702F900F003
:10E6E00038F801987968884234BF0626072614E076
:10E6F0000646524659464046FFF756FF09EB0613B9
:10E700001022514603F11000FFF7C1F91A480480A6
:10E71000468000F01EF8002013E086F001073A461C
:10E720004FEA060115A0FDF7A6F953461022FE2177
:10E730003846FFF78AFE53465A4641463046FFF7B1
:10E7400048FF05B0BDE8F08F53465A464146A0B297
:10E75000F5E7462064E6084B014618885B8800030D
:10E760001030102200EB0310FFF7BBB8000FFC5D68
:10E770004241545F4C4F470000350020736563747D
:10E780006F72203A2025642C2025640D0A000000B9
:10E790000000000000000000000000000000000079
:10E7A0000338FDD8704700000000000000000000A2
:10E7B00010B5040008D000BF95A14FF47A4041F095
:10E7C00001018847641EF6D110BD00002DE9F04F0D
:10E7D00099B04FF0000818901791144616931698A8
:10E7E000804561D26078179915904144A0781490C3
:10E7F000E07813902079129060791190A279E379F2
:10E80000267A677A94F80AC094F80BE094F80C50D2
:10E8100094F80D9094F80EA094F80FB05FA01091AA
:10E8200021780F911899F9B1CDF838B0CDF834A00E
:10E83000CDF830900B9505920693CDF828E0CDF8F1
:10E8400024C008970796119A12990F9B049203917E
:10E85000139A1499029201910146159A0092002090
:10E86000109AFDF718FC1BE0CDF834B0CDF830A0BD
:10E87000CDF82C900A95049205931199129A039160
:10E880000292CDF824E01399149A01910092CDF8E8
:10E8900020C0159B0F9A109907970696FDF7EBF885
:10E8A000103408F110089AE7002019B0BDE8F08F85
:10E8B00070B504460129C0B088BF4FF0FF3019D8A9
:10E8C0000D0300264FF480726946284604F0A5F82F
:10E8D00000280ED44FF480736A4631022046FFF7B9
:10E8E00075FF0120FFF764FF761C102E05F580757B
:10E8F000E8DB002040B070BD2DE9F84F0D46032D38
:10E90000C0B0834616460CD1706822A1FEF75CF9B0
:10E9100038B9B068FEF76CF801465846FFF7C8FFF3
:10E9200034E001270FF270080FF2CC092BE056F803
:10E930002700FEF75DF88246BAF1000F25D4524653
:10E9400049465846FBF778FF002404EB0A104FF4C1
:10E95000807269460002FEF7C4FF60B94FF480730D
:10E960006A4621025846FFF731FF0120FFF720FFDA
:10E97000641C102CE9DB681E874203DA41465846C6
:10E98000FBF75AFF7F1CAF42D1DB002041B0BDE84E
:10E99000F08F00002D6900000D0A0000253034586A
:10E9A000203A202530325820253032582025303268
:10E9B0005820253032582025303258202530325802
:10E9C00020253032582025303258202D2025303255
:10E9D00058202530325820253032582025303258E2
:10E9E000202530325820253032582025303258200A
:10E9F000253032580D0A0000536563746F7220256C
:10EA0000643A0D0A0A000000000000000000000047
:10EA10000338FDD870470000E0B5002010210190B8
:10EA200000914FF48073042200213C4803F036F932
:10EA300000200EBD10B50446FEF718F8241838481B
:10EA40008462002010BD00007FB5354C207801287D
:10EA500008BF4FF0FF303CD0FFF79CF9606000200A
:10EA60002081FEF703F82F4E05463068962802D223
:10EA7000002161811DE0A16A2846FDF7FAFF00F53B
:10EA8000E8405B306081B4F90A00401D0B2810D3C8
:10EA90006068FFF769FAB4F90A10238BE28A0291E1
:10EAA00031680191618B00914FEA000141A0FCF7B0
:10EAB000E2FFA56202F0F3FDA0811B480188E1811D
:10EAC0001A49088820821A480188618200200121A1
:10EAD000217004B070BD10B50346114C1022211DE9
:10EAE00004F1140003F00EF908B90021217010BDE3
:10EAF0000B48C08A1EE038B50948C18A04290CBFFA
:10EB0000052504250224284600F014F8042D0CBF26
:10EB100005250425641EF6D1002032BDAC5D002021
:10EB2000985D002044320020965C002006350020CD
:10EB3000165F00202DE9F04389B0804600240FF2D3
:10EB4000A0092602002506EB08362701102205A998
:10EB5000A819FEF7C6FE059810F1010F22D0BDF8E6
:10EB60001800D8B90598FFF7FFF90346BDF8220051
:10EB7000BDF8201004900391BDF81E00BDF81C10D4
:10EB8000029001914146BDF91A000090E81005EB92
:10EB9000107007EB20124846FCF76DFF1035B5F5F5
:10EBA000807FD3DB641C102CCBDB002009B0BDE8D8
:10EBB000F08300002573203A206C6F6E6720696E29
:10EBC00074657276616C202825642C2025642C20C5
:10EBD00025642C20256429202D3E2025640D0A0063
:10EBE00025642530336420202573202025642C20C3
:10EBF00025642C2025642C2025642C2025640D0AF6
:10EC00000000000000000000000000000000000004
:10EC100030B5039D049C41EA420141EA830141EA87
:10EC200005213F4A41EA044142F8201030BDE0B5D9
:10EC300000210191009100230122012105E0E0B5AE
:10EC40000B460021002201910092FFF7E1FF07BD72
:10EC500080B534480178012908D100211920FFF737
:10EC6000EEFF00211A20FFF7EAFF05E01920FFF769
:10EC7000DEFF1A20FFF7DBFF00210320FFF7DFFF95
:10EC80001F20FFF7D4FF1E20FFF7D1FF1D20FFF745
:10EC9000CEFF00210220FFF7D2FF00211B20FFF74B
:10ECA000CEFF00211C20FFF7CAFF002002BD1E4935
:10ECB00000E01E494FF00070086070471A4900E0FC
:10ECC0001A494FF080600860704717494FF00040C4
:10ECD00008607047144900E014494FF08040086014
:10ECE0007047114900E011494FF00050086070472B
:10ECF0000E484FF0804101604FF0005101604FF02D
:10ED0000004101607047000009480068C00EFFE73D
:10ED100000F00100704706480068C008F8E70000EE
:10ED20000007005034600020080500500C0500501A
:10ED3000100500500000000000000000F8B5044677
:10ED40000D46A2F10C07A0B0394605F10C00FFF703
:10ED500028FAA96845A6884207D000BF45A33246D5
:10ED600000212046FBF786FD25E06868042804D3CF
:10ED700031462046FBF79AFD1DE000973A46A86809
:10ED8000019005F10C0102A8FFF7C4FA686807F1C9
:10ED900008036A460021FDF71DFD002807D408A3DB
:10EDA000324601212046FBF765FD002005E0314693
:10EDB0002046FBF78FFD4FF0FF3021B0F0BD000083
:10EDC0005345540080B50846111F001D03F069FF2C
:10EDD000002002BD80B50846A2F10803C18800F1F9
:10EDE000080280889BB203F074FF002002BD084631
:10EDF000C1888088FEF76FBB80B54B885B1E0AD048
:10EE00002F3B11D05B1E13D05B1E14D0CF3B05D01F
:10EE10005B1E06D013E0BDE808408FE7BDE8084060
:10EE2000D0E7BDE80840D5E78888FEF775FB04E029
:10EE3000BDE80840DBE7FEF78BFB002002BD4FF08A
:10EE4000FF3002BD44F64252028089B20122FDF732
:10EE5000D5B8E0B54FF48071ADF80210ADF80400FC
:10EE600006216846FFF7EEFF0EBD0000444346470B
:10EE700000000000435243204572726F7200000090
:10EE80002DE9F84F74A7A2B0D7E90045CDE90045B8
:10EE90002C9EDFF8307C04918DF843605FF0000118
:10EEA0006FA40D9112944FF0FF368246904699461A
:10EEB0000FE0C3462C461BF8011B0498D0470028DE
:10EEC000049000F0B2800D98401C641E0D90F2D1A9
:10EED000A84498F80000252807D10021079108913F
:10EEE00009910A910B910C910DE06A46314640461A
:10EEF00004F064F8050001D10D98B5E0D9D50125DD
:10EF0000E6E741F0010118F8010F2028F9D0232885
:10EF10000CD02B2804D02D2805D0302809D086E02D
:10EF200041F00201EFE741F00401ECE741F0080194
:10EF3000E9E741F01001E6E700200F900AE00F98A2
:10EF4000B84205DA00EB800302EB4302303A0F923D
:10EF500008F1010898F80020A2F130000A28EED349
:10EF600098F800002E2818BF0E9629D118F8010F26
:10EF70002A280BD1D9F80000C9F8000008F10108CF
:10EF800050F8042BC9F800000E9219E02D280CBF90
:10EF900018F8010B002000220E920BE040B90E9AE7
:10EFA000BA4205DA02EB820403EB4403303B0E93D2
:10EFB00008F1010898F80030A3F130020A2AEDD3D5
:10EFC000ADF84010129898F80010FCF793FC08B1C7
:10EFD00018F8010B8DF842009DF84200682804BF24
:10EFE00098F80010682903D162208DF8420008E0EB
:10EFF0006C2804BF98F800006C2804D171218DF8AA
:10F00000421008F1010813A806904A4618F8013B7F
:10F0100002A9504600F068F838B913AA02A9504670
:10F0200000F0CAF900287FF554AF30461CE02A28CA
:10F0300082D1D9F80020C9F8002052F8040BC9F891
:10F04000002000280F9003D540420F9041F00401AA
:10F0500008F1010884E70000000000000000000043
:10F06000686A6C747A4C000023B0BDE8F08F6228A7
:10F0700020D0682811D06A2803D06C2827D07128A6
:10F0800025D10868C01D20F007000860D0E90023E2
:10F0900008300860194610467047002A0A680A605E
:10F0A000106803D0121D0A6000B217E0121D0A603A
:10F0B00080B217E0002A0A680A60106803D0121DA7
:10F0C0000A6040B20AE0121D0A60C0B20AE0002ADB
:10F0D0000A680A60106803D0121D0A60C1177047E1
:10F0E000121D0A60002170477CB50D4611461C4672
:10F0F0002E69B4F1250200F04D811C3A00F08680A3
:10F10000121F022A40F282800E3A00F00781521F3D
:10F110005AD0093A7AD0921E16D0521E35D0521EBD
:10F12000022A73D9121F30D0521F00F09A80521E4B
:10F130004AD0521E00F0E480D21E00F0FD80921EE4
:10F1400042D0D21E40D02BE195F83A206C2A09D04B
:10F150006869421C6A610A680A6052F8043B0A60E6
:10F16000335427E10A680A6052F8043B0A60002120
:10F17000009301914FF0FF322A6329466A4600F05E
:10F1800096F9002840F1168101E195F83A00012234
:10F19000FFF76DFFC5E900010023994204DA6869B1
:10F1A000411C69612D210DE0288F810704D5686914
:10F1B000411C69612B2105E0C00722D56869411C0B
:10F1C0006961202131541CE095F83A000022FFF7D4
:10F1D0004EFFC5E9000195F83800010711D5D5E9C2
:10F1E00000230020834208BF82420AD044F020005E
:10F1F000782806D1686930213154401C411C69616E
:10F200003454214668693044E86083E00868C01DD2
:10F2100020F007000860D0E9002308300860C5E945
:10F220000023D5E90001C80F04D06869411C696159
:10F230002D210DE0288F810704D56869411C696183
:10F240002B2105E0C00704D56869411C69612021B4
:10F25000315468693044E8602146284600F032FAAB
:10F26000A8E005F13A02507820B14FF0FF340FF6D4
:10F27000243070E01078622808D0682824D06A28EA
:10F2800012D06C282ED071280ED02BE00A680A60AC
:10F2900052F8040B0A6020B94FF0FF340FF60C301F
:10F2A00059E0E96A017085E00A680A6052F8040BC7
:10F2B0000A6020B94FF0FF340FF6F0204BE0EA6A05
:10F2C000D317C0E9002375E00A680A6052F8040BFE
:10F2D0000A6020B94FF0FF340FF6D0203BE0E96A16
:10F2E000018067E00A680A6052F8040B0A6020B9DE
:10F2F0004FF0FF340FF6B4202DE0E96A016059E0C9
:10F300000A680A6052F8040B0A600021C5E900018E
:10F31000EE607821284600F029F94BE06C2285F850
:10F320003A200B680B6053F8042B0B6052BB4FF074
:10F33000FF340FF6AC200EE095F83A206C2AF0D09E
:10F340000868086050F8044B0860EC603CB94FF066
:10F35000FF340FF6702003F03BFE201A76BD2E6BB3
:10F36000002E04D52046FCF779FA044608E0324620
:10F370000021204602F018FB002814BF041B34466D
:10F38000AC6117E0294600F092F8002812D54FF042
:10F39000FF3076BD6869411C69612521315409E05F
:10F3A0006969481C686125227254210002D0411C01
:10F3B00069613454002076BD2DE9F0410E460546C2
:10F3C000716B7069B46A091A306A091AB069091A4E
:10F3D000706A091AF069091A96F838000C1B41077F
:10F3E00090460DD4002C0BDD2746B0682021A8479D
:10F3F0000028B06057D0F06A401C7F1EF062F4D144
:10F40000736942463146284600F0ACFC00284AD1D8
:10F41000376A002F0ADDB0683021A8470028B060A5
:10F4200041D0F06A401C7F1EF062F4D1B369F268EB
:10F430003146284600F096FCA8BB776A002F09DD0C
:10F44000B0683021A847B06068B3F06A401C7F1EE6
:10F45000F062F5D1F068B169F36942183146284687
:10F4600000F080FCF8B9B76A002F09DDB0683021E0
:10F47000A847B060B8B1F06A401C7F1EF062F5D1B9
:10F4800096F8380041070BD5002C09DDB068202123
:10F49000A847B06038B1F06A401C641EF062F5D134
:10F4A0000020BDE8F0814FF0FF30BDE8F0812DE98C
:10F4B000F8470D46A3B02F6B002F8146904648BFFA
:10F4C0006FF0004703F0A4FD696B40180FF62C1194
:10F4D0008128D1E90023CDE9012328BF4FF0FF3077
:10F4E0003ED20024002F2FDDD8F8001001AA684674
:10F4F00003F066FD0646002E35D4D8F8000008B9A2
:10F50000761E30D4B7421FDB6869301881280AD3D1
:10F510000020686303AA29464846FFF74DFF040010
:10F5200012D40020686103A8D5F814A032466946B9
:10F530005044FEF7DFFEB244C5F814A058F8040B9F
:10F54000002818BFBF1BCDD12CB903AA29464846B5
:10F55000FFF732FF044614B9002068616863204653
:10F5600024B0BDE8F0874FF0FF34F8E72DE9FC4701
:10F5700007468A463E69BAF16F0F08BF082405D0D6
:10F580004AF02001782914BF0A2410243C25D7E929
:10F590000023BAF1640F18BFBAF1690F904699467B
:10F5A00006D100218B4203DAD8F1000869EB490942
:10F5B0000020814508BF80451FD1386BE8B9082C71
:10F5C0004CD197F83800010748D530203B2586F804
:10F5D0003B0043E000280ED597F8380000F01400F7
:10F5E000102808D17A6B7869121A386A121A511ADF
:10F5F0000029C8BF3962BDE8F3878DF800A04046F6
:10F6000049462246E31703F0C7F83032D0B26D1EE8
:10F610003A28019504DB9DF80000A0F151018A18F9
:10F620007255404649462246E31703F0B5F8804636
:10F6300089460020814508BF804503D0F8687119CC
:10F640008842DCD3082C09D197F83800010705D58A
:10F65000715D302902D06D1E30207055C5F13C011E
:10F66000B9617019F860386B8142B3DA411A3962B6
:10F670004FF6EF70398F01403987BDE8F3872DE9E8
:10F68000D04306460F4614464FF00008DFF8389482
:10F6900012E0E00707D542464B463046394603F0B4
:10F6A000C3FC06460F464046494642464B4603F0D9
:10F6B000BBFC641080468946002CEAD130463946AE
:10F6C000BDE8D0832DE9F34F054641F020048DB00D
:10F6D000D5E90089612C02AE09D0286B002848BF0B
:10F6E000062003D408BF672C01D101202863D5E987
:10F6F000002358004015401C0ED119030CD00320E4
:10F70000A8619DF8380061381A2802D20FF2F4611E
:10F7100011E00FF2F4610EE058004015401C0FD1CB
:10F7200019030DD10320A8619DF8380061381A280B
:10F7300014D30FF2DC61E8680322FEF7DBFDD3E1AE
:10F74000194621F00043B3F5801F10460DD2002763
:10F75000BB4208BFBA42019703D111E00FF2AC617E
:10F76000E9E701AA03F036FD0AE0DFF8607307EB72
:10F770001352DFF85C3301921940DFF85833194314
:10F78000C5E90001612C0ED1E86830210170811CAF
:10F79000E9609DF8381061290CBF7821582141702B
:10F7A0006869801C6861D5E900AB2BF0004300203C
:10F7B0002AF00002834204BF8242002300F05A81F3
:10F7C000612C40F0A980286B00284CBF2120401CF0
:10F7D00000904046009F7F1C49460022002303F012
:10F7E00031FDD94601988DF8082038BF89F00049CD
:10F7F000001F0190002FD0460DF1090040F3498110
:10F8000040F2FF71DFF8D0B20C91064640464946FF
:10F810000022002303F032FD80F03A814800400DC1
:10F8200000F11C0210D0002A0EDD0C98824205DB8C
:10F8300009F0004040EA0B01002013E0A448084012
:10F8400040EA025140460DE029F00043002028F034
:10F850000002834208BF82420FBF40461C2240463E
:10F8600003F024FD8046894603F0BEFDFF1F002FF4
:10F87000044609DD03F0D6FD02460B4640464946E4
:10F8800003F0E2FD80468946F01D072104E004F004
:10F890000F0200F8012D2411002C01DD491EF6D5C0
:10F8A000491E5CBF002200F8012DF9D5ECE00020D4
:10F8B000194602AA0A4400E05B1E12F80149491EDB
:10F8C0008442F9D00F2804D10DF10900425C521C8A
:10F8D0004254002904D50198001D02AE5B1C019022
:10F8E000591E12D49DF838007218147804F13008AB
:10F8F0005FFA88F4392CC4BFA0F13A04A044491E31
:10F9000002F80189F1D58DF83800286B002840F104
:10F91000B080591E2963ACE04046494600220023CE
:10F9200003F090FC019938BF89F0004947F29750E5
:10F9300041436A4A91FBF2F20192D2F1070204DDDF
:10F9400040464946FFF79BFE0AE0524200206449C8
:10F95000FFF795FE02460B464046494603F0E6FD9A
:10F960008046662C286BDFF87CB106BF019F0A3702
:10F9700006273F18142FC8BF142730208DF8080021
:10F9800089460DF1090000E03046002F34DD0646BF
:10F990004046494603F0EEFE01460A4606F10803DA
:10F9A00004200A26B2FBF6F606EB860EA2EB4E0208
:10F9B000303203F8012C0A22B6FBF2F202EB820E7F
:10F9C000A6EB4E063036401E03F8026DE9D1083F23
:10F9D000002F03F10806D7DD084603F0DFFE0246DC
:10F9E0000B464046494603F02FFD00225B4603F0DC
:10F9F0001BFB80468946CBE70DF10901401A0DF14A
:10FA0000090604E00199491E401E0191761C3178D7
:10FA10003029F7D0662C02D10199491C03E0652CEE
:10FA20000CBF012100212B6BCB189842B8BF431E9D
:10FA3000002B1ED4834204DAF05C3528A8BF39209D
:10FA400000DA30201946721E02EB010800E05B1E4E
:10FA500018F80199491E8145F9D0392802D1705C06
:10FA6000401C7054002904D50198401C16465B1CAC
:10FA70000190019800B200901BB29DF838103246F8
:10FA8000284600F035F82FE0C61D002F3FF7BEAE28
:10FA900030460DF10901401A009903468842C8BF5B
:10FAA0000B46002B0DF109063FF52FAF8342BFF641
:10FAB000FEAE0DF10900C05C07287FF7F8AE0F20FD
:10FAC000F6E60000CBCCCC0C0000244002FCFFFF8B
:10FAD000FFFF0F800000E03F0000F07FA0860100E4
:10FAE0000000F03F84D797410FB0BDE8F08F0000D1
:10FAF0002DE9F84783B006468A461746984603F034
:10FB000061FAB8F1000F406A356B90F8009002DCA2
:10FB10004FF00108BFA7BDF930404AF02000662829
:10FB200008BF641C15D0672840F0848014F1040FCE
:10FB3000C0F28680AC4280F2838096F83800641C64
:10FB4000010702D4A845B8BF454620B22D1A48BFC8
:10FB500000250FFA84FAF068B169BAF1000F25DCCC
:10FB60004A1C30234354002D03DC96F8380001076B
:10FB700003D5F06800F80290521C15EB0A0FB8BFCD
:10FB80006C4220B2441941424445B8BFA046B2611C
:10FB900071620FFA88F5F561F068B3692A46394653
:10FBA0001844FEF7A7FB641BB462C4E022B2904580
:10FBB000084417DA42463946FEF79CFBB0694044D8
:10FBC000B061AAEB0801002D716203DC96F83810D1
:10FBD0000A0705D5F16801F80090F069401CF06152
:10FBE000B562A8E03946FEF785FBB069002D5044A8
:10FBF000A8EB040803DC96F838100A0703D5F1686F
:10FC000001F80090401CB0610FFA88F08542F0685E
:10FC1000B369B8BFA8460FFA88F207EB0A01184487
:10FC2000FEF768FBB0690FFA88F10844B061681A02
:10FC3000706280E0BAF1610F14D14FF0700A16E0E3
:10FC4000A84504DA96F838100A0758BF45466D1ED5
:10FC500048BF0025BAF1670F14BF4FF0450A4FF0B7
:10FC6000650A04E0BAF1410F08BF4FF0500AB169CC
:10FC7000F368481CB061002D17F8012B5A5403DCBF
:10FC800096F838100A071BD5F168431CB36101F8D8
:10FC90000090002D14DDA8F101080FFA88F08542CC
:10FCA000F068B8BFA8460FFA88F239461844FEF744
:10FCB00021FBB0690FFA88F108446D1AB0617562D2
:10FCC000F068B1690844002C80F800A003D42B210F
:10FCD0004170811C03E02D2141706442811C002091
:10FCE0006A460AE023460A2493FBF4F404EB8405F5
:10FCF000A3EB450302F8013B401C24B2002CF1DCCD
:10FD0000012806DC4AF02002652A04BF302201F8EF
:10FD1000012B48B9302001F8010B07E0401E1DF807
:10FD20000020303201F8012B0028F7DCF068B269BE
:10FD30001044091AF16196F8380000F014001028F8
:10FD40000DD17169B0694118706A4118F0694118A4
:10FD5000B06A4118706B8142BCBF411A316204B075
:10FD6000BDE8F087F8B505460E4617461C4600204C
:10FD700074B117F8011BB068A847B06030B1F06AE1
:10FD8000401CF0620020641EF3D1F2BD4FF0FF3042
:10FD9000F2BD00007072696E74665F733A20256E62
:10FDA00020646973616C6C6F776564007072696E52
:10FDB00074663A2062616420256E20617267756DF9
:10FDC000656E74007072696E74665F733A2062616A
:10FDD0006420257320617267756D656E7400000084
:10FDE0007072696E74665F733A2062616420256C7C
:10FDF0007320617267756D656E740000000000000D
:10FE0000000000006E616E004E414E00696E66009B
:10FE1000494E46003000036A23B9C069B0FA80F049
:10FE2000400970470020704718B404789A4B1B5D56
:10FE30001BB118BC001D03F0D6BD18BC0C3004F07B
:10FE40004AB81CB50178954C002942D0022928D027
:10FE500060D2017AD9B14168097804F1180004F040
:10FE60007FF920B101218DF80010019006E0206A91
:10FE7000616A081A05D000208DF800006846A16B61
:10FE80008847206AA18B626A101A814206D3012238
:10FE900004F13D01201DFFF7C7FF13BD01202070B5
:10FEA00013BD8DF80010C06822797B490190885CF1
:10FEB00038B1012204F13D0104F1080003F093FD83
:10FEC00025E0012204F13D0104F1100004F003F8E3
:10FED0001DE004F13C0104F1280004F054F998B944
:10FEE00021796D48405C38B1012204F13C0104F1F4
:10FEF000080003F026FD13BD012204F13C0104F1CA
:10FF0000100003F067FF13BD03208DF80000684662
:10FF1000A16B884713BD00002DE9F0475F4D0646F1
:10FF20000C0088B01F46AA6308BF072050D0626843
:10FF3000216892B205F1180004F0FEF8002847D1BC
:10FF4000E268A16892B205F1280004F0F5F80028F3
:10FF50003ED100BF53A191E81C57684680E81C576A
:10FF600071690691307C8DF81C70401E8041C04341
:10FF7000C00F8DF81400707C00B10E208DF81500B4
:10FF8000474AF0680290B068039031680191694671
:10FF900070680090281D04F022F9C8B928703068F4
:10FFA00010F1010F13D02A793B49885C38B1012246
:10FFB00005F13D0105F1080003F015FD08E00122FF
:10FFC00005F13D0105F1100003F085FF00E0002080
:10FFD00008B0BDE8F08770B5304C2678014604F1D2
:10FFE000180004F0D0F80546BEB1002121702A485F
:10FFF0002179405C38B1012204F13D0104F108008F
:020000040002F8
:1000000003F0F1FC06E0012204F13D0104F11000CF
:1000100003F061FF08B100F0CFF8284670BD70B55D
:1000200001461E4D05F1280004F09AF8040027D17E
:100030002979194E705C20B105F1080003F0CAFC63
:1000400003E005F1100003F00AFFC8B905F13C0117
:1000500005F1280004F097F890B92979705C38B15F
:10006000012205F13C0105F1080003F06AFC06E0FD
:10007000012205F13C0105F1100003F0ABFE04463E
:10008000204670BD0548016B406B411A481E8041F7
:10009000C00F704700000000AC5F0020403400201B
:1000A00043FE0100FFFFFFFFFFFFFFFFFFFFFFFF1A
:1000B000FFFFFFFF00000000000000000000D6016D
:1000C000060100001F480021016441648166C16689
:1000D000002070471B494A6C01EB8203521C082A1E
:1000E000986428BF00224A640020704715490A6CB2
:1000F000486C824201D10020704701EB82004830F9
:10010000521C082A28BF00220A6470470D48016C5F
:10011000406C814200D1704780B5FFF7E7FFBDE832
:10012000024004F09FB807498A6EC86E824201D12E
:100130000020704701EBC200521C082A28BF002291
:100140008A667047C85B0020014948657047000017
:100150004432002038B5044600252046FFF75FFFF3
:1001600048B1042807D10120FBF702FC6D1CB5F54E
:10017000FA7FF2DB0D2032BD0CB430B583B00446FB
:1001800006A802900A4600250194009502AB01A939
:10019000084878441E30FEF773FE01990D70002860
:1001A0004EBF04460198041B204603B030BC5DF8E6
:1001B0000CFB00BF1730000018B583B06946002261
:1001C0000023002481E81C0002906A46002144F2CA
:1001D0000100FEF7EFF804B010BD002818BF002999
:1001E00001D10E2070470278DE2A01D10820704725
:1001F00009684160DE2101704FF6FF7107E008B920
:100200000E2070470278DE2A01D008207047418016
:10021000002070470246107A58B15088002166DFEE
:1002200008B91172704711281CBF51680847012096
:1002300010727047F8B505460C0018BF002D84B049
:100240004FD02078DE284CD1A9886088814204BF35
:100250002046FFF7DFFF2888012805D0112839D074
:1002600051280FD005B0F0BD287A012802BFA98817
:100270006088814235D1012020722046FFF7CAFFF5
:1002800005B0F0BDA8886188884204BFA87902281B
:1002900027D1A87B04281CBF0628052821D1684641
:1002A000002100220023002680E84E004FF4C07099
:1002B0000227ADF804008DF80070A87B052808BF60
:1002C000ADF80410A8886946B0DF50B1616888476E
:1002D00005B0F0BDA8886188884204BF4FF6FF7062
:1002E000608005B0F0BD036810B4DC690022A4464C
:1002F00001235DF8044B604730B505460C4687B0D6
:10030000A18868696A4604F037F8182101A8FDF74A
:1003100095FE0295A088ADF80C00009804902989FC
:10032000E088884204BF218A022913D1009808B3CB
:1003300004F1120004F04AF820B10099012008707D
:10034000022102E00099087003218DF80410A969C8
:1003500081B10DE0A98988420CD1A96951B1002071
:100360008DF8040004F112020592208AADF81800FD
:1003700001A8884707B030BD38B505460C0018BF46
:10038000002D8AB05ED02888102805D0502836D09D
:1003900057283AD00BB030BD002000906A46A9889B
:1003A000606903F0E9FF02A800210022C0E9001201
:1003B00001A80221ADF808100390ADF80A202189A8
:1003C000A88802AAADDF00283CD1A069002839D056
:1003D000039803F0FBFFA8B3009808B10121017056
:1003E000182104A8FDF72AFE02208DF810000594BC
:1003F000A888ADF818000098079004A820E02946C6
:100400002046FFF779FF0BB030BDA98860696A46C6
:1004100003F0B2FFB0B90098017800291CBFA069B1
:1004200000280FD0182101A8FDF708FE01208DF843
:1004300004000294A888ADF80C000098049001A86C
:10044000A16988470BB030BDF0B500BF4DA292E85E
:10045000E8008DB0040009A880E8E80014BF002976
:100460000E2058D00868A061214609A862DF002844
:1004700051D120788DF802000121ADF80010A21CA6
:1004800069460120A8DF002845D1202101A8FDF7F9
:10049000D5FD0220ADF80400F4202178ADF8080065
:1004A0008DF8061001219DF81100ADF80A1040F0FA
:1004B0000C008DF811008DF810108DF815108DF8C6
:1004C000161004F10C02608801A903F085FF10BB2F
:1004D000202101A8FDF7B2FD0320ADF80400F420AF
:1004E0002178ADF808008DF8061001219DF8110063
:1004F000ADF80A1040F010008DF811008DF81010C2
:100500008DF815108DF816108DF81710221D6088C3
:1005100001A903F061FF0DB0F0BDF0B5040085B096
:100520000D4616461F4608BF0E2029D060696A4650
:10053000394603F021FF18BB4FF6FF718F421ABFF7
:100540000098002805201BD0007810B9082005B0BD
:10055000F0BD3188F529A8BF072011DA01A80021D4
:10056000002200238C4680E80E10A088ADF804001D
:10057000049501208DF80600039601A93846AEDFE8
:1005800005B0F0BD9ECADC240EE5A9E093F3A3B547
:100590000000406EF8B486881746BC19B24228BFE6
:1005A0003746F51BC2881F4607EB020C934228BF53
:1005B0001746D61B4A8803889A4224BF4088904237
:1005C00009D38888A84228BF844204D3C888B0428F
:1005D00028BF844502D2F2BC00207047F2BC012043
:1005E000704738B5804A04461089A1B288422BD1A1
:1005F0007E4D107C297B88420FD202F11201A0B2FD
:1006000075DF30B111281CBFA96900291CD08847AB
:1006100031BD107C401C107431BD00211174287C48
:1006200048B13B21A0B276DF002818BF082802D0CD
:10063000A96901B18847696931B100208DF80000CE
:10064000ADF802406846884731BDF8B5010001D1D8
:100650000E20F2BD91E8FC10644880E8FC10624C6A
:1006600004600868A8B17ADFB8B909682046082292
:10067000FDF740FE4FF6FF70208104F12000E0609E
:1006800000215B4A04F10C0004F010F828B10320AB
:10069000F2BD20467BDF0028ECD0F2BD1CB50B4636
:1006A0000246597A514C71B9187A002858680CBF23
:1006B0006168A16804F00CF800281CBFA16900293A
:1006C0000CD0884713BD00201872616931B1012038
:1006D0008DF80000ADF802206846884713BD2DE96B
:1006E000FC4104462088102807D011282FD012285A
:1006F00061D050283ED0BDE8F381E07BA588012879
:100700006FD1394E394F30894FF6FF78404519D1B6
:1007100000203074358106F1120031460822FDF7C1
:10072000E9FD434640F2F31204F1100106F1120014
:10073000FFF730FF7074F889002852D106F10801E4
:1007400028464BE0B96900294BD0042030E0264D03
:10075000A1882889884244D1E86803F0E9FF00288D
:100760001FBF22498969002988474FF6FF702881F9
:10077000BDE8F3811D4DE088E989884204BF208AE5
:10078000022801BFA788184E3089B84229D104F148
:10079000120003F01BFE18B106F1080138461DE0F7
:1007A000F06803F0C5FF00281CBFA969002918D014
:1007B000BDE8FC4108470C4DA6882889B04210D1FD
:1007C0004FF6FF7340F2F31204F1080105F1120035
:1007D000FFF7E0FE687405F108013046BDE8FC4112
:1007E0005CE7BDE8F3810000285D0020845E002006
:1007F000E3050200417949B100F22E41087828B999
:100800008978481E8041C043C00F70470020704760
:1008100080F830107047F8B504460D0018BF002C62
:1008200001D10E20F2BD05F17A000178012904BF43
:10083000807F012831D005F19C07786804281CBF0F
:100840003968042929D00020A07005F17801201D05
:100850002C22FDF75FFD04F12406002030730721F0
:10086000B8683061F868706104F582674FF6FF7010
:10087000B8823F6104F2264003F07CFF207818B96B
:1008800004F15002FF21117104F1550038603078F5
:1008900001280CBFEE201F2001E00720F2BDB88028
:1008A00004F2144204F15501284604F0A6F828BBCE
:1008B00004F23121B96004F21C42307801280CBFE7
:1008C000EE201F20B88105F13C0004F096F8A8B98D
:1008D00004F150000121417004F13C02A169B1848E
:1008E000012131760021F16101706069306204F10B
:1008F000540072DF10B9012020700020F2BD00000A
:100900002DE9FC4105460F46287810B90820BDE8BE
:10091000F68105F22648AF700721404603F02AFF12
:10092000A87905F5826605F1240410B1A97801299A
:1009300006D0E87968B1A878012818BF022808D144
:10094000216921B1012070770820884701E000204B
:100950007077F07D002804BF317E00290DD1707EB4
:10096000002804BFB17E002907D1F07E28B9317F6D
:10097000481E8041C043C00F00E001207F1E032FAE
:1009800018D8DFE807F002090F13AA7922B12178FD
:1009900011B938B101200EE0E97900291CBF002807
:1009A000022008D1287A08B1032004E0687A08B14F
:1009B000042000E00020A870216981B1A8780328F4
:1009C00018BF04280BD16A794AB1B07F38B9002228
:1009D00085F830240120F0770720884701E00020C7
:1009E000F077182105F13C00FDF728FB0120207667
:1009F00005F15007A06801281CBF0228012078706B
:100A0000207828B1616801291CBF02290121B97031
:100A100000213970A978042943D8DFE801F0740374
:100A20000F1F510001206073002030612062C4F864
:100A30001C80022020768020A08434E0022100283F
:100A400014BF07200320207661732869A08400204A
:100A50003061C4F81C80E868206224E06969216282
:100A60000028A969A18414BF062001202076284609
:100A7000FFF7C0FE90B1022038700122B1883068C3
:100A800004F0F7F808B10421017005F13C02314689
:100A900005F1540072DF20B9052000E003206073E7
:100AA0003661A87888B3316905F13C0205F154003C
:100AB00072DF78BB217B387973DF30B3BDE8F68114
:100AC000E96921620028296AA18414BF0620012057
:100AD00020762846FFF78EFE98B10220387001225A
:100AE000B188306804F0C5F808B10421017005F13F
:100AF0003C02314605F1540072DF0028D1D10620B6
:100B0000CDE70420CBE700206073216909B1607B49
:100B100088470020BDE8F6811CB50C4601881029E5
:100B200004D0112909D0262914D013BDC17B012975
:100B30002BD18088A4F8240413BD04F224410022A0
:100B40008A7280880988884204BF207900281CD1D5
:100B500001210FE0007A012818BF022815D1A078E2
:100B6000401C81B24CF6CD424A43910C01EB81010D
:100B7000401AC1B22046FFF7C3FE00281CBFA16B7C
:100B8000002902D0BDE81C40084713BD000000004A
:100B900010B5040008D00FF2D8214FF47A4041F08C
:100BA00001018847641EF6D110BDDCB50022CDE9F5
:100BB0000022012824D10220009001900224002666
:100BC0005DF82670384600F038F86420FFF7E0FF43
:100BD000384600F03FF84FF41670FFF7D9FF04F0E5
:100BE00057F8761C022EEBDB641EE8D106244FF486
:100BF000FA70FFF7CDFF04F04BF8641EF7D1DDE784
:100C0000022803D1009001210191D7E704280ED1D9
:100C1000032000F012F8824C02E004F039F830BFF3
:100C2000A07E0028F9D0032000F014F8D3BD0328DB
:100C300002D100900321E7E7D3BD10B50446E007D9
:100C400048BFFEF734F8A00703D5BDE81040FEF713
:100C500035B810BD10B50446E00748BFFEF729F8C7
:100C6000A00703D5BDE81040FEF72AB810BD80B537
:100C7000FEF724F8BDE80140FEF719B880B5FEF78D
:100C80001FF8BDE80140FEF714B866480168491C2A
:100C90000160C80748BFFEF70AB8FEF70FB8614801
:100CA0000178CA0748BFFEF704B8FEF709B85C48E8
:100CB0000168B1F5967F3CBF0320FFF7BEBF5948DE
:100CC0000168491C01600320B1FBF0F000EB40001B
:100CD000091A012908BFFDF7F1BF704750480168A4
:100CE000B1F5967F3CBF0320FFF7B4BF4D490868BC
:100CF0000322B0FBF2F202EB4202801A012808BF85
:100D0000FDF7DEBF704780B500F027F803D2BDE8DD
:100D10000240032091E743480168491C0160032019
:100D2000B1FBF0F000EB4000091A012900D19FE768
:100D300001BD80B500F011F803D2BDE802400320E8
:100D400088E7384908680322B0FBF2F202EB42025E
:100D5000801A012800D192E701BD31480168B1F540
:100D6000967F70472E480168B1F5967F3CBF0320FF
:100D7000FFF763BF2B480168491C01600320B1FBEA
:100D8000F0F000EB4000091A012908BFFDF78FBF02
:100D9000704723480168B1F5967F3CBF0320FFF7F9
:100DA00059BF204908680322B0FBF2F202EB42026D
:100DB000801A012808BFFDF77CBF704710B50446B4
:100DC000FDF77EFFFDF775FF012C20461649174AF7
:100DD0001DD0022C02D11649164A18E0032C02D16C
:100DE0001549164A13E0042C02D11549154A0EE0A4
:100DF000052C02D11449154A09E0062C02D11449E8
:100E0000144A04E0072C06BF1349144A0120144B6E
:100E10009A605960186010BD114800687047000062
:100E2000443200200C600020AFEC0100B3EC010064
:100E3000BDEC0100C1EC01006F0C02007D0C020052
:100E40008B0C02009F0C0200AF0C0200DD0C0200B4
:100E5000070D0200330D0200650D0200930D020024
:100E60008C310020000000000000000000000000A5
:100E70000338FDD87047000080B50D48017801297E
:100E800007D1FDF732F920B90A49012081F80401A0
:100E900001BDFDF72AF9012805D1BDE80440322142
:100EA000002000F03EB8BDE802400920FFF712B96B
:100EB000346000201C35002010B53B493B4C0A68CB
:100EC00000E00C34A06840B120688242F9D3A068E9
:100ED00080472168606841182160002010BD2DE91D
:100EE000F041334D2888C8B100242F1DA0462E4E56
:100EF0000EE0386848B13168641C814205D37868D7
:100F0000804700285CBF00203860083708F10108DE
:100F100028888045EDDB0CB9002028800020BDE842
:100F2000F081F0B508B9234B12E0012808BF224B2D
:100F30000ED0022808BF214B0AD0032808BF204B3F
:100F400006D0042808BF1F4B02D0052829D11E4B0C
:100F5000174A1788141D4FF0FF35002601E00834AA
:100F6000761CBE4219DA206810B9002D48BF3546FC
:100F700060689842F3D1002E0FD4354602E03D461A
:100F80007F1C1780084804680919141D02EBC5006E
:100F900044F8351083600020F0BD002DF2D5062FF7
:100FA000EDDB4FF0FF30F0BD4432002088330020ED
:100FB000DC33002099AC0200BFAC0200C5AC0200DB
:100FC000F7AC020001AD020025AD02002028014669
:100FD00004DA7348C84000F001007047402808DA7E
:100FE0000122A1F1200012FA00F018BF0120C0B2C6
:100FF00070470120704700001FB5044678A168467D
:1010000003F07FFE02E0684603F08CFE029A3AB1DC
:1010100051681268204690470028F4D1112000E062
:10102000002004B010BD00001FB504466FA1684643
:1010300003F067FE06E05168126820469047684654
:1010400003F070FE029A002AF5D11FBD80B516206C
:10105000FFF7BCFF28B942F20100BDE80240FFF7EC
:10106000ABB8504800784009082803D2EC21C140B1
:10107000C80702D442F20200EFE74B49886820B16A
:101080000A6842F480020A6001BD48494FF48000BA
:10109000086001BD80B51620FFF798FF28B9BDE8AC
:1010A000024042F20100FFF787B83F49886820B14B
:1010B0000A6822F480020A6001BD3D494FF48000B5
:1010C0000860BFF34F8FBFF36F8F01BD3EB5394D41
:1010D000287808B108203EBD0121A970FFF78CFFD8
:1010E000112820D00020FFF79FFF00BF45A0016816
:1010F000019100228DF80020684603F023FE2E495E
:1011000001A810DF0446401E8041C00F00F034F8F3
:101110000CB120463EBD0020A8706870FFF796FF16
:101120000120FFF781FF00203EBD38B5214D287812
:1011300008B9082032BD0121A9700120FFF75CFF2A
:10114000112817D00220FFF76FFF00208DF8000054
:10115000684603F0F7FD11DF0446002000F00CF8AC
:101160000CB1204632BD0020A870FFF793FF03208A
:10117000FFF75AFF002032BD28709DF8000003F0F1
:10118000FDBD0C48817809B9082070470078002817
:1011900018BFFFF7CABF99E70648007870470000FC
:1011A000FC06FFBD16E400E0885F002000E100E0DF
:1011B00080E100E030600020B5E30100E0B500BF51
:1011C0000DA1684603F09DFD05E048680968884761
:1011D000684603F0A7FD02990029F6D107BDEDE7A7
:1011E00000B8020010B802000800000010B80200A9
:1011F00020B802000800000020B8020030B8020049
:1012000008000000020000053EB50B00044601D1B5
:101210000E203EBD4048186000216846002200258F
:1012200080E82600012028218DF800408DF802007A
:10123000ADF8041069461A68202069DF00F037F81D
:1012400001208DF8010069461A68402069DF00F02E
:101250002EF8F7208DF80040ADF8020069461A68B4
:10126000232069DF684600210022002480E8160060
:1012700001208DF8000069461A6869DF00F011F856
:101280004FF4B060009069461A68A12069DF00F051
:1012900008F88DF8001069461A68A02069DF002060
:1012A0003EBD68460021002280E81600704768466F
:1012B0000021002280E82600704760DF10B9174A3D
:1012C0000121117070470000144900B50878ADF590
:1012D000017D88B903E0052818BFFEF76DFF0DF505
:1012E000017D00BD5168126804A8904701A803F071
:1012F00019FD039A002AF5D14FF4FA70ADF80000F9
:10130000694604A861DF0028E5D100BF04A101A857
:1013100003F0F7FCEDE70000B82A0020336000205E
:10132000E8B9020008BA020008000000F7210180B5
:1013300017214180002101714171FB2181711B2125
:10134000C171704730B400BF6EA284B0D2E90045CD
:10135000CDE90045ADF80010ADF8021067A1D1E964
:101360000023CDE90223694602AA21E008B90E2034
:1013700070470161F72101804180FB210171F72154
:10138000C1801721018100218172C172FB2101738B
:101390001B2141730020704708B90E207047A1F14E
:1013A0001702E12A01D3072070470180002070470F
:1013B00090DF04B030BC7047F0B502468BB0908827
:1013C00000280C4640F09880118810290BD0112974
:1013D00019D0232900F07D8024295DD03A2916D028
:1013E00055293AD07FE0A01D21798171D27B012A55
:1013F00003D0022A03D1628800E022880280C079EB
:10140000884270D26CE0A01DFFF790FF6BE0A51D35
:1014100050892988884228BF08466880688817282C
:10142000B8BF17206880216900291CBF687900288F
:101430000FD000BF35A10020D1E90023CDE9002362
:10144000ADF8020069466888ADF8040020462269BC
:10145000904700206871287145E0D088A21D1728A8
:101460001188B8BF1720884228BF08465080002046
:101470001071B5DF5179002935D12069002832D0AB
:1014800024A10020D1E90067CDE90067ADF8020092
:101490005088ADF8040017E0111D68462C22FCF7B7
:1014A00039FFBDF80010BDF8040004EBC102507311
:1014B0002069C0B119A3D3E90067CDE90067ADF891
:1014C0000210507B8DF8040069462269204690473F
:1014D00009E0A01D12898179D2B2914288BF1146DC
:1014E0000020FFF72FFFA07A30B1E1880020A5DFB0
:1014F00010B9A0720120E0720BB0F0BD0000000036
:10150000000000000000000000000000770A00005A
:1015100000000000770A0000000000007ADA0000F6
:101520000000000012F003030FD1094B9A6001F193
:10153000010C4FEACC4C02EB1C42DA6000225A70DC
:101540001A7058809980002070470720704700006B
:10155000505F002080B5FAF781F9801C032190FBD1
:10156000F1F0800002BD00002DE9FC4205001446A8
:1015700018BF002C89461E4603D0FFF7EBFF8642BA
:1015800041DA00203DE0021D954249DB9CF8002035
:101590009208B25C0A5438469CF800709CF801200E
:1015A0003F0107F0300747EA22171A19F75D0F5479
:1015B0001F197F789278BF0007F03C0747EAA2170F
:1015C000401CF75D0F54401C1F19E41CBF7807F046
:1015D0003F07F65D0E54401C1AE01A192D0152788F
:1015E00005F0300545EA22151A19755DCD5552787A
:1015F00002F00F0216F822300B54401C3D220A5410
:10160000401CBDE8F6822B462146354600240020CA
:10161000471CA9F10202944203EB040C0BA6B2DBB7
:101620004C45EEDA9CF80050AD08725D0A54781C07
:10163000A9F101029CF800509442CED105F00305B7
:101640002D01725DCA553D220A54D6E751375354D5
:1016500066696A6768775A306E5770715573494A80
:10166000364C4142797A444345334748753459787A
:101670004D39504F6164386272566F586B6C6D31E2
:10168000324676354B52634E74652B2F00000000B6
:10169000254A5168106001B9506000207047224807
:1016A000006870477CB521481F4E017864240129E9
:1016B00040F6020512D1FDF72EFB012813D1306848
:1016C00040F6C411884201D3632076BDA8420ED3F0
:1016D000A0F6020044434FF4E1700FE0306840F69A
:1016E0004C11884201D3642076BDA84201D200206B
:1016F00076BDA0F6020044434FF4A570B4FBF0F0B1
:1017000076BD0948016840F63902914202D2084884
:1017100001224275704705480178012908BFFDF78D
:10172000FABA002070470000B42F00203460002077
:101730004432002010B5814CE06021616261A361F8
:1017400010BD7E4AD16849B1098810885D390F29DA
:1017500038BF401C01D308B1002010807047000042
:1017600038B5764CE06828B3754991F80421012A10
:1017700015D1018804F12C0003F04BFB78B1714DB9
:10178000E96D01202876642041430420FFF7C9FB5E
:10179000D5F8001074A0FAF76EF903F0ADFBE1681C
:1017A0000A8820885D3A0F2A38BF401C01D308B14F
:1017B0000020208031BD012860490CBF6248634889
:1017C000C86170475D49886270477CB55D4D5B4E6E
:1017D0002868401CC107286040D55D480178012970
:1017E00078D0B06803F0BAFB0446E86B208040F67E
:1017F000FF7188420CBF0120401CE863286C18B1BF
:10180000228854490A432280287D18B1218841F456
:10181000804104E0687D18B1218841F400512180A5
:10182000A01C03F009FC88B9FBF720F93062A01C6A
:10183000B16A88470446306AFBF723F9716A401899
:1018400070623CB1E0B203F047FC03E0208840F452
:1018500080502080B06803F083FB1CE071688842F0
:1018600003D30A317160FFF727FBF06980473A48DC
:10187000016800290FD4394A1068002803D40020D9
:10188000FAF7AEFD07E03648016800295CBF4FF06B
:10189000FF30FAF7A7FEA8682968814208D300F54F
:1018A000EA403030A8602F49087808B9FDF7CCF835
:1018B000A87D01280ED17088082802D1FDF7FEF915
:1018C00005E00A2803D100207080FDF7F9F970883F
:1018D000401C708073BD10B51021962003F018FBDA
:1018E000164CA06010B94FF0FF3010BD15484D21C7
:1018F000416057218160FFF704FF0A210220FFF7B2
:1019000010FB0320FFF75AFA03F018FC04F12C0037
:1019100003F04EFA002010BD0A490A686423B2FBA6
:10192000F3F3642000FB13234D2B02D24D32D21A65
:1019300002E06432D21A4D324A607047A832002069
:101940001C350020443200206117020043170200BA
:10195000346000200080FFFF9C2F0020A02F00207B
:10196000A42F0020985D00202564202074726967F0
:101970006765722C207061757365642E0D0A000016
:1019800010B5044601F0EAFA01462046096ABDE8AE
:101990001040084710B5044601F0E0FA0146204621
:1019A000896ABDE810400847C9B2830706D0521EB5
:1019B00022D310F8013B9942F7D11FE0083A13D324
:1019C00002F1040241EA012141EA014150F8043BDD
:1019D000121F21BF4B40A3F1013C2CEA030C1CF069
:1019E000803FF3D0C9B2001F083210F8013B521EED
:1019F00028BF91EA030FF8D818BF0120401E704796
:101A00000FB581B00020C04602492222425001B0E9
:101A10000FBD00002C60002000000000000000004E
:101A200028B10FF28C31800141F001010847704765
:101A3000C1888289491CC18089B2914210D100219C
:101A4000C1808188C289491C818089B2914207D1B5
:101A500000218180428841898A4208BF491C418017
:101A600070472DE9F44F064694B04FF0FF30778A67
:101A70000390019000244FEA570904A88B467F1E6B
:101A8000A04600901AE00021039128790228C8BFDF
:101A900008F10108308A33884FEA0B3A02460AEB14
:101AA000034304A909FB0030FBF71BFF00F098F883
:101AB0003FD14F4600F08EF801200190381B0828D6
:101AC0006DDA00980025A24608E0029A05A90AF1FD
:101AD000010A8B5C022BC8BF08F1010857455DDB8A
:101AE0006801029004A802990144009100F07DF879
:101AF0000AFB0030FBF7F5FE009801686D1C11F140
:101B0000010F05F00105E0D1B089328AA6F802B0D4
:101B1000AAF1010A9AFBF0F1B18000FB11AA04A816
:101B2000A6F806A000EB45111498FCF7E3FB002093
:101B300031E0287902280198C8BF08F1010810F1A6
:101B4000010F23D1308A338802460AEB034304A9EC
:101B500007FB0030FBF7C5FE00F042F808BF4C461B
:101B6000A8D0328A149804A9FCF7C4FB9DF814008D
:101B70000228C8BF08F10108B8F1020F0ADD0020F1
:101B8000A6F802B0B080F080012004E04C4600F0DE
:101B900021F893E7022015B0BDE8F08F009003987C
:101BA00010F1010F04AD7FF475AF00F01EF804A929
:101BB00004FB0030FBF795FE00F012F87FF463AFF2
:101BC000B089A6F802B094FBF0F100FB1144B1809B
:101BD000F480D9E7381B00EBD07004EB6009704744
:101BE0000098016811F1010F7047308A33884FEA7D
:101BF0000B3C02460CEB03437047F8B5C2B00546F8
:101C00000C460027698902A800EBC71679183246EE
:101C100089B22846FFF725FF4DF8270080B17F1CC9
:101C2000022FEFDB0020A880E8800098022811D165
:101C30000198022817D122980299884220D214E0F4
:101C400024B12A8A31462046FCF754FB2846FFF788
:101C5000EFFE1DE001281DD1019901290ED16889EF
:101C60006880012018E0012814D124B12A8A02A931
:101C70002046FCF73FFB6889401C08E0022909D197
:101C800024B12A8A22A92046FCF734FB688968809F
:101C9000002001E04FF0FF3043B0F0BD2DE9FE46DB
:101CA0000A9C212CBFBF1D4605FB04F341F201062F
:101CB000B34202DA0E2A164605DD0720FEF744FA83
:101CC0004FF0FF301CE0DDF82C908A4607461421C7
:101CD00002F050FDA7F800A0002038817E814FF46B
:101CE000807090FBF4F0B8814946B88995FBF0F01C
:101CF000F8817D823C82384603B0BDE8F0467CE73F
:101D0000BDE8FE86F8B505460C462889012816462A
:101D10001F4605D1FBF74DFE012811D00220288176
:101D2000A988002904BFE88800280FD1288948B96C
:101D300068883946FBF74AFE012F07D10120288128
:101D40001120F2BD022804BF00202881FAF78EFE80
:101D5000074668882B88000300EB0340AB882146C8
:101D600000EB03202C8AEB88B2B203FB0400FBF7E4
:101D70008EFE04464620FFF753FEFAF777FE3946FB
:101D8000FAF777FEC928084E02D33088401C30800D
:101D90002846FFF74DFE0CB90020F2BD3088401CEC
:101DA00030802046F2BD0000165F002000000000D9
:101DB0000338FDD87047000000000000000000005C
:101DC00028B10FF25C31800141F0010108477047F2
:101DD000428AC188521C08314282C18089B242893C
:101DE00091421CD30021C1808188491C818089B225
:101DF000102914DB002181804188491C418089B26F
:101E000010290CDB0021418041820188491C01809E
:101E100089B2C289521C9142A4BF818901800020ED
:101E200070477FB504461503668905EB0145761EAC
:101E300005EB032512E000F0B4F8009911F1010F51
:101E400004BF019810F1010F1ED1029911F1010F89
:101E500004BF039810F1010F16D1761E002E0FD487
:101E6000208A1022694606FB0050FBF73AFD002845
:101E7000E1D54FF0FF3005E0761CE680002001E060
:101E80000020E08004B070BD6089401E8642F3D11E
:101E9000E6802046FFF79CFFF0E72DE9FF4216465B
:101EA0008946370304460F2507EB09471022694688
:101EB00007EB0520FBF715FD002819D400F071F899
:101EC000009810F1010F04BF019911F1010F12D117
:101ED000029810F1010F04BF039911F1010F0AD10B
:101EE0006D1EE3D50020A080E08004B0BDE8F08244
:101EF0004FF0FF30F9E7A5802B4632464946204691
:101F0000FFF78FFFF1E7F8B50D4684B004460F27C1
:101F10002E041022694606EB0730FBF7E2FC00288E
:101F200019D400F03EF8009810F1010F04BF019998
:101F300011F1010F12D1029810F1010F04BF0399A2
:101F400011F1010F0AD17F1EE3D500206080A0802F
:101F5000E08005B0F0BD4FF0FF30FAE767803A4609
:101F600029462046FFF799FFF3E7F8B504464FF0FE
:101F7000FF35A689374607E000F013F80099A9421B
:101F80003CBF0D463E467F1CE089B84207DB042279
:101F900069463804FBF7A5FC0028EDD5B8E03046CB
:101FA000F2BD46200CE7DFB506464FF6F074B78960
:101FB00012E0FFF7F6FF009911F1010F04BF01983D
:101FC00010F1010F07D1029911F1010F04BF03981D
:101FD00010F1010F0ED07F1CF089B84210DB1022E7
:101FE000694604EB0740FBF77CFC0028E1D54FF085
:101FF000FF300DE0378039463046FFF784FF07E0B9
:102000003046FFF7B2FF308000207080B080F08053
:1020100004B0D0BD2DE9F0410E46069C054617469A
:102020009846142102F0A6FB00202881002E4FF4D0
:10203000807090FBF7F068812F82A5F80C80EC810E
:1020400003D52846FFF7AFFF00E02E802888000563
:102050000021000CFBF7BAFC0020BDE8F081F8B5C8
:1020600005460C4628890128164605D1FBF7A1FC38
:1020700001281CD002202881A988002904BFE888F3
:1020800000281CD12889B0B9EB8969882A889A422E
:1020900008BF0F2901EB021002D10121102002E03C
:1020A000401C012180B2FBF791FC01202881112006
:1020B000FEF74AF82CE0022804BF00202881FAF736
:1020C000D5FC074668882B88000300EB03402146B7
:1020D000AB88EC8800EB0320B2B200EB0410FBF7F6
:1020E000D6FC0446FAF7C2FC3946FAF7C2FCC92806
:1020F000094E02D33088401C3080FFF752FF28463B
:10210000FFF766FE0CB90020F2BD3088401C30801D
:102110004FF0FF30F2BD0000165F0020000000000D
:102120000338FDD870470000CB074CBF09230023BC
:10213000D380C1F34303C1F34311938051801080D6
:1021400070472DE9F04104463C4F2088788098463E
:10215000B980154660882388000300EB0340A388FC
:10216000E4880E2600EB03207E22B91D06FB040046
:10217000FBF7B7FB002807D4B7F90610002904BF06
:10218000B7F90800002802D14FF0FF300EE0012D12
:1021900004D100F035F84643B61D00E084264246DF
:1021A000B1B23846BDE8F041F9F728BFBDE8F0818B
:1021B0007CB515460C461E466A46FFF7B5FF33460A
:1021C0002A4644F400416846FFF7BBFF76BD38B5A8
:1021D00004461B481B4A13680D46016899420DD0FE
:1021E000FDF7A1FF0168042906D14068010C2B46C8
:1021F000224680B2FFF7DCFF012032BD002032BD55
:1022000010B500203E210D4A02EB4103B3F9064010
:1022100014F1010F02D1401C491EF5D50721B0FB76
:10222000F1F0C0F1090010BD024604484FF6FF71FD
:10223000418081800621F9F7E1BE0000FC2F0020DB
:10224000305C0020345C00202DE9FC4704460F463A
:102250002179DFF8CCA24FF02C0818FB01F00AEB33
:1022600000051646287F994610B10820BDE8F6877C
:102270000FF2CC22206852F8211002F0A2FF10B118
:102280001120BDE8F6872E60C5F804903A783B7BB4
:10229000A448012101FA02F2012BD4BF426002607E
:1022A000A14A97F800C042F82C107B78FF2B06D08B
:1022B00001FA03F64660032642F8236001E04FF07E
:1022C000FF3397F802C0BCF1FF0F1ABF002642F897
:1022D0002C604FF0FF3C94F804E0BE7818FB0EFE33
:1022E000D6448EF81F60FE78FF2E07D001FA06F65E
:1022F0000660032097F803E042F82E002079FA7870
:1023000018FB00F05044827720683A7800F5A0600E
:102310008260C360C0F810C0BA6842627A7B3B7BBF
:10232000521E9241D243D20F012B09D00AD3032B64
:1023300003D038BF42F0040204E042F0060201E09C
:1023400042F00202426522797B7918FB02F80AEB1F
:10235000080282F8203001602868D0B120683A79FC
:10236000000300165201002802D4704B1A5405E0F5
:102370006F4B00F00F00184400F8042C2268120381
:10238000121606D402F01F006A4B8140520943F82E
:10239000221000206877012028770020BDE8F6870A
:1023A00038B400F5A36210688DF800008B69486AA4
:1023B000984203D29DF800304C6923544B6A91F83F
:1023C00028005B1C4B625C1C48B10869844298BFC2
:1023D000204608618869844298BF20468861086960
:1023E000844203D2C868005D50600DE08D69AC4244
:1023F00003D291F82000506006E0834204D3AB4240
:1024000032BC8041C00F704732BC01207047F8B524
:102410000579434C2C2313FB05F52C440025667FDE
:102420000EB11120F2BD23680BB10126667704F1CD
:102430000C0391E8C05083E8C050A37F84F8285073
:10244000FF2B04D0012606FA03F3364E736012B157
:102450006577062540E00668656206F5417204204E
:102460005060C6F80851D6F808010090009B4868F3
:1024700000281ABF0B68187894F82000C6F81C05CD
:102480004868022804D309684878C6F81C0506E0A5
:10249000C868022824BF94F82010C6F81C152068CC
:1024A00010B10421116017E0D6F808010028FBD014
:1024B000C6F80851D6F80801009030460099214628
:1024C000FFF76EFF0028EFD1A07FFF2804D0012185
:1024D00001FA00F0134908602846F2BD1CB5164801
:1024E0000F4C0021016000680090009913482146BC
:1024F000FFF756FF90B9A07FFF2804D0012101FA11
:1025000000F0084908600020607720726168226846
:1025100004F1080002B0BDE81040104713BD0000F0
:10252000C45D0020080500500007005000E400E0F2
:1025300018ED00E000E100E0083102400030024008
:10254000DD2402001CB5049C0094001D03F09DF8DE
:1025500016BD00007FB504460D4616464FEA0D0035
:1025600037A11022FBF7D6FE00950196002300222A
:102570006946204603F05CF920B1FDF7E5FD4FF018
:10258000FF3003E0201D02F0AEFE002004B070BD5D
:1025900010B5094C082209212046FFF7DBFF30B9AE
:1025A0000622072104F11000FFF7D4FF18B1FDF750
:1025B000CBFD4FF0FF3010BD6433002038B504462A
:1025C000012000900D462046FFF7BCFF30B9059B67
:1025D000049A2946201D03F071F818B1FDF7B4FDE7
:1025E0004FF0FF3032BDF0B585B00024002501AEBC
:1025F00005E0102C18DA575D3755641C6D1C9D42A0
:10260000F7DB0B9A0A9B002595420FDA102CBFBF0F
:102610005F5D3755641C6D1CF6DB05E0FDF794FD2E
:102620004FF0FF3005B0F0BD0720F7E70122009220
:10263000E3B201AAFFF786FF0028EFD1F2E700001E
:102640000000000000000000000068060201000019
:1026500000B500BF130096469446103928BFA0E885
:102660000C50FAD85FEA417C28BF0CC048BF40F844
:10267000042BC90728BF20F8022B48BF00F8012B04
:1026800000BD0EB483B004AB019303B003B0704738
:10269000B0F5A07F07D13A49087808B902224A70FC
:1026A0008868496808477047E0B500BF38A0002136
:1026B000D0E90023CDE900238DF801108DF8021038
:1026C00004218DF800102F4A2FA0694603F024F949
:1026D00010B92B4A0121517003B000BD2DE9FC4710
:1026E00004460F46380091461E4608BF0E2037D0DC
:1026F000012C07D14FF00108214D687850B908200E
:10270000BDE8F687200008BF4FF48078F4D007209A
:10271000BDE8F68703280FF2700A05D1504603F092
:102720006DF90220687001E0022802D1504603F0E2
:1027300069F92C706F60AE600120009043464A46F4
:102740000021504603F07CF968780228504602D1F7
:1027500003F050F901E003F040F903206870002015
:10276000BDE8F68710B5064C6178032905D100BF96
:1027700005A003F043F902216170002010BD0000A4
:10278000A05F00209126020000900040010400009C
:102790000000000600000000B3BBD9B1B2F5803FD5
:1027A0007DD2022A1ED98C46B1FBF2F102FB11C385
:1027B0001B0443EA1043B3FBF2FC02FB1C3380B260
:1027C00040EA0343B3FBF2F002FB103240EA0C4054
:1027D00000237047022A05D98446B0FBF2F002FBC1
:1027E00010C270474AB105D100F0010249085FEA02
:1027F0003000704700220023704703F07BB90B00C4
:102800000200002100207047904271EB030CF6D3C8
:10281000B3F5803F2FD2F0B5B3FA83F7B1FA81F464
:10282000A7F10F0E3D1B5340CEF1200602FA0EF227
:10283000F3415340B5F10F0746D80F3C2C444140BB
:10284000C4F12006A040F1414140B1FBF3F603FB87
:102850001611A2FB0645001BA94102D2761E801864
:10286000594180EA010221FA0EF362FA0EF20021C8
:102870005A403046F0BD30B4B1FBF3FC03FB1C11F1
:10288000A2FB0C45001BA94103D2ACF1010C80183E
:10289000594130BC02460B46604600217047B2F1F8
:1028A000807F65D3F0B5B2FA82F7B1FA81F4C7F14F
:1028B0000F063D1B22FA06F307F1110EF2412035F7
:1028C0005A40B5F10F07B8D94140C4F12006A040E5
:1028D000F1414140B1FBF3FC03FB1C11A2FB0C4591
:1028E000001BA94103D2BCF1010C801859410F2FE4
:1028F00012D30F3FC90341EA5041B1FBF3F603FB8A
:102900001611A2FB0645D4EBC030A94102D2761EB7
:102910008018594146EACC3C07B34140C7F1200634
:10292000B840F1414140B1FBF3F603FB1611A2FBA5
:102930000645001BA94102D2761E8018594180EA43
:10294000010221FA0EF3C7F1200462FA0EF20CFA2A
:1029500007F05A402CFA04F13043F0BD80EA01023E
:1029600021FA0EF3002162FA0EF260465A40F0BDE1
:102970008C46B1FBF2F102FB11C31B0243EA106368
:10298000B3FBF2FC02FB1C331B024CEA002043EABF
:102990001063B3FBF2FC02FB1C331B024CEA002069
:1029A00043EA1063B3FBF2FC02FB1C331B024CEA4C
:1029B000002043EA1063B3FBF2FC02FB1C324CEA3A
:1029C00000200023704780B5002003F0B1F808B163
:1029D0004FF0FF3002BD80B50421684603F0CCF80B
:1029E00008B9009802BD4FF0FF3002BD704780B5B6
:1029F00000222D492D4803F017F918B1FDF7A4FB6B
:102A00004FF0FF3002BD10B5284C00E041DF2046FA
:102A100003F08CF90028F9D110BD80B51346B0F54C
:102A2000CE2F3EBF1A18521EB2F5CE2F06D200F09E
:102A30001EF803F004F918B1FDF786FB4FF0FF30E4
:102A400002BD80B51346B0F5CE2F3EBF1A18521EF8
:102A5000B2F5CE2F08D20022009200F008F803F061
:102A600011F918B1FDF770FB4FF0FF3002BD0A46B7
:102A700000F5C8310D48704780B50A46B0F5CE2F35
:102A80003EBF00EB0231491EB1F5CE2F08D200F552
:102A9000C8310023054803F025F918B1FDF754FBB0
:102AA0004FF0FF3002BD000008BA020008350020D8
:102AB00080B5DFF8D403DFF8D4230168D2F800042E
:102AC000814206D3DFF8C81391F8040108B100F081
:102AD000C4F9002002BDDFF8B403D0F80C14890A51
:102AE000A0F80A14704780B501464FF4B2624FF463
:102AF000CC20FFF792FFBDE80140FFF784BF10B57F
:102B0000044601214FF4CC20FFF7B6FFFFF77BFF0F
:102B10004FF4B26221464FF4CC20FFF792FFBDE89C
:102B20001040FFF770BFF8B5ADF5B26D07460C4623
:102B300015466846FFF7D7FF4FF6FF718F42E2AEAA
:102B400007D0B7802FB9D148D0F80C14E291FFF725
:102B5000C2FF2CB12A462146E4A8FBF7CBFBF58047
:102B60006846FFF7CCFF0DF5A06D25B0F0BD18B598
:102B70005968C84BCA689A4215D1C74C6168426807
:102B80008368002904BFA068002803D000212170B9
:102B900011BD521C10785B1E0106FAD4511C012095
:102BA0006160A360207011BD30B50A46ADF54F7D60
:102BB000014604A803F037F900F04AF8B748B64CCC
:102BC00003904FF44771002020706060A06008A857
:102BD000FBF734FA4FF4477108A8FBF72FFA08AA5D
:102BE000AF49684603F0E3FB30B39DF88C01002841
:102BF0001EBF63ADA879002826D0A268616804A82A
:102C000003F011F900F024F84FF4B27165A8FBF756
:102C100015FA65AA9F49684603F0C9FB20B90FF26F
:102C20009020F8F728FF07E0286F9E49884206D3D6
:102C300048F20100FCF70DF94FF0FF3005E0934931
:102C4000C1F80C04FFF747FF00200DF54F7D30BDA4
:102C5000684604A91022FBF75DBB80B59249088045
:102C60004FF46C30C860FFF736FFBDE80140E1E08B
:102C700010B5ADF5B26D6846FFF735FFE29911F179
:102C8000010F0BD08148E2ACC0F80C14A2880FF2FF
:102C90003C20F8F7F0FEA088FFF7DFFF0DF5B26DDE
:102CA00010BD38B504460D46FFF77EFF00280FD44F
:102CB0007648D0F80C140FF23820F8F7DCFE2A46DC
:102CC00021460020FFF72FFFBDE832400020C4E777
:102CD00031BD2DE9F84FDFF8B48108F20445934681
:102CE0002A88814690421F4618BF4FF0FF3045D1D9
:102CF000C1F30E06CC0BB246BAF1070F08BF012490
:102D000005D026B949460FF20820F8F7B4FE012095
:102D100000FA06F6688830422FD159463A4608EB49
:102D2000CA10FBF7E7FAA8883F18AF806888064307
:102D30006E80E88881450DD12888A968800210FA44
:102D400087F0884216D100F01BF8FFF75CFE00F018
:102D50002FF812E0B6B2FF2E0CD100F011F828883F
:102D6000401C28800022002180B2FFF7DCFE00F02A
:102D700061F802E00CB100F070F80020BDE8F28FBD
:102D800070B5424C04F204452888EE6810F0030F39
:102D900006EB802605D101213046FFF76DFEFFF7D7
:102DA00032FEAA8821463046FFF74BFE002070BD58
:102DB00038B5ADF5B26D6846E2ADFFF794FE4FF061
:102DC000FF34EA88E294E4A917A8FBF7A3FAE8889D
:102DD0000E900F900146E4A8FBF7E3F9334DE96844
:102DE000109014911591286900F5C830FBF7D9F9B6
:102DF000E96809911290002113900A9008910491BA
:102E0000012001210B90059101A85821FBF7C9F978
:102E100000906846FFF773FE2C600120FCF719F85C
:102E20000FF2F800F8F727FE2C600DF5A06D0020DA
:102E300025B030BDE0B51D4800210181C18040F2C0
:102E4000031311490A68ADF8023002F59672026068
:102E500006218088ADF8040011E0E0B50A49134866
:102E60000A688188ADF8041002F5967202604FF48A
:102E70008273C088ADF80600ADF8023008216846BC
:102E8000FBF7E0FF0EBD000044320020882B00203D
:102E90001C350020C09802007C5F00206F2B0200D0
:102EA000E0990200014002008C2F0020882F0020B2
:102EB00070625F6465636F64652829202D3E20661B
:102EC00061696C65642E0D0A00000000504446558F
:102ED000203A20537461727420282564206279742A
:102EE00065732C20626C6F636B202564290D0A00CA
:102EF00050444655203A206170705F73697A652CA2
:102F00002025642062797465732E0D0A000000008C
:102F100050444655203A2025640D0A005044465539
:102F2000203A2066696E69736865642E0D0A000098
:102F3000FFE741381A288041C00F7047A0F109010E
:102F4000052901D3202801D10120704700207047B6
:102F5000A0F141011A2938BF203070471A48704744
:102F600030B45368D418042B09DA41B1057804F859
:102F7000015B10F8015B15B15B1C491EF3E7536060
:102F800030BC704738B514461D4661B1FFF7E8FF05
:102F900061686A6B204690476FF00102811A02D087
:102FA000491E03D005E06FF0010032BD4FF0FF3045
:102FB00032BD0021616032BDDA6B1047024BE1E7A0
:102FC000014BF9E701487047B834002080340020F5
:102FD00080B500B906A005490B681BB1222200216B
:102FE000984701E0F7F776FB222002BD2060002021
:102FF000636F6E73747261696E742068616E646C65
:1030000065723A20626164206D6573736167650063
:1030100080B5FFF7A3FF006C02BDC3695940036A86
:10302000C161013B03627047B0B581EA030C0CF04B
:10303000004C40F2FF7515EA11541DBF15EA1357F5
:10304000AC42AF4239E0E41923EA455343F480131C
:10305000C90241F0004141EA505EC7021100A7FBDE
:10306000020200284FF00000EEFB01204FF00001AB
:10307000E3FB072118BF42F001024018002149413B
:10308000E3FB0E01A4F580640F0302D2520040411D
:10309000494154F101046CDD470872F1004250F1DE
:1030A000000051EB0451A1F580115CBF41EA0C0115
:1030B000B0BD4CEA05510020B0BD05EA1357AC4243
:1030C00014BFAF4241E050EA410E1CBF52EA430E2A
:1030D00002E061460020B0BD24423C441BD15FEABF
:1030E000070EF6D0090302BF01460020AEF1140E10
:1030F000B1FA81F7AEEB070401FA07FE0C37C7F10E
:10310000200100FA07F7C8404EEA000E23EA4553B3
:1031100043F48013A2E733F00043B3FA83F704BF0C
:10312000B2FA82FE77440B3FE41BB7F1200E2FBFAB
:1031300002FA0EF3BB40C7F1200E22FA0EFE38BF92
:1031400043EA0E03BA40641C82E750EA410E14BF02
:1031500052EA430E6FF000014FF4001717EB430FD4
:103160008ABF194617EB410FB5E74CEA055100201D
:10317000B0BDD4F10104B4F120070FDAC4F1200787
:10318000520828BF42F0010210FA07F501FA07F7CA
:10319000E1BF2A43E0403843E1400FE0352C98DCA2
:1031A000C7F1200452EA400220FA07F218BF42F0A9
:1031B000010231FA07F0A1400A43002172F10042F6
:1031C00050F1000051EB0C01B0BD0268531C0360CC
:1031D0001170704710B5144600F002F8226010BD5F
:1031E000C1F30A5343B14A0012F5001F28D2A3F2DB
:1031F000FE32A1EB0251704750EA410C20D001F0A1
:10320000004C31EA0C01B1FA81F204BFB0FA80F34C
:10321000D2180B3AB2F120032CBF00FA03F191400F
:1032200041EA0C013EBFC2F1200C20FA0CF3194315
:103230009040524240F2FD33D21A01EB03517047E5
:10324000002270474FF4001C1CEB410F94BF1CEB95
:10325000430F09E041EA030C50EA4C0C52EA0C0C13
:1032600003D2994208BF9042704714BF8B428242FA
:1032700070478068036810229B6818474FF4001C51
:103280001CEB410F94BF1CEB430F09E041EA030C18
:1032900050EA4C0C52EA0C0C03D28B4208BF82421B
:1032A000704714BF994290427047FEE7124254D4CF
:1032B00040F2FF7C1CEA11530FD0634531D09B18BC
:1032C00063453CBF01EB0251704701F0004141EA08
:1032D0000C510020FEF794BB704750EA410320D008
:1032E00001F0004C91EA0C011CD0B1FA81F30B3BC8
:1032F0009A420DD9D21A994051EA0C01C3F1200C1F
:1033000020FA0CFC61449840531C40F2FF7CD7E744
:10331000914041EA0C01C2F1200C20FA0CF3194350
:1033200090407047B0FA80F31533202BE0D3202A69
:10333000EED3203A203B9A4209D9D21A00FA03F17F
:1033400041EA0C010020531C40F2FF7CB8E700FA70
:1033500002F141EA0C0100207047524240F2FF7C2A
:103360001CEA11530DD06345DBD0B2EB030C3CBF1C
:10337000A1EB025170470CF1010221EA035141F423
:10338000801150EA410CCCD001F0004C352A27DCEA
:1033900030B481EA0C01B2F1200309DAC2F1200352
:1033A000044601FA03F5D0402843D1409C400CE08C
:1033B000C3F12002450020FA03F418BF44F00104D1
:1033C00021FA03F091400C43002174F1004550F1C3
:1033D000000051EB0C01244230BC7FF47BAF7047FE
:1033E0006146002076E7FEE7C1F30A5340F2FE3261
:1033F0009B1A14DDD3F120034FEAE17208DDC90204
:1034000041EA505141F00040D84080185040704788
:1034100003F2E13010B1D24382F000407047002047
:103420007047FEE7C11768B14840401AB0FA80F211
:103430009040D21CC907C2F5846241EA025202EBF5
:10344000D02140057047FEE770B44FF0004591EA87
:10345000030F43F111816B40841A71EB030603D211
:10346000001BB141121973414FF4001C1CEB410FBA
:1034700034BF7CEB430442E00C0DA4EB1356352E15
:103480004FDC45EAC323DB0A45EAC121C912B6F184
:1034900020050DDD63FA05F6EB4086EA03051242CE
:1034A00018BF45F00105C01851F100010CD213E01E
:1034B00062FA06F5F2405540F3415A40B340F340FA
:1034C0005A408018594107D349085FEA30005FEA43
:1034D000350528BF45F0010501F58011420875F159
:1034E000004250F1000041EB04514E0016F5001F60
:1034F00070BC38BF70470020090D090570471CEBF0
:10350000410F10D252EA43060BD0BCEB410F05D855
:103510000C0DAB43661E342EB6DD02E0AB438018C3
:10352000594170BC704770BC7047FEE7F0B540F27F
:10353000FF7581EA030C0CF0004C15EA11541DBF15
:1035400015EA1357AC42AF42E5E0BC41C1F31301A9
:10355000C3F31303801A994143F4801304D2641E09
:103560004000494180185941C90241EA5051B1FB1C
:10357000F3F603FB1611A2FB0675D7EBC020A94199
:1035800002D2761E80185941C90241EA5051B1FB5E
:10359000F3FE03FB1E11A2FB0E75D7EBC020A94161
:1035A00003D2AEF1010E80185941890241EA9051CF
:1035B000760546EA8E2EB1FBF3F603FB1611A2FB4D
:1035C0000675D7EB8020A94102D2761E801859419A
:1035D000C90241EA50514EEA060EB1FBF3F603FB75
:1035E0001611A2FB0675D7EBC020A94102D2761EA8
:1035F00080185941C90241EA5051B1FBF3F703FB6E
:103600001711A2FB0735D3EBC020A94167F10007D2
:103610000CBF004247F0010766F3D5274FEA1E3181
:10362000B80814F5806412DDBD0775F1004250EB57
:103630000E5051EB045111F5801F5CBF41EA0C01A3
:10364000F0BD4CF07F6141F0E0410020F0BDBD07CE
:103650006D0840EA0E5041F48011D4F10104B4F138
:1036600020060ADAC4F120060200E04001FA06F35F
:10367000E1401843B24015430EE0342C13DCC6F190
:10368000200445EA40056D0820FA06F2154321FAA8
:1036900006F0A1400D43002175F1004250F10000F9
:1036A00051EB0C01F0BD00205FEA0C01F0BDCFB979
:1036B00092185B41B3FA83F704BFB2FA82F6BF19DE
:1036C0000B3FB7F120062FBF02FA06F3BB40C7F14C
:1036D000200622FA06F638BF3343BA401CB1E4197B
:1036E000641E33E77F4231F00041B1FA81F404BF38
:1036F000B0FA80F6A4190B3CB4F120062FBF00FAF3
:1037000006F1A140C4F1200620FA06F638BF314385
:10371000A0403C1B1AE7AC421ABF05EA1357AF4260
:1037200012E050EA41061CBF52EA4306BFE750EAE6
:103730004107304661461CBF41EA0551F0BD52EADF
:10374000430C08BFC143F0BD00204FF4001616EB38
:10375000410F98BF16EB430F08BF16EB410F24BF74
:10376000C14305E016EB430F0CBF61464CEA05511F
:10377000F0BDFEE7400D491840EA81200CD2490D0A
:10378000A1F58061491C40F0004005DBD1F11F012B
:1037900054BFC840C017704700207047014648B169
:1037A000B0FA80F18840C91CC1F58461090501EBBC
:1037B000D02140057047FEE718B40A6812F1010FE6
:1037C0000BD0012303FA02F2DFF854341A60DFF859
:1037D00054340C68032243F824204A6812F1010F84
:1037E00004D0DFF84044002344F82230026888699E
:1037F00002F2245318604C7D087D04439C644868A1
:103800000B6802F20C542360A060087D01281ED1D1
:10381000886810F1010F04D0DFF80844002344F851
:103820002030C86810F1010F0BD0012303FA00F01B
:10383000DFF8EC331860DFF8EC33CC68032043F892
:10384000240002F5A1628868C9681160906011BC0B
:1038500070470000F8B504460E462179DFF8C8032A
:10386000174601EBC10200EB820595F8200008B174
:103870000820F2BD0FF2C832206852F8211001F082
:10388000A0FC08B11120F2BD31462046FFF794FF9D
:103890006F60306928606868002845D02068317FF3
:1038A0000022C0F810214901D0F810210092002216
:1038B000009BC0F82021D0F8202100920022009B1C
:1038C000C0F82421D0F8242100920022009BC0F8E7
:1038D0004421D0F8442100920022009BC0F85821D6
:1038E000D0F858210092009BDFF84023C0F8042351
:1038F00000030016002803D4DFF83423115406E037
:10390000DFF8302300F00F00104400F8041C216899
:103910000903091608D4012201F01F00DFF818334B
:103920008240490943F8212021680820C1F8000598
:103930000020A861E8616861012085F8200000206E
:10394000F2BD78B40479DFF8E03204EBC40503EB90
:10395000850301F06045B5F1005F1C462AD15B6923
:103960005BBB6261A1600021056805F59073196079
:1039700018680090009AC5F85811D5F858010090C1
:10398000009A6069A66805F24452166050600120F2
:10399000A8606068D8B91A68501E80419A6BC0430D
:1039A000521E9241D243D20F52EAD070F3D03AB1B4
:1039B0000F210AE072BC1020704772BC11207047C2
:1039C0000120E860986B0028FCD000226261084664
:1039D00072BC70470079944900EBC00201EB820190
:1039E0004B69581E81E02DE9F84103468E4E187947
:1039F00000EBC00406EB840C0F4607F06044B4F102
:103A0000005F1AD1DCF80400002538B1D3F800E0DB
:103A10000EF541784FF40474C8F80440DCF81840FF
:103A20009CB1DCF81C505DB120B119684FF40470F2
:103A3000C1F804031120BDE8F2811020BDE8F28135
:103A40000125CCF81010104604E0CCF81820CCF872
:103A50000C100020CCF81C000024196801F5887EA9
:103A6000CEF80040DEF8000000900098C1F8444114
:103A7000D1F844010090009801F234500760426090
:103A800015B90120086005E0D1F8000240F02000DF
:103A9000C1F800021A7902EBC2008300301DC05841
:103AA000E0B9DEF80010481E8041DEF83410C04353
:103AB0004A1E9241D243DEF81410D20F491E8941AA
:103AC000C943C90F42EAD0700843EAD006F118058D
:103AD000EC5001B103242AB10F2403E04FF4047029
:103AE000C1F804032046BDE8F2818041C043C00F05
:103AF000704780B584B00346012002918DF8000024
:103B00000192684619685A680DE080B584B0024693
:103B100000208DF800000291002190680190516111
:103B2000684611685268904705B000BD78B50446F4
:103B300004F5887685B00D467169D9B930680028DA
:103B400036D03160316800910098D4F83C15A869EE
:103B500081422DD1EA68E86930B3D4F8003223F00D
:103B60002003C4F80032E869A8612869E8600020F1
:103B7000E8611AE0002070617069009002200099ED
:103B80008DF804000021D4F88004C4F88004049067
:103B9000D4F83C050390E8680290A961E96101A8A6
:103BA00029686A68904703E0A8612846FFF7A1FFEB
:103BB000706B78B100217163706B00900099A869F7
:103BC00040B10021A961E9612846D4F83C15EA68B2
:103BD000FFF78FFF306970B10021316130690090CB
:103BE00001200099E060686928B104F23C51284640
:103BF0000969FFF78AFFB06C60B10021B164B06C55
:103C000000900099686928B104F23C51284609697E
:103C1000FFF77BFF06B070BD0349084886E7000048
:103C20000805005000070050405E002010034200CD
:103C300000E400E018ED00E000E100E000200040BA
:103C4000193C020018B40A6812F1010F0BD00123CD
:103C500003FA02F2DFF8BC341A60DFF8BC340C68F7
:103C6000032243F824204A6812F1010F04D0DFF840
:103C7000A844002344F822300268886902F22453E1
:103C800018604C7D087D04439C6448680B6802F210
:103C90000C54A0602360087D01281ED1886810F1B3
:103CA000010F04D0DFF87044002344F82030C868C6
:103CB00010F1010F0BD0012303FA00F0DFF85434A8
:103CC0001860DFF85434CC68032043F8240002F570
:103CD000A1628868C9681160906011BC70470000DB
:103CE0002DE9FC4104460F4690462179DFF82C046B
:103CF0002C2212FB01F2851805F12906707810B10B
:103D00000820BDE8F6810FF22C42206852F82110FD
:103D100001F057FA00B19FE039462046FFF792FFC5
:103D2000C5F8048038692860686880B32068397FE6
:103D30000022C0F81C214901D0F81C210092002269
:103D4000009BC0F84421D0F844210092009BDFF88A
:103D5000D023C0F8042300030016002803D4DFF8A2
:103D6000C423115406E0DFF8C02300F00F00104414
:103D700000F8041C21680903091608D4012201F087
:103D80001F00DFF8A8338240490943F82120216849
:103D90000420C1F800050020A861E8613070686166
:103DA000012070700020BDE8F68181B00022C0F8CB
:103DB0001C21D0F81C210092009B8A680B6AD25CFF
:103DC000D1F820C00CF1010CC1F820C0C0F81C25AE
:103DD00001B070472DE9FC4104462C202579DFF81D
:103DE0003C3310FB05F51D446869B8B96A61A960E8
:103DF000286285F8280000262068C0F81C61D0F8E9
:103E00001C1100910121009A81602946FFF7CDFF26
:103E1000686860B9D4F800806F690FE01CE0D1F8E1
:103E20001C010028FBD00122CA60002068613046D6
:103E3000BDE8F68129464046FFF7B7FF286A2168AA
:103E4000B842ECD2D8F81C110029F3D195F828001B
:103E50000028F7D00F26E8E71120BDE8F6810279A7
:103E6000DFF8B8122C2010FB02F288184169A2E09A
:103E700081B000680021C0F82411D0F8241100910D
:103E80000021009AC0F80811D0F808110091012112
:103E9000009A016001B0704781B08A6952B900216F
:103EA000C0F80811D0F808110091009AD0F8180550
:103EB00001B070470022C0F80821D0F80821009214
:103EC000009B4A6AD0F81805CB689854486A401C91
:103ED000486201B07047F8B506462C2034798F4B04
:103EE00010FB04F41F190023786828B1356805F524
:103EF00041704FF401744460B86970B1FB6943B11B
:103F0000786820B132684FF40171C2F804131120AF
:103F1000F2BD01233961FA6103E0BA61F9607862A8
:103F2000F86197F82900034304BF3046FFF7A0FF6C
:103F300078683168002838D10022C1F84421D1F8CE
:103F4000440100900099326802F58471C869441EEA
:103F5000A441E4430868C96BE40F401E8041C0439C
:103F60004D1EAD41ED43ED0F45EAD0702043EAD040
:103F700055EA040007D139461046FFF78DFF786AED
:103F8000B9698842DFD30020B8610CB10320F2BDCB
:103F90000DB10F20F2BD97F829003168002807BF46
:103FA00001224A6001220A6003E04FF40170C1F867
:103FB00004030020F2BD481E8041C043C00F70477B
:103FC00080B584B00346012002918DF80000019273
:103FD000684619685A680DE080B584B00246002032
:103FE0008DF80000029100219068019051616846AF
:103FF00011685268904705B000BDF0B585B00D4618
:10400000044604F5417704F584763868810523D5A4
:10401000F06908B30021F16105F12802F069009010
:104020004FF4017000997860507808B901216160FF
:1040300002208DF804000021D4F88004C4F8800424
:104040000490A8690390E8680290A961E96101A859
:1040500029686A68904727E03968480724D530689E
:1040600010B329462046FFF717FFA869696A8842FE
:104070001AD1E86940B1EA68696AA8612869E8600C
:104080000020E86168620CE005F12801487808B971
:10409000012161604FF4017078600020EA68A86136
:1040A000696A2846FFF78CFF7069B0B16869296AB0
:1040B000814207D295F8280020B929462046FFF70B
:1040C00074FE0AE0002171617069009000996869CE
:1040D00018B169692846FFF77FFFF06B98B100219E
:1040E000F163F06B0090009905F12801487808B160
:1040F00001212160A86930B10021A9612846EA6840
:10410000696AFFF75DFF05B0F0BD0449084874E730
:10411000000000000805005000070050F05D00207E
:104120008000020000E400E018ED00E000E100E0A3
:10413000002000400B41020009B90E207047130017
:1041400004D0A2F1010C1CEA020F01D00920704733
:104150000160511E818000218160C1600020704794
:1041600083688288D0F80CC0ACEB03039A4208D372
:104170000368D0F80CC002EA0C029954C168491CCB
:10418000EBE7042070478268C3689A1A0BD0036873
:10419000D0F808C0828802EA0C0C13F80C300B70BF
:1041A0008168491C01E0052070478160002070474C
:1041B00080B500E080B584B002788DF800204368B7
:1041C000019382688DF80820C068174A039002EBBB
:1041D0008102684691685268904705B000BD2DE99C
:1041E000F84F88B00378104C04EB83056A600E69C1
:1041F000AE604D7FE5546D4691E8C05F85E8C05FD5
:1042000004930378E15C31B102B1084A6946001DAC
:10421000FFF720FB05E002B1054A69460C30FFF7C5
:104220005FFD09B0BDE8F08FAC5F0020B141020036
:10423000B541020000000000000000000000000086
:1042400028B100BF4AA1800141F001010847704731
:1042500010B5040005D04FF47A70FFF7F1FF641E2B
:10426000F9D110BD38B5C0B00068354C354D401E91
:10427000092862D8DFE800F0051428612B323544A4
:104280004C5CF7F7F1FB01466846F9F7E9FEF7F7F2
:10429000EDFB6846F7F7E2FA02466946002010E0B7
:1042A000F7F7A3FE0446F7F79EFE0146621C684638
:1042B000FAF720F8F7F79DFEF7F797FE02466946F2
:1042C0000120F7F791F838E002F097FA35E041F273
:1042D0009410FFF7B5FFFAF7FDFC2EE0F7F730FC7E
:1042E0002BE043F69820FFF7B3FF0020A07595F868
:1042F000040101280CBF07200120FCF75FFD1CE032
:104300004FF47A70FFF7A4FF206CF8F769F814E017
:104310000DA0F7F7B0FB4FF4FA60FFF799FF01200B
:1043200085F8040100F0E0FD002000F0E1FD04E06C
:104330004FF4FA71022002F0A1FA002041B030BD22
:10434000443200201C3500205359535F4D455347DC
:104350005F424C455F434F4E4E45435445442C20ED
:1043600072656365697665642E0D0A0000000000C1
:104370000338FDD87047000038B5054614001EBF4D
:1043800000202060002D01D0286808B90E2032BD21
:10439000E888420800EB92729208B0EB820001D0EC
:1043A000072032BD084602F055FBC0B2142801D1E7
:1043B000052032BD2979884201DB042032BDE9881D
:1043C0002A68484310442060002032BD0078FFE78F
:1043D00000F0010070470000F8B50F4690B00546A8
:1043E000B878164600B901208DF80E0003213888F0
:1043F000ADF80C0001A8F9F721FE787C401E0021E1
:1044000004288DF8041011D8DFE800F00D09070525
:104410000300222008E0122102E0312004E02121E3
:104420008DF8041002E011208DF80400B87C401EC5
:10443000002104288DF8051011D8DFE800F00D09DF
:1044400007050300222008E0122102E0312004E0E9
:1044500021218DF8051002E011208DF80500F87B70
:104460009DF80610421E9241D24301F0F701D20F8F
:1044700041EAC2018DF8061001F0EF01387C421EBE
:104480009241D243D20F41EA02118DF8061001F099
:10449000FE013A7B501E8041C04341EAD0718DF845
:1044A000061001F0F901387D002814BF0220012018
:1044B00041EA40018DF8061009A81C21F9F7BEFD5C
:1044C000787B10F0300F29D0032102A8F9F7B6FD50
:1044D000F87C401E002104288DF8091011D8DFE86F
:1044E00000F00D0907050300222008E0122102E078
:1044F000312004E021218DF8091002E011208DF80F
:1045000009009DF80A0000F0F90040F002008DF863
:104510000A00112102A88DF808100E90787B8DF802
:10452000240004A8B97B8DF825101421F9F786FD25
:1045300003A8049001A90591B888ADF81C00B868DB
:1045400018B1F988ADF818100890BC69002C71D02A
:1045500003216846F9F772FD2088ADF82C00002190
:104560006088ADF82E0060680A90CDF834D0207BCA
:104570008DF80010401E042811D8DFE800F00D0966
:1045800007050300222008E0122102E0312004E0A8
:1045900021218DF8001002E011208DF80000B9698A
:1045A000487B401E002204288DF8012011D8DFE846
:1045B00000F00D0907050300222008E0122102E0A7
:1045C000312004E021218DF8011002E011208DF846
:1045D0000100B869817A481E80419DF80210C043ED
:1045E000C00F01F0F70141EAC0018DF8021001F09F
:1045F000EF01B869C27A501E8041C043C00F41EA42
:1046000000118DF8021001F0FE01B869027A501E07
:104610008041C04341EAD0718DF8021001F0F901E8
:10462000BA69907B002814BF0220012041EA4001B2
:104630008DF80210F86900B10C90334604AA09A95C
:104640002846AADF11B0F0BD10B5DFF8244104F10F
:104650001C0002F015FAD4E9022300211018594178
:10466000D4E90423994206D828BF904203D2B0F17E
:104670007F4061F1FF3110BD7CB504460D463C4ED4
:10468000694606F17C0002F053FA68B10470456097
:10469000694606F17C0002F073FA18B106F11C00BD
:1046A00002F0F2F9002076BD042076BD10B41300AC
:1046B00008BF07200AD000684FF0FF34C0E9024469
:1046C000012918BF002142610161002010BC704720
:1046D0002DE9FC410E46002105468DF8001090465C
:1046E000684600F02FFBD5E902234FF0FF308342EC
:1046F00008BF824208D1FFF7A7FF00278019794140
:10470000C5E90201012400E000249DF8000000F04A
:1047100035FB14B90020BDE8F6812869C5F818807A
:1047200000B12E6129460020FFF7A6FFBDE8F68103
:1047300038B5002105468DF80010684600F002FBF0
:10474000D5E902234FF0FF30834207BF82420024A5
:10475000C5E9020001249DF8000000F00FFB0CB930
:10476000002032BD29460120FFF786FF32BD000040
:10477000B82A0020002202F051BA78B405460C464F
:104780002978012902BF68780028072045D01088C1
:10479000861CB3422ED3012904D169784118891CA3
:1047A0008B4227D31B1A9B1E9BB2ADF80030694683
:1047B00010882044801C7DDF78BB2878022804D034
:1047C0006978BDF80060B14205D3BDF800108B4296
:1047D000A8BF09210ADA0821012805D16878834297
:1047E000A8BFADF8000001DAADF80030BDF8000058
:1047F000FF2802D372BC0C2070471388401CE05481
:104800001088401C108080B221541188491C1180EE
:10481000BDF8000041181180002072BC70472DE9DE
:10482000FC470A9FDDF82C803D881C460023064685
:104830008A46964699461DE039889DF80020521810
:104840001018804538DB43B9491C3980012389B2EF
:1048500004F801A03888401C388069463A88224410
:1048600001A864DFE8B939889DF80000081838808D
:1048700009F101093088814515DA706850F829007E
:1048800001900022694601A864DF50B99DF800003C
:104890007045EDD1002B14BF00200220CCE76055FD
:1048A0000020BDE8F687002BFAD03888401B401E58
:1048B00081B2B1F5807FF2DB0C20BDE8F6872DE9EF
:1048C000FC41089F099C01941646054698460097AE
:1048D0000222FFF7A4FF38B9019400974346102243
:1048E00031462846FFF79BFFBDE8F681F0B41488F7
:1048F000A51DAB4238BF0C2014D30388062B10DB58
:1049000040F68146B34203DB4FF6FF77BB4208D146
:104910004588062D05DBB5424FF6FF7704DBBD4227
:1049200006D00720F0BC7047BB4201D09D42F8D3AF
:1049300005230B55122413885B1C13809BB2CC54A7
:1049400013885B1C13809BB20B4404881C70240AE0
:104950005C7013889B1C13809BB2194440880870BC
:10496000000A48701088801C10800020F0BC70473E
:104970002DE9FC4100F12807884638681646B0B397
:10498000002523E03188401C08F8010016213088FA
:10499000401C308080B208F800103088401C308005
:1049A00080B2404421880170090A41703088801C1F
:1049B0003080A2884AB1A168C9B180B24044F9F7F9
:1049C00099FC3088A188081830806D1CE8B23979CC
:1049D00088420FD23868E9B201EB410200EB820451
:1049E000A088801CFF28CDD30C20BDE8F6810720CD
:1049F000BDE8F6810020BDE8F6812DE9FC471746A9
:104A00000546B7F80080002405F12C090E463C80CD
:104A100099F8011071B3B8F1090FC0F0FD80684634
:104A20006DDF002840F0F4803888082131541B21C4
:104A30003888401C3880062280B231540DF10101C3
:104A40003888401C388080B23044F9F753FC3988EC
:104A5000891D39809DF80000400805D189B2745441
:104A60003888401C388005E089B2012272543988A8
:104A7000491C3980A878F8B13988091D8845C0F0EB
:104A8000CB80684679DF002840F0C2803988032057
:104A9000705419213888401C388080B231543888CD
:104AA000401C388080B23044BDF800100170090A03
:104AB00041703888801C3880E878A8B13988CB1CD0
:104AC000984540B2C0F0A880022272540122398871
:104AD000491C398089B272543988491C398089B29D
:104AE00070543888401C38806868A8B139880057ED
:104AF000CB1C9845C0F09080022272540A2239885B
:104B0000491C398089B272543988491C398089B26C
:104B100070543888401C3880288958B1CDF80480FA
:104B2000009733460622022105F10800FFF7C7FE71
:104B300004006ED1288A58B1CDF80480009733461E
:104B40000722032105F11000FFF7B9FE040060D130
:104B5000288B58B1CDF804800097334615221421D4
:104B600005F11800FFF7ABFE040052D1286A30B1FE
:104B700043463A463146FFF7B9FE040049D1D5F81D
:104B800024A0BAF1000F30D0BAF804003988801C94
:104B900043189B1C98453FD3FF283DD2401C7054BE
:104BA000FF213888401C388080B231543888401C3E
:104BB000388080B23044BAF800100170090A4170A0
:104BC0003888801C3880BAF804206AB1DAF80810F6
:104BD00009B907241DE080B23044F9F78BFB39880E
:104BE000BAF8040041183980002499F8000038B15F
:104BF00043463A4631462846FFF7BAFE040008D13C
:104C0000287830B143463A4631462846FFF7B5FD8D
:104C100004462046BDE8F6870C24FAE738B400289D
:104C200018BF002A22D00024651C8D4210DA158896
:104C3000AC4203DB05196D789D4209D02546045D21
:104C40002C19641CA4B2EFE7138080B232BC704709
:104C50008C420BDA005DA31C00281EBF401E84B2EC
:104C6000002C03D014FA83F4A142EDDA32BC002008
:104C700070471CB504460020ADF8000013466A4694
:104C80002046FFF7CBFF10B1BDF80000204416BD51
:104C900080B501F0F3FF0F480F4A0168136899428D
:104CA00005D0FBF723FABDE80240FFF7DBBA0B485B
:104CB000D0F8001411F1010F03D0BDE80140FDF759
:104CC000F7BEF9F712FA012803D1BDE8014002F05E
:104CD00089B801BD085C00200C5C0020882B0020F6
:104CE00005E00A684B689A4209D1083141600268C0
:104CF000416853689942F4D1002181607047826015
:104D000070470160096804E00A684B689A4207D15D
:104D1000083141600268416853689942F4D1002229
:104D200082607047816859B103689A685118426877
:104D300081605368994203D102F108014160CFE7D5
:104D40007047FEE730B4EFF3108272B6144B9968E7
:104D500071B901249C601349134C25680D401D60F6
:104D60002160616859604FF0FF316160002100E00F
:104D70000121017002B962B630BC7047084A9168DF
:104D800061B158B9EFF3108072B6084913680B602F
:104D900053684B600021916000B962B67047000013
:104DA000885F0020FC06FFBD80E100E000E100E03C
:104DB00010B504469021F9F741F9204610BD00F1E5
:104DC00080014A68098850F83100121A142A80417B
:104DD000C043C00F704730B5B0F88230D0F884407F
:104DE00000F1400101EBC302082152F80859651B8C
:104DF000152D0ADA082D0ADA5B1E04D5083300F1F6
:104E0000400202EBC302491EEFD1002030BD012059
:104E100030BD2DE9F041804608F180060C46B068AF
:104E20000025271AF168002F13DD002931DC462CFC
:104E30002FDA3088401C81B20829A8BF00203080BA
:104E40003088716808EBC000491E0160B26842609A
:104E50001FE000291DDD96281BDB4046FFF7AFFF52
:104E6000012816D14046FFF7B6FF01287088726806
:104E700008BF0125401C81B20829A8BF002070800E
:104E8000521E708808EBC00101F140000260B16859
:104E90004160B460F7607068401C70602846BDE8EF
:104EA000F081FEE780B5012289B2F7F7A7F814492F
:104EB0000A68002804D4521CB2F57A7F28BF002269
:104EC0000A6002BD00B5C1B04FF48073009301AB1E
:104ED00001F08AFF01460129B2BF4FF0FF3001A85F
:104EE000FFF7E0FF41B000BD002200210120E9E70B
:104EF000014600220020E5E70248C26D05E00000FF
:104F0000F45F002044320020002205210520D9E76B
:104F1000F8B505460E46AF0006FB05771037384654
:104F2000F5F700F8040001D10020F2BD3946FFF783
:104F300021FC00202560A060E060666004F11000A4
:104F400000EB8500002104F1100203E042F821008B
:104F5000491C3044A942F9D32046F2BD81680EE0D5
:104F600081680268491C914228BF002181600020AD
:104F70007047C1688268914201D10020704700EB00
:104F8000810000697047C1680268491C914228BFCE
:104F90000021C160002070471CB5049C0094001DD6
:104FA00000F073FB16BD7FB575208DF80800012059
:104FB000474D484C2978019003AE0096012302AA80
:104FC0002046FDF7FBFAA8B99DF80C00672818BF2A
:104FD00008200FD11F208DF8080002AE0F2100F02D
:104FE00012F838B9202000F00BF818B9212000F091
:104FF00007F818B1FBF7A8F84FF0FF3004B070BD08
:105000008DF8080046217170012000900223297854
:1050100002AA2046C0E7E0B51F2000218DF8040059
:105020008DF8051001202A4909780090022301AA71
:105030002848FFF7B1FF0EBD78B585B004460B20B8
:105040008DF804000120224E224D3178009001237A
:1050500001AA2846FFF7A0FF30B931780C2302AA35
:10506000281D00F02BFB38B17188491C7180FBF7BB
:105070006BF84FF0FF3028E002A89DF80810427846
:1050800042EA0122228081789DF80B2042EA012227
:105090005242628001799DF80D2042EA012252427B
:1050A000A28081799DF80F2042EA0122E280017AF4
:1050B0009DF8112042EA012252422281817AC07A6F
:1050C00040EA012040426081002006B070BD00002F
:1050D000043500206433002070B50446F9F714FE4F
:1050E000154E05463068B0F5967F23D3B17D012972
:1050F00020D00120B0750220FBF760FE307E10B991
:10510000F9F7E8FD02E00720FAF7E4FF2046F7F799
:1051100067F92046012D04BF00F598508830F7F755
:105120003DFE3464204601F0A3FF2046BDE87040F8
:10513000FFF7DEBE70BD00BF4432002030B5A3B023
:1051400002F054F8040034D0002000900122694697
:10515000F7F7EEFA0125002810D4009803280DD2A5
:105160000546782205A9F7F709FB002806D4012097
:10517000009005A9A2682846904705E0002000900D
:105180000021A2682846904700900098002810D47B
:10519000656901AB02AA03A904A8A847019B029A6A
:1051A00003990498FCF7C6FAE068FCF70BFB0020B3
:1051B00001E04FF0FF3023B030BDFEE70F4801683B
:1051C000084738B50D460E49884214D100248DF8A1
:1051D00000406846FFF7B6FD08490879002811BF6E
:1051E00001240D6001220A719DF80000FFF7C6FD41
:1051F0000CB1112032BD002032BD0000E45F002060
:105200000020004001460320CA0748BF4FF4024077
:105210008A0748BF48F20120490748BF48F20220E8
:10522000704700002DE9F84305460E462979DFF85E
:1052300074059046C1EB011200EB820707F12D04C3
:105240009946607810B10820BDE8F2830FF27852D9
:10525000286852F82110FFF7B4FF10B11120BDE803
:10526000F283C7F80080C7F80490B86020702071FE
:10527000E07040F20C61707BE0723268DFF8280564
:1052800040F82210736840F823102968706832686B
:1052900001F5A1631A605860B068D8613868E8B158
:1052A000307B090309164001002903D4DFF8FC24F0
:1052B000505406E0DFF8F82401F00F01114401F822
:1052C000040C29680903091608D4012201F01F0003
:1052D000DFF8E0348240490943F821200120607062
:1052E0000020BDE8F2830279DFF8B8140068C2EB51
:1052F000021301EB83010523C0F80035022281F877
:105300002E20704701F12C03D1F828C09A6862451D
:1053100004D2496A895CC0F81C150FE01A7812B1F2
:105320000121C16106E091F820104A0604D501224E
:10533000C2615A700020704701214161012070470D
:10534000F8B400F582760022336823B13260326807
:1053500000920122009B01F12C05EB787BB1002427
:105360003462336A00930023009CB361B3690093F5
:105370000023009C736073680093009C25E0336AEF
:10538000B3BBB469002C3CD17368F3B1746073682B
:105390000093009C336A5BBBAB688C6AA34214D257
:1053A00000F5A064A6694C6AE654AB685B1CAB6070
:1053B0008C6A661EB34247D191F82060770643D4C9
:1053C0000223C0F8003201230362002A4AD00022DF
:1053D0006A70EA78002A42D1AB68896A8B423CD075
:1053E00000F5A0600021016005210160012035E089
:1053F00000233362336A00930123009C4361EB7006
:10540000E3E7B361B3690093009CAC68641CAC60D3
:10541000336A002BECD18E6AB44205D24B6A1B5D15
:1054200000F5A064E361D0E72B7813B10121C161DD
:1054300015E091F820305C0603D50121C161697047
:105440000DE001234361C0E7A342BCD10B6A5C06B7
:10545000BBD5B8D50220687001E00020E870F2BC2E
:1054600000207047F2BC01207047FEB50446DFF80B
:105470004C030090002504F582700E46056006F18D
:105480002D0701680191019A0562016A0191019A53
:10549000856181690191019A456040680190012010
:1054A0000199C4F800527563BD70206238780128F4
:1054B0001CBF0121A16031462046FFF723FF306861
:1054C000E8B140F28621B160B068C4F8040315E089
:1054D00031462046FFF734FF00281EBF0098401ECB
:1054E00000900CD10EE003250098012806DA04F2A2
:1054F000C4400021C16303250521C1636DE000990B
:105500000129E5DAB8780028EED004F2C441086831
:1055100008600028E7D0FFF775FE0546E4E7FEB512
:105520000446A6480090002504F582700E460560EA
:1055300006F12D0701680191019A0562016A019146
:10554000019A856181690191019A456040680190E5
:1055500001997563BD70B06A012805D196F82010D5
:10556000480658BF022000D50120C4F800020120DF
:1055700020623978022918BF20603068E8B140F213
:105580008621B160B068C4F8040315E031462046B6
:10559000FFF7D6FE00281EBF0098401E00900CD1D9
:1055A0000EE003250098012806DA04F2C440002129
:1055B000C16303250521C1630FE000990129E5DAE4
:1055C000B8780028EED004F2C441086808600028CA
:1055D000E7D0FFF717FE0546E4E7284603B0F0BD25
:1055E0002DE9FC410D4605F12C04617801290DD10E
:1055F000117801290FD000F541766F4F776021793E
:1056000061B1A86830601120BDE8F6810229F2D1AD
:1056100011780129EFD00820BDE8F6819E0806F038
:10562000010686F0010626712B6205F10C0192E855
:10563000C05181E8C0515168A962D168696251784E
:10564000C0F88815117801290AD0002906BF5B0926
:1056500003F00103012323702946FFF706FF02E050
:105660002946FFF75CFF296809B900222271BDE8CD
:10567000F68130B41346047900680A464949C4EB00
:10568000041501EB850130BCAAE7F0B585B06D4685
:105690000A9C00260027B446A5E8C010C0C58DF8B6
:1056A000011003920193002C14BF202200226946AE
:1056B000FFF7DFFF05B0F0BD000000002DE9F84165
:1056C00043A595E8C05185B06C4684E8C0518DF87B
:1056D00001100392019300226946FFF7CAFF06B04A
:1056E000BDE8F081F8B586B005460C46FFF728FE08
:1056F00000284DD104F12C01C878F0B9207B022894
:1057000011BF0328626AA3699A4216D1E2696262F4
:1057100000236269A262226A4B70520902F0010200
:105720000A7003282146284603D1FFF79EFE07B0E2
:10573000F0BDFFF7F4FE07B0F0BD04F10C0292E8F3
:10574000C85001A880E8C850C87898B1D5F8C404FA
:10575000C5F8C404820748BF01200BD4420748BFE4
:10576000022007D4C20748BF032003D404228DF8C7
:10577000002001E08DF8000000220A7194F820005A
:10578000420701D5C87818B1616822686846904719
:1057900007B0F0BD03490A48A4E70A494FF040208A
:1057A000A0E70000505B00200007005000E400E08C
:1057B00018ED00E000E100E086420400A086010050
:1057C000003000408C5B0020955702009B57020080
:1057D00001000000000000000000000000000000C8
:1057E00000000000000000000000000000000000B9
:1057F00010B584B00A4601788DF8001003798DF851
:10580000043041793C4B8DF8051003EB820481682C
:105810008DF80610C1688DF8071001690291406982
:105820000390A16853F822206846904704B010BD49
:105830002DE9F84F80460E4698F800B02E48924663
:1058400000EB8B0140F82BA08B60707B00284CD0C4
:105850002A4832682A4C40F20C6140F82210012795
:10586000736840F823100025316807FA01F12160C0
:10587000716807FA01F1216040F20D61326840F869
:105880002210736840F8231021A040F001094FF462
:105890008070C847A0687168C840C0071AD43068D3
:1058A00007FA00F060606D1C4FF48070C8473068E4
:1058B00007FA00F020604FF48070C847082DE9DD3A
:1058C00009E05B46314608F1040001B0BDE8F04F45
:1058D000FFF7A8BC4DB1706807FA00F060604FF4A4
:1058E0008070C847706887402760BAF1000F14BF06
:1058F000044A0022E5E70000605F00200007005036
:1059000008050050F15702000000000000000000F0
:105910000338FDD87047000078B404796C4B04EB71
:10592000440503EB8504237A13B172BC0820704749
:10593000226000264A68626000220AE04FF4A073E9
:10594000D5B203EB850503685E51521C5B59009389
:10595000009D4579D3B2AB42F0D30268CB781203F5
:1059600012165B01002A02D45A4DAB5405E05A4D81
:1059700002F00F022A4402F8043C03681B031B16C2
:1059800007D4012503F01F02544E95405B0946F8E9
:10599000235000684A78D0F804359B0802F00302CF
:1059A00042EA8302C0F804258A78D0F808359B08BB
:1059B00002F0030242EA8302C0F808250978D0F811
:1059C0001025120901F00F0141EA0211C0F810156B
:1059D00001202072002072BC704702680121116012
:1059E0000223FFE700793A4900EB400201EB820114
:1059F0000B72704700680121016070470068012147
:105A00004160704700680121C160704778B4006848
:105A10004FF480348C4000F5417553B14FF4A073BE
:105A200003EB81030026C650C3580093009E2C60F0
:105A300000E06C6000EB8100C0F8402571BC70474D
:105A4000FCB41C460568069BD5F8006240F20117BD
:105A50008F40BE43C5F80062D5F800623443C5F8F4
:105A6000004202B0F0BCD1E72DE9FC41054690466A
:105A700000275FEA08000E461BD04FF480344FF435
:105A8000A07000EB870211B2685800281EBFD5F83D
:105A9000043304FA07F0034208D000206850685825
:105AA000009010B200997168326890477F1C47459A
:105AB000E5DBBDE8F381042205490948D4E7042267
:105AC00008490948D0E7042208490948CCE7000002
:105AD0001C5E002000E400E018ED00E000E100E0C2
:105AE00000800040285E002000900040345E0020CE
:105AF00000A000407047FEE711B581B000218DF88D
:105B000000106846FFF71EF9FBF746FB50B9424C00
:105B100001A9204601F0D1FB204601F0C0FB08B1ED
:105B200001F0B9FC9DF80000FFF728F913BD000053
:105B300038B53A4D2978002409B1852032BD00B925
:105B400038A00088A5F801008DF800406846FFF7EE
:105B5000F9F8FBF721FB38B93149681C01F06AFC00
:105B6000040008D101F089FC012028709DF8000094
:105B7000FFF704F9204632BD2DE9F846054689466F
:105B8000002742F20706DFF890A000218DF80010F0
:105B90006846FFF7D7F8FBF7FFFA040007D14A463B
:105BA0002946504601F027FC074601F066FC9DF8A7
:105BB0000000FFF7E3F82CB14946284631DF0746DD
:105BC000B74204D0022FE0D03846BDE8F286052760
:105BD000FAE780B510B1032809D001BD0F4801785C
:105BE000012918D101F057FC01F05BFC01BD002038
:105BF0008DF800006846FFF7A5F8084801780129EC
:105C000005D10749401C01F015FC01F036FC9DF858
:105C10000000FFF7B3F801BDE8BB020014600020EC
:105C2000F95A02000106FEE7002818BF002901D139
:105C30000E20704701601146026813681847F8B5D6
:105C40000600154618BF002D0F461C4601D10E2038
:105C5000F2BD306808B90820F2BD0CB90920F2BDC8
:105C600017F0030F04D12246304600F089F808B936
:105C70001020F2BD234634682A46A56839463046CE
:105C8000A847F2BDF8B50400154618BF002D0F4611
:105C90001E4601D10E20F2BD206808B90820F2BDD1
:105CA00036B160684068B6FBF0F100FB116008B1E6
:105CB0000920F2BD17F0030F08BF15F0030005D14E
:105CC00032463946204600F05BF808B91020F2BD94
:105CD000069800902A4620462468E56833463946EF
:105CE000A847F2BDF8B505000E4614461F4601D17F
:105CF0000E20F2BD286808B90820F2BD0CB90920B1
:105D0000F2BD68680268511E0E4205D162433146F9
:105D1000284600F035F808B91020F2BD22462C685C
:105D2000284625693B463146A847F2BD38B50028CC
:105D30001CBF0168002915D10D490E480E4B091AE8
:105D4000A1FB0332140909D00C4D296819B1C969A6
:105D50002846884720B91435641EF6D1002032BD8C
:105D6000012032BDC969BDE8344008470000000089
:105D70001C35002008350020CDCCCCCC08350020C7
:105D8000C368994207D300695118491E884280416F
:105D9000C043C00F704700207047FEE710B543684E
:105DA0009C18446041B103E013F8010B01F8010BAA
:105DB0001046421E0028F7D1012010BD38B584B02E
:105DC0000446154669B920681D4A904209D000E092
:105DD000103D102D15D9102200F0C3F80028F7D17E
:105DE0000DE0A068A84238BF002008D323682A46E7
:105DF0002046984718B1A068451BA560012005B052
:105E000030BD2A4600F0ADF8F9E710B50446A068A9
:105E100040B1236801222046984718B1A068401E6F
:105E2000A060012010BDF8B5054B009301910292CE
:105E30000023039369461022F8F76CFA05B000BD01
:105E40009D5D0200F8B50C4605466946FFF7DDFF8B
:105E5000E0B19DF80000010603D40646266001204B
:105E6000F2BD072700F07F0669462846FFF7CDFF01
:105E700060B19DF8000000F07F00B84006439DF837
:105E80000000FF1D0106E9D5202FEDD30020F2BD53
:105E90002DE9FC410E460027002400258046694676
:105EA0004046FFF7B2FF80B19DF8000000F07F0090
:105EB00000213A4601F02CFB04439DF800000D43FD
:105EC000FF1D010603D5402FE9D3002002E0C6E9FB
:105ED00000450120BDE8F681F8B507461C460D4691
:105EE0000020164620702870306069463846FFF75B
:105EF000A9FF28B9B86808B9012121700020F2BDB6
:105F0000009810B901212170F2BDC0083060012055
:105F1000009901F007012970F2BD1CB5044631B1AA
:105F200001290ED002290ED0052913D017E0012235
:105F300000F017F8A0B19DF800000106F7D4012089
:105F400016BD082207E000F041FB48B1009A00218D
:105F5000204601E004220021FFF730FF16BD00209B
:105F600016BD6946204629E738B50D46044600F0BF
:105F70002DFB80B1284621461022F8F7CBF9A868FE
:105F80000099884201D2002032BDA9600098A16822
:105F9000091AA160012032BD2DE9FF4104461646D1
:105FA000084671680FF2AC658A7802F00F0355F865
:105FB000238012F0300709D0102F04D0202F07D0F3
:105FC000302F36D04AE0726901201070326942E009
:105FD000022822D1042B20DC756969462046FFF790
:105FE000C3FF012718B93AE02888401C288002988E
:105FF00068B1716828884A89904208D20B89326951
:10600000584302446846C0470028EDD10027019854
:106010006060029810BB384621E0736932691F88BE
:106020000E8948897E438742324417D27F1C1F80E5
:1060300011E073690888188002F00F02072A08D15E
:1060400009893069FEF796FB70683169C06800F015
:10605000FEF8326971682046C04700E0002004B0B5
:10606000BDE8F0812DE9F841144687B02569064660
:10607000286818B93046FFF750FF3DE0022911D1DA
:1060800069463046FFF770FFD8B161682B682A1D5A
:1060900068469847A8B102980028F6D10198706028
:1060A000012029E0E84671B1012903D0052908D172
:1060B000042700E008273A4669463046FFF77EFE8F
:1060C00080B9002018E000277F1C0B2FF9D2012295
:1060D00041463046FFF772FE0028F2D018F8010B57
:1060E0000106F1D43A46694603A8FFF79CFE6168B1
:1060F0002B682A1D03A8984708B0BDE8F08110B5A9
:1061000053689C7814F0C00402D0402C03D005E002
:10611000BDE8104040E7BDE81040A3E7002010BDF7
:1061200070B50D460446286886686A683146204680
:1061300001F0FFF96868206105F10C006061B0783A
:1061400000F0C000802804BF291D216170BD2DE929
:10615000F84386B006461869B768046889469046D1
:1061600000E0A468ECB1B06887421AD120680568E5
:106170002DB143464A4621463046A8470EE0806886
:1061800001884945EDD121466846FFF7C9FF012046
:1061900020736A4641463046FFF7B1FF0028E0D140
:1061A00000E0012007B0BDE8F08310B586B042687A
:1061B000937803F00F0108290ED100690468002CC0
:1061C00043D00021217368462146FFF7A9FF6846A6
:1061D000FFF7EBFFA468F2E713F0C00127D103F04B
:1061E0003004102C0DD1436919709178D36800697F
:1061F00001F00F01072910D10146184600F027F8D9
:1062000023E003F0300120291CBF03F03003302BC2
:10621000EBD140690021018017E0118923B10A46C2
:106220001946F8F767F810E0FEF7A4FA0DE08029A8
:106230000BD1016900220A6003F03001202919BF47
:1062400003F03003302B4069028006B010BD80B5EA
:106250000A4686B00146684601F06BF938B16846D7
:10626000FFF7A3FF684601F076F90028F7D107B0E1
:1062700000BD2DE9F8438AB002AB0024C3E9004415
:10628000054604A801F055F900274FF001094FF029
:10629000FF360DF10808A868002838D00DF1010379
:1062A00001AA69462846FFF717FE60B3019904A8C2
:1062B00001F091F9002840D10198B8421DD3059C06
:1062C0000598817801F00F01082934D004A801F065
:1062D00042F90598A042F3D137460198B8420CD351
:1062E000AC689DF80020014604AB2846FFF72FFF5D
:1062F000002856D0A8688442CDD19DF800102846C9
:10630000FFF70BFE39E09DF80100002849D0059801
:106310008578069C04A801F01EF90028F7D115F035
:10632000300F03D10599088800B1641C002C3AD0C5
:10633000002061092AE00788CFE70598817811F0ED
:10634000300F0CD10698402809D2410958F8212075
:1063500000F01F0009FA00F0104348F82100EC6833
:106360002CB19DF80020019904AB2846A0479DF868
:10637000001004AA2846FFF7C2FE00288BD110E0C7
:1063800058F8202012F1010F0BD1401C8842F7D39E
:1063900004F01F0458F82100C4F12004E640B04284
:1063A00001D0002000E001200BB0BDE8F08370B503
:1063B00004460D46164631462846FFF748FF32464A
:1063C00029462046BDE8704053E73EB50C46694675
:1063D000FFF75EFD68B1DDE90023DDE900015B0840
:1063E0004FEA3202C50744BFD243DB43C4E900236E
:1063F00001203EBD1CB50C4604226946FFF7DEFCB9
:1064000078B19DF800009DF8011040EA01209DF848
:10641000021040EA01409DF8031040EA016020604C
:10642000012016BD1CB50C4608226946FFF7C6FCC4
:10643000F0B19DF800209DF801009DF8043042EA7B
:1064400000229DF8020042EA00429DF8030042EA61
:1064500000629DF8050043EA00239DF8060043EA28
:1064600000439DF8070043EA0063C4E900230120CC
:1064700016BD3EB500F051F818B32A89DDE90001D8
:10648000082A08D1C4E90001D4E900238B4215D1C0
:10649000824215D012E0C117042A03D120600246BF
:1064A000D317F3E7022A03D12080B4F90020F7E7DD
:1064B000012A03D1207094F90020F1E700203EBDAD
:1064C00001203EBD3EB500F028F828B328890828F1
:1064D0000AD1DDE90001C4E90001DDE900239942A8
:1064E00017D1904217D014E0042804D1DDE900014F
:1064F00020600021F1E7022804D1DDE900012080BD
:106500002088F6E7012804D1DDE900012070207819
:10651000EFE700203EBD01203EBD0D461446694612
:10652000B6E43EB50D4614466946FFF74EFF38B354
:10653000288908280AD1DDE90001C4E90001DDE964
:106540000023994219D1904219D016E0042804D1B1
:10655000DDE900012060C117F1E7022805D1DDE97E
:1065600000012080B4F90000F5E7012805D1DDE93C
:106570000001207094F90000EDE700203EBD0120ED
:106580003EBD114636E711464CE77CB50E46044643
:10659000154600F01BF8C0B10098B0F5803F0BD253
:1065A0000099801C884207D3B17801F0C00180298E
:1065B00002D03189814201D2002076BD0098288026
:1065C000A91C009A2046FFF7F9FB76BD694639E41D
:1065D0007CB50E4605461446FFF7F8FFB0B10098AB
:1065E0000099401C884207D3B17801F0C00180298E
:1065F00002D03189814201D2002076BD009A214625
:106600002846FFF7DBFB009A0021A15476BDF8B5C0
:106610000D4684B0EF6800F017F800281ABFE8684C
:10662000002800200ED0A87800F030002028324644
:106630003946684602D1FFF7BAFE01E0FFF719FEBE
:106640000199616005B0F0BD0446164669468BE4C9
:106650000000000073640200C564020023650200AC
:1066600083650200876502008B650200D165020028
:106670000F66020000000000841A71EB030604D2CA
:106680006E40001BB141121973414FF4001C1CEB0A
:10669000410F34BF7CEB430682E00C0DA4EB135694
:1066A000362E7BDC012E45EAC32341DC43EA5253FC
:1066B00012BFD20292025B08240545EAC12141EAD9
:1066C0005051D2EBC020994125D407D1B0FA80F6C1
:1066D00010FA06F162D00020203608E0B1FA81F607
:1066E000B140C6F1200220FA02F21143B0404FEA55
:1066F000F474B4EB465434F001064FEA74040AD83B
:10670000D6F50016760D04F00044F04061FA06F26A
:106710005040F1404840C00A40EA415021F0004159
:1067200028BF5FEA500550F1000044EBD12135E06D
:10673000DB0A45EAC121C90AB6F120050EDD42EAAD
:106740000242120CC5F1200603FA06F6EB4042EABB
:1067500006056D42984161F100010DE062FA06F50F
:10676000F240554063FA06FC82EA0C02F3405A40BC
:106770006D42904161EB030111F4801F05D1641E4D
:10678000620502D06D004041494121F48011430867
:1067900075F1004350F1000041EB045170BC7047AB
:1067A0001CEB410F15D223F0004352EA43060BD0F5
:1067B0004FEA4C0CBCEB410F04D80C0D661E342E76
:1067C000B7DDEBE7801A994150EA410608BF002186
:1067D000E4E708BF1CEB430F28BF6FF00001DDE7C3
:1067E00010B5040008D000BF15A14FF47A4041F065
:1067F00001018847641EF6D110BD80B5F7F769FC2A
:10680000F8F776FAF8F75CFAF8F753FAFEF703FCB4
:10681000F7F790F94FF47A70FFF7E2FF33DFF8F7FC
:1068200046FA6420FFF7DCFFF8F743FA4FF4617093
:10683000FFF7D6FFF3E700000000000000000000B3
:106840000338FDD870470000000000000000000081
:106850003EB500BF24A191E81C0068460C2580E8E5
:106860001C008DF80050002269461B4800F0D8FE3D
:1068700008B1F9F7A1FC00203EBD000010B50C46A0
:1068800000F00EF844B100BF15A14FF47A4041F07A
:1068900001018847641EF6D1BDE8104016E00000F3
:1068A0001FB54FF4B961484341100C4C00EB917097
:1068B00080102080102268460EA1F7F72BFD0223DE
:1068C00001226946201D00F063FF1FBD012102481F
:1068D00000F092BF000000009430002090300020B3
:1068E0000338FDD870470000FFFFFFFF07020000DC
:1068F000C8050000903000200100000000000000EA
:106900000000000033B58BB00446002000900C99C5
:1069100081B1002529460CA800F0F7FF38B1009896
:10692000694601EB400295800098401C00906D1C68
:10693000142DEFD32046694687E082B012B102B031
:1069400000F0CEBF02B000F0D5BF2DE9F04F0746F2
:1069500097B03888B7F80480102806D0112845D0A1
:10696000192865D01A2846D06CE0DFF80461B068B9
:10697000C04300906846716800F0DEFF00990CA8E3
:10698000FFF7C0FF01A80CA92C22F7F7C3FC019860
:1069900098B10DF108090546B9F800A006F1040BFD
:1069A0001E245146584600F0A5FF641E0BF1040B4F
:1069B000F7D16D1E09F10209EED1B8F1140F03DB16
:1069C0000420F9F7F9FB3DE0414606F1080000F02C
:1069D00087FF4146301D00F083FFF87B022831D14C
:1069E000414606F10C0000F07BFF2BE041462148B8
:1069F00000F080FF26E03D7A1D4C2D09042DACBF30
:106A000001220022414604F11800FFF796FF022DF3
:106A1000CCBF01220022414604F11400FFF78DFF94
:106A2000022DACBF01220022414604F1100007E014
:106A3000387A38B97A7A1048D20802F00102414611
:106A4000FFF77BFF17B0BDE8F08F2C22F7F762FC51
:106A50000DB030BD10B51428044606DA21460748AB
:106A600000F053FF08B1204610BD142010BD0000F7
:106A7000D45A0020DC5A0020EC5A0020D85A0020BA
:106A80000068D0F80405704790F90410080007D496
:106A9000012201F01F00064B8240490943F82120E2
:106AA000704702490868896808470000B85F0020FD
:106AB00000E200E0000000000000000050B411B946
:106AC00050BC0E207047144694FBF3F603FB1644AB
:106AD00014B150BC092070470160828100214160DF
:106AE0008160C381002050BC7047000081B050E835
:106AF000022FC188B2EB324F4FF0000317BF92B2A2
:106B000041EA014142EA014104E04268B2EB324FFE
:106B100008BF012340E80212002AE8D18DF80030B6
:106B20009DF80000002814BF0020112001B070471C
:106B30003CB450E8015FAAB2C3891A4483899A42DF
:106B400028BFD21A03899A4202BFBFF32F8F0024B5
:106B500007E0C2EA050240E80123002BE9D14FF02B
:106B6000010401958DF80040019A0A609DF800200B
:106B7000002A1DBF006809884018002036BC7047F5
:106B80000A8849888A4209D150E8011FC1EA0141B7
:106B900040E80112002AF7D1012070470020704719
:106BA0003CB450E8025F1FFAA5F2C3889A4202BFC4
:106BB000BFF32F8F00240DE0C3891A4483899A42C2
:106BC00028BFD21AC5EA024240E80223002BE8D1CE
:106BD0004FF0010401958DF80040019A0A609DF87C
:106BE0000020002A1DBF006849884018002036BCDC
:106BF000704700000A8849888A4209D150E8021F7C
:106C0000C1EA214140E80212002AF7D10120704771
:106C10000020704762F30F2262F31F42401810F009
:106C2000030308D0C91A1FD3DB0748BF00F8012DA2
:106C300028BF20F8022D130030B414461546103931
:106C400028BF20E93C00FAD8490728BF20E90C00FA
:106C500048BF40F8042D890028BF20F8022D48BF06
:106C600000F8012D30BC7047C91818BF00F8012D7D
:106C7000CB0728BF00F8012D7047FEE74F48016899
:106C8000002900D47047F8B5F6F793FE01280DD01F
:106C90004B4E30687168884209D30120F6F772F8CC
:106CA000002803D1706800F6B8307060F1BDB1689B
:106CB00088420AD30120F7F70EFF00287DD1B06883
:106CC00000F5EA403030B060F1BD3E4F3E4C3868D0
:106CD0003E4DFEF74EF90028606039D03C4E3188B9
:106CE000802912DB06F10800F6F7EDF9002864D1DF
:106CF00030802078012804D100228621B01CF5F7CD
:106D00007DF9606800F034FE1DE000F031FE30884F
:106D1000802818DB2988B1806A8AF28020780128CF
:106D200004BF2C48F4F7A7FE06F10800F6F7CBF9EC
:106D3000002802BF30802078012804D1002286215B
:106D4000B01CF5F75BF93868BDE8F240FEF71BB9F7
:106D500020693168814230D3801D20611E4991F83D
:106D6000040150B3F6F725FE012826D0A168288833
:106D7000E268814204BF688A824205D14FF0FF3049
:106D8000206101202070F1BD1448F4F774FEE16821
:106D9000A068F6F7A0FB00280FD4E16840F2FF10CE
:106DA000491C8142E16008DD0021E160A168491CC5
:106DB000A1608142A4BF0120A060F1BDA02F0020EE
:106DC00044320020B032002020320020005F00203A
:106DD00098310020A8BA02001C350020ACBB02008C
:106DE00000F0D8BD00F0E3BD2DE9F84F012896B0C2
:106DF00098464A4D4A4F4B4E38D111A8F7F710FA32
:106E00000CA8F5F76BF901220BA90020F5F790FC0F
:106E1000307E441EA4413878E40F20B1FAF742FCDA
:106E200000F1C80702E0FAF73DFC0746F7F7A2F8C1
:106E300029683D4D0A910CAAF16D099108940692BA
:106E4000029011AB0B99306E079105930190039757
:106E500006F11B032968049140463449D1F800200B
:106E600037A100920122F9F787F953E0002818BFF3
:106E7000022808913CD108000CBF4FF0000A4FF0E7
:106E8000020AF7F741FF8346387818B1FAF70AFC8F
:106E9000C83001E0FAF706FC254A29681388254C1A
:106EA000DFF89490079106936188B9F80030234F7A
:106EB0003A885B1A0593012321880290521A089898
:106EC0002BA10190049206F11B000090CDF80CB0AC
:106ED00052464046F9F750F939882288914218BF46
:106EE0002180B9F800106288914213D0618011E0CE
:106EF00005280DD1D5F8000026A10290019206F1D7
:106F00001B030898009001224046F9F735F901E08B
:106F10004FF0FF3017B0BDE8F08F0000F45F0020A5
:106F2000346000204432002008600020B02F002090
:106F3000005F0020FC5F0020165F00200635002067
:106F4000513D313B323B25643B25733B25733A254C
:106F5000732C25732C25642C253038582C25732C44
:106F600025732C25642C25642C25643B25640000A6
:106F7000513D25643B323B25643B25733B25642C06
:106F800025642C25642C25642C25642C25643B2544
:106F900064000000513D353B323B25643B25733B8B
:106FA00025642C25643B25640000000038B500F002
:106FB00087FDFAF774FB5C4C014640F60202607DE7
:106FC000914214D200F04FF806281CBF0620F9F7B2
:106FD000F5FE2069062826D2401C0628206122D30F
:106FE0005AA0F4F748FD0320F9F774F81BE0A1F666
:106FF0000301362907D200F036F8052813D0052002
:10700000F9F7DCFE0FE001280DD10020607547493B
:1070100091F80401002814BF07200120F9F7CEFEE3
:1070200000202061E0600120C04620B90120607589
:107030000520F9F7C3FE3E4C2068401C96282060CE
:107040000FD3002020600025F7F75EFE012860685E
:1070500008BF41F28835854203D02846F5F79EFEE9
:107060006560002032BD08B901206075F9F7D4BE13
:1070700010B530492C4B4860002008602E481C6831
:10708000C2680169141B8C423CBF8918C16010BDE5
:1070900010B5284C6068002809DDC0B2FDF728FF54
:1070A0002068401C20600428C4BF002060600020CD
:1070B00010BD80B52149088808B1F9F710FF2049B3
:1070C0000878012805D0184A907D10B91D490A6832
:1070D0009047002002BD80B519490878002802BFFA
:1070E000114A907D002802D117490A689047002074
:1070F00002BD80B50020FDF7FBFE002002BD10B5EB
:107100000F48094C0078E17D81420AD0E0750020EB
:10711000FDF7EEFEE17D012903D1F7F7D1FDF7F789
:10712000C8FD002010BD0000443200201C350020A6
:10713000CC5F0020D45F002088330020DC330020A7
:10714000346000209031002094310020456E746539
:1071500072205374616E646279206D6F64652121C1
:107160002121210D0A000000BFF35F8FBFF34F8F75
:10717000374800210160416081603649C1600521C6
:107180000160BFF34F8FBFF36F8F002070478842BD
:1071900002D35118884201D3002070470120704764
:1071A00010B50A46011D0C6801462046FFF7EFFFA7
:1071B00010B94FF0FF3010BDA047002010BD2DE9E1
:1071C000F0410D4604462F689046002600E0761CEC
:1071D000A64208DA57F8260042462946FFF7D7FFAD
:1071E0000028F4D100E03846BDE8F08130B58BB01E
:1071F000FFF7BAFF184D286880474FF410314FF45D
:107200004030FFF7CDFF002808D44FF410324FF480
:1072100040310620FFF7D3FF040001D1002015E024
:10722000606880470D4908664FEA00020FF244018A
:107230000CA0F4F720FC2C2229466846F7F76AF8E0
:1072400007480A9068462168884720460BB030BD41
:1072500094ED00E0250000031434002044320020A7
:1072600077BA01004657203A2025732C2025730D4C
:107270000A0A000046572D4E52462D302E342E302D
:107280000000000001460A6810685268824201D37B
:10729000101A70478968491C081A1018704702684C
:1072A000116852688068824234BF521C00228A42B0
:1072B00001D10120704700207047F8B50446002531
:1072C0000E468DF800506846FDF73CFD2046FFF75E
:1072D000E6FF00281CBF217C002941D121684B68B2
:1072E0004A68A768BA4234BF521C00224A6030B1D3
:1072F0000868A268904234BF401C00200860E26821
:10730000012A06D0022A08D0042A0BD0082A0ED05F
:1073100015E061683078C85418E06168308821F859
:10732000130013E06168306841F823000EE06268E2
:10733000D6E9000102EBC302C2E9000106E0606881
:1073400002FB030331461846F6F7D4FF2046FFF749
:1073500099FF21688B68984238BF1846886000E022
:1073600004259DF80000FDF709FD2846F2BD024600
:10737000136818685B6839B1834203D39168491C6C
:10738000C81A7047C01A7047834201D3181A704751
:107390009268521C101A70472DE9F843044688463B
:1073A0002068D0F80090154600212046FFF7DFFF47
:1073B0000646E7686168AE4207FB09110AD307FB7E
:1073C00005F24046F6F796FFA0684D44A8420ED25B
:1073D00000250CE077433A464046F6F78BFFE2681B
:1073E0006168AD1B6A4307EB0800F6F783FF20686E
:1073F0000560BDE8F183F8B505460E461446002742
:107400000CB90020F2BD8DF800706846FDF79AFCBB
:107410002846FFF737FFA04205D3224631462846CB
:10742000FFF7BAFF00E005279DF80000FDF7A6FC76
:107430003846F2BD2A4B1A780AB185207047596048
:107440000178CA0704D527490A6842F001020A6098
:107450002549D1F800C04FEA5C0C4FEA4C0CC1F84A
:1074600000C0407821494001087021484FF4005184
:10747000016001201870002070471E4881B0002173
:10748000016000681C4A0090012000991B491060AF
:10749000086001B070471A491A4A0120086010605C
:1074A00070471749174A0120086010604FF40050D8
:1074B000154A1060BFF34F8FBFF36F8F0021084A4A
:1074C000117070470B4882B0002101600068044AC7
:1074D000009000990D4800685168C0B202B008479A
:1074E000EC5F002004D5004000D200400DE400E035
:1074F00000E100E000D1004004D3004000D0004093
:1075000008D3004004D0004080E100E008D50040EE
:10751000D2B2203A22BF00FA02F100207047524254
:10752000D041D2F1200291404140D04090404140B2
:10753000704701604160C2600021816041688B88B2
:107540001A440261B1F906301A444261088800B158
:107550000120C0B27047F8B543681A46118839B1A6
:1075600010334360198829B9C2680168FFF7E1FF49
:107570000020F2BD917814890D4605F03006302EBA
:1075800002BF9F7807F03007302F06D19588016938
:107590006D422944002401610BE001F0F001202933
:1075A00002D151894C4304E005F0C005802D08BF8D
:1075B0000424917811F0300F02D18168491C816058
:1075C00001699A88214411440161B3F906201144EC
:1075D00041610120F2BD70B504460D4666686068E1
:1075E0000188A94204D1807800F00F00082807D153
:1075F0002046FFF7B0FF6068B042F0D1002070BDB8
:10760000012070BD00EB411000F5A460116801601D
:107610009188416091688160D168C16070470000C5
:107620002DE9F04384B00C460346A648197900EBD7
:10763000C105287918B1082004B0BDE8F0832A609C
:107640006E46224604214FF0FF37DFF87CC2DFF898
:107650007CE21078FF280FD020F080084FF001095D
:1076600009FA08F9C00914BFCEF80090CEF80490CA
:1076700003204CF8280000E0B846521C491E46F88A
:10768000048BE6D11968009E01F5AC6001F2045745
:107690000660019E4660029E8660039AC26001F504
:1076A000A06001220260A679228994F805C0C7F87B
:1076B00008C03E607A60E67AA27A42EA0622026157
:1076C0000020C1F80002C1F80003C1F81C01D1F884
:1076D0001C0100900020009AC1F81001D1F810019F
:1076E00000900020009AC1F81401D1F81401009014
:1076F0000020009AC1F80401D1F804010090009A1A
:107700002868D0B12079090309164001002902D464
:107710006F4A505405E06F4A01F00F01114401F81F
:10772000040C19680903091607D4012201F01F008F
:10773000694B8240490943F821200120287104B097
:107740000020BDE8F08318B402240C714A71096866
:1077500071B18221540748BF9221140748BF41F0FC
:107760002001D406046848BF21F08001C4F800134A
:1077700000210068C0F80411D0F80411009111062E
:10778000009C4FBFC0180121C150002012BC70479F
:107790002DE9F041174604464A482279884600EB15
:1077A000C20620681D4642460021FFF72BFF2068D5
:1077B00042460121FFF726FF07F00100216800EB98
:1077C000570292B2C1F81425EA0748BF102207D425
:1077D000AA0704D500280CBF0422082200E00022DA
:1077E000C1F800223146EAB200282046BDE8F04147
:1077F00014BF0C230823A6E770B504460D46206885
:107800000026C0F8006201214160204600F00BF81C
:1078100038B9204600F007F818B92800F9D13046E9
:1078200070BD0126FBE7014626480A7900EBC2023B
:1078300000201379D1F800C0DCF80411022B18BF26
:10784000012009B101201071704738B5234C1D4D3E
:10785000E06858B10021E160E06800900099687923
:10786000410703D5296809B101208847206958B12B
:10787000002121612069009000996879010703D5F2
:10788000296809B102208847A06958B10021A16187
:10789000A069009000996879C10603D4296809B1EC
:1078A00000208847206860B1002121602168009194
:1078B000012100982971296819B1BDE834400320DD
:1078C000084731BDDC5F002000070050080500506C
:1078D00000E400E018ED00E000E100E004C1014038
:1078E0000B46012103F01F025B09914000EB83006E
:1078F00000F014B80B46012103F01F0291405B0910
:10790000C94300EB830000F017B84A0950F8220081
:1079100001F01F01C84000F00100704710B402469A
:1079200052E8004F44EA010042E8000393F0000FE0
:10793000F6D110BC7047000010B4024652E8004F68
:1079400004EA010042E8000393F0000FF6D110BCF6
:107950007047000010B40146012451E8000F40EACE
:10796000040341E8003292F0000FF6D110BC7047DA
:1079700030B507490A888B180833002450F8245082
:1079800043F82450641C042CF8DB10320A8030BD0C
:107990009831002080B51548002141700161BFF386
:1079A0005F8F001D13A1FDF7ACF9002002BD80B56B
:1079B00000218DF800106846FDF7C4F9F1EE100AB9
:1079C00020F09F00E1EE100ABFF35F8F08484021CE
:1079D00001609DF80000FDF7D1F9F9F7DDFB08B172
:1079E00041DF01BD20BF40BF20BF01BD2C5F002093
:1079F00084E200E034BB02004CBB02000400000043
:107A000070B50446207858BB6068022100F0ADF9DB
:107A10000022264B1D69586958B90021656835F95F
:107A2000125023F811504019491C0829F6DB012592
:107A30000CE0616831F9126033F9151023F8156014
:107A4000401A80196D1C082D28BF0025521C012AE0
:107A500058611D61DEDDBDE87040C008F9F718BE51
:107A600070BD00007FB500BF1AA100BF1CA52E6825
:107A7000009601A891E81C0080E81C0002228DF805
:107A8000002068460A4900F0D7F868B901A900F05B
:107A900017F948B9074C0221204600F066F918B9D9
:107AA0000221201D00F061F904B070BDB85E002015
:107AB000017A0200C45F002080B5FFF7D3FF02E027
:107AC00080B500F09AF918B1F8F73EFB4FF0FF309F
:107AD00002BD0000000000000200000100000000E4
:107AE0000100060078B5DFF83463DFF8345383B063
:107AF000706805F12D0420B300217160706800905A
:107B00000099607808B1A178D9B169680191002223
:107B10008DF800202989ADF80810E96809B92A74A0
:107B20000AE02A8B6A8369602A810021E96018B91A
:107B3000DFF8F0020121016068462A6890470020C2
:107B4000A070617800291CBF306800282DD000216A
:107B5000316031680091009821786A8B91420AD295
:107B6000501A688380B22B896C68DFF8BC22181A1F
:107B700004EB400009E08A420ED1E86840B10122DE
:107B8000A27000226A83DFF8A0221060516003E037
:107B90000120A0700020688300207060DFF884223C
:107BA00070680090012000995060306960B1002138
:107BB00031613069009000200099287402208DF80E
:107BC0000000684629688847706918B96C694FF0E9
:107BD00000462DE00020706170690090002000993F
:107BE000287404B070BDB4FA84F026FA00F18C4316
:107BF000810001F58C7109B2DFF828225058B8B124
:107C000000235350A1F58C73525800920906890E37
:107C100001F0010181F0010100988DF805100122A9
:107C2000DB088DF800208DF8043068462968884705
:107C3000002CD8D104B070BD38B4DFF8E44104F1B1
:107C40002C031A7812B132BC0820704721600278E8
:107C5000DFF8D8110A6042784A606FF00042C178BC
:107C60009970012119700021217459706161D970D6
:107C70000024DFF8BC114A60DFF8A021546054688A
:107C800000940024009D1460146800940024009D5A
:107C9000546152690092009C8078DFF8982140017D
:107CA0001070DFF89401802202600220086098784A
:107CB00008B101220A600121DFF88001016051E072
:107CC00038B4DFF85C3103F11004227812B132BC11
:107CD000112070470A79002A18BF012A03D1DFF862
:107CE0005C5100222A6003EB40031A7F12B9657FC2
:107CF0006D1C65770001CA791A770A7A5A774C7831
:107D00000B78DFF83C21240103F0030304F0300476
:107D100023438C78240204F4E0642343CC782403C6
:107D200004F4805423430C79240404F4E024234312
:107D30004C79240504F4801423438C79240604F040
:107D4000807402F1080523432B50151DCB790C7A62
:107D50002C5013500879002818BF012802D1374948
:107D600001200860002032BC704738B40246304C15
:107D70002B4B12206060187C022808BF122105D00E
:107D80001D7C012D1BD1D86820B10221216011205A
:107D900032BC704703F12D00DA60198343785BB978
:107DA0001E4B18680028FBD000251D601B6800933F
:107DB00000981D4802604160022121601CE0022001
:107DC000206003F12D05012018745A6019810020EC
:107DD000D860154C687820B128785983226060609B
:107DE0000AE02260616000210C480E4A01600068D0
:107DF0000090012000991060B4E712490A78002031
:107E0000012A01D008207047897F064A11B1012359
:107E100013607047012353607047000000710040F9
:107E2000685D0020007000402C760040F075004036
:107E30000473004007E400E000E100E0007500404A
:107E400010750040785D0020000000000000000078
:107E500028B10FF2EC51800141F001010847704751
:107E600010B5040005D04FF47A70FFF7F1FF641EDF
:107E7000F9D110BD80B5F6F72CF9DFF808040068D9
:107E8000C10548BF042002D4410505D50120BDE845
:107E90000240F8F78ABE01BD010448BF0220F6D4B3
:107EA0008004F8D50320F2E71CB5012269460220C0
:107EB000F4F73EFC0028DFF8D04305D40098401FBB
:107EC0001A283CBF0098E065012269460120F4F7BA
:107ED0002FFC002814D400990FF2F43001290DD1A1
:107EE000E26D052A0AD30120607611460FF2BC30FC
:107EF000F3F7C1FD0120F9F75EFC13BDF3F7BBFDFD
:107F000013BD00002DE9F04395B000F09DFA002864
:107F100044BF0FF2D430F3F7AEFDF6F799FE002818
:107F2000D84C03D5206840F001002060F3F774FDC1
:107F3000002803D5206840F004002060FFF7BCFD56
:107F4000002803D5206840F0080020601420FFF7C7
:107F50007FFFF4F77DFD002803D5206840F48040C2
:107F60002060F6F7A3F8002803D5206840F0200031
:107F70002060FEF76DFCF4F779FD05460020F6F76A
:107F800099F81420FFF76CFFFFF79AFD6420C046B4
:107F90000146BE480FF2CC3902680FF268300FF28A
:107FA000B038B94FF3F767FD0FF29430F3F763FD84
:107FB000F8F788F82078A9A6C1074CBF4A46324690
:107FC0000FF2983100F066F9207841074CBF4A461D
:107FD00032460FF2983100F05DF9207881064CBFEF
:107FE0004A4632460FF28C3100F054F920684104C1
:107FF0004CBF4A4632460FF2843100F04BF9FEF78F
:10800000EFFEFAF7C5FA002803D5206840F010000B
:1080100013E01420FFF724FFFCF7C5FF002803D569
:10802000206840F480602060F5F7DFFD002806DC62
:108030000020B876206840F48070206001E00121C3
:10804000B9762078C1064CBF4A46324684A100F07A
:1080500021F9206841054CBF4A46324681A100F013
:1080600019F92068C1054CBF4A4632467EA100F08E
:1080700011F900F027FA002804D5206840F04000EC
:10808000206014E0F5F7F8FB00280CD46846F5F7FB
:1080900019FC002807D49DF80000002804BF9DF8B3
:1080A0000100002803D1216841F400512160F6F756
:1080B0002BFE18B1206840F400402060FAF797FCCE
:1080C000002803D5206840F40070206007F11B00F1
:1080D000F4F704FB65A107F11B00F4F775FD70B917
:1080E00005A8F6F7B8F805AB5FF00102A5A107F106
:1080F0001B00F8F741F807F11B00F4F7DFFA05A8B9
:10810000F4F790FB05A8F3F7A9FB042804D207F1C4
:108110001B0105A8F5F7A4FF05A8F3F73EFF00280B
:1081200003D5206840F480302060217848064CBF99
:108130004A4632464EA100F0ADF8206881044CBF9B
:108140004A46324692A100F0A5F8207801074CBFBC
:108150004A46324647A100F09DF82068C10348BF57
:108160004E46324644A100F095F81420FFF778FE01
:10817000FFF7A6FC05A8F3F7B1FF05AA07F11B015D
:1081800085A0434EF3F777FCF5F7F4FE4FEA0001C4
:1081900086A0F3F770FC00BF88A0F3F76CFCF9F73A
:1081A0009AFBFFF781FE3078002814BF00200120E1
:1081B000F4F79FFDF9F773FA0746F4F7CAFC01AA32
:1081C0003946F6F74FFA019805A9F5F7DDFEBDF837
:1081D0001010BDF80E30BDF80C2000914FEA0001E0
:1081E0007BA0F3F748FC0120C04618B9206840F492
:1081F0000060206021A0F3F73EFCF4F7C3FC20A050
:10820000F3F739FCF6F708FC00E030BFF4F72EFC7A
:10821000401BC828F9D3F5F75CFFF6F751FDF6F7D8
:1082200048FD3078012808BF00F090F90320F8F7E6
:10823000C5FD216851B1FFF71DFE206830B100BFB8
:1082400074A0F3F718FC4FF0FF3003E076A0F3F7CB
:1082500012FC002015B0BDE8F08300006F6B000039
:1082600074776900696D750072746300585858001E
:108270007370690061646300626C65000D0A000040
:108280000D0A0A000860002044320020B02F0020B0
:10829000346000204046F3F7EEBB80B50120F5F7CF
:1082A00009FF0020F6F7C6FB002002BD50415553E0
:1082B00045203A20656E61626C6564202825642043
:1082C0007365636F6E6473290D0A0D0A0000000068
:1082D0005041555345203A2064697361626C65646E
:1082E0000D0A0D0A000000006770696F74652C208C
:1082F0006E6F7420696E697469616C697A65642E49
:108300000D0A00000D0A53746172742120434C4B16
:108310003D36344D487A2C20494D553D34472C3557
:1083200030304450532C2054494D45523D2564482B
:108330007A2C205645523D25730D0A0A0000000094
:108340003C5253542D44312E303E0D0A0A00000099
:10835000253873203A2025730D0A00006770696F75
:10836000000000006661756C740000007561727435
:108370000000000074696D65720000007469636B31
:1083800000000000535725303264257300000000C0
:1083900077323571000000000D0A4944203A20254B
:1083A0007320282573290D0A0A00000054494D4501
:1083B000203A2025730D0A0A0000000041637475FD
:1083C00061746F72203A2023310D0A0D0A000000FB
:1083D0005553414745203A2025732C2025642074AD
:1083E000696D657320757365642E0D0A0D0A42412F
:1083F0005454455259203A2025642C202564207479
:10840000696D657320636861726765642E0D0A0D7E
:108410000A00000053797374656D204661696C75BC
:108420007265210D0A0A000053797374656D20523C
:1084300065616479210D0A0A000000000000000057
:108440000338FDD87047000080B51A490020086045
:1084500000F0BCF968B900BF19A0016800910322BF
:108460008DF8012069460FF235020B2000F0FCF96F
:1084700020B1F7F769FE4FF0FF3002BD01210B205C
:1084800000F04CFA0C480D490068C00A00F00100E9
:1084900080F001000870002002BD00000B2808D108
:1084A000054806490068C00A00F0010080F001009C
:1084B000087070472C0700501005005034600020F1
:1084C000030002001FB5684612A11022F5F722FF33
:1084D00011208DF802000E210D208DF801108DF86D
:1084E00000004FF08051002002918DF80C00122402
:1084F0008DF80340002300226946054800F040FB48
:1085000018B1F7F721FE4FF0FF3004B010BD0000A6
:1085100034320020FFFFFFFF06FF00000000004094
:10852000000000000000000000000000000000004B
:1085300010B5040008D000BF7DA14FF47A4041F08F
:1085400001018847641EF6D110BD00002DE9F047F7
:10855000F4F78CFADFF82C1160A40FF2601A4A4E7F
:108560004A4FDFF82C810FF2341908604846F3F7C0
:1085700082FA0CE038683168884203D0F7F7B6FD1C
:10858000FBF770FE00F056F80120FFF7D1FF98F8D6
:1085900004010028EED05046F3F76DFA40F6B830EB
:1085A000FFF7C6FFF4F762FA054698F804010128C0
:1085B000DCD1F4F75BFA85420AD20020FCF798FC84
:1085C0002046F3F758FAF4F751FA00F56A4560359A
:1085D00038683168884203D0F7F788FDFBF742FE20
:1085E00000F028F80120FFF7A3FFDEE738B5F9F720
:1085F00056F8044640F6FC00844218D2F4F736FAE6
:1086000020490D68451B2348854210D34868241A29
:108610002246294637A0F3F72EFA1E48B5FBF0F0A4
:10862000B4FBF0F005288041C043C00F32BD0120EB
:1086300032BD00007CB5F4F719FA124CA1688142F2
:108640001FD2FFF73DFAF9F766F80546F6F763FB28
:108650000646F9F724F8104991F800302AA101954F
:10866000024600960020F3F716FD606810B9F9F78E
:1086700016F86060FFF7BAFFF4F7F8F900F6B830C3
:10868000A06073BD705F00200C5C0020085C0020BF
:108690001C350020C0270900346000204368656352
:1086A0006B696E6720424C4520636F6E6E65637424
:1086B00069766974792E2E2E0D0A0000476F696E57
:1086C0006720746F2073656E6420424C45206D6591
:1086D0007373616765732E2E2E0D0A0053746174D7
:1086E0007573206D6573736167652C2073656E7497
:1086F0002E0D0A0062617474657279203A20256437
:108700002C2025640D0A0000506F776572202564C7
:108710002C204368617267696E672025642D25648B
:108720002D25640D0A00000000000000000000007C
:108730000338FDD87047000038B40FF20C442568A8
:1087400000950B1898420DD26C4604EB800050F84F
:10875000043BD3F820451460491E52F8044BC3F87B
:108760002045F4D131BC7047DFF8B42302EBD001CF
:10877000012391F8542000F0070003FA00F01043A1
:10878000FFE781F854007047F0B4140007BF0824D5
:108790000C2500240825DFF888634FF0FF3306EB33
:1087A000840700E0641CAC420DD257F804CB9C4512
:1087B000F8D1331883F8304046F8241012B9311933
:1087C00081F84800234658B2F0BC7047B8B4DFF8CF
:1087D000502302F15001087A10B1B2BC0820704752
:1087E000002302F130044FF0FF35DFB24FF0000CF0
:1087F000780908BFAC4607F01F072CFA07F0C0073E
:1088000048BF25705B1C641CD8B22028EDDB1560C6
:1088100055609560D560156155619561D5611562AA
:1088200055629562D56202F15400002202600D701B
:108830004D708D70CD70C020DFF8E822DFF8E8328F
:10884000107040221A60DFF8E40200230360006821
:10885000DFF8DC3200904FF00040009A18600123EE
:108860000B720020B2BC70472DE9FC410546DFF8D1
:10887000B0627019002490F930000F4600281146AC
:108880000ED5BA78520802F001022846FFF77CFFA5
:10889000804618F1010F05D104242046BDE8F68179
:1088A0000824FAE7B878410715D4C0070AD54FF075
:1088B000A04000EB8500D0F8001721F00201C0F8BD
:1088C000001705E07878DFF87012800041F8250085
:1088D0002846FFF749FFB8783978820713D5954ABB
:1088E000964852F82830034042F828302D020904F7
:1088F00052F8280005F4F85501F440310D430543C2
:1089000042F82850C9E706EB080090F8480040EA12
:10891000811006EB080181F84800BEE738B4804BAF
:108920001C1894F93020082A23DA20D2814850F804
:10893000225045F0010540F82250900000F580706B
:1089400000B200F1804000F5C0400025056000291C
:1089500000680090009D1EBF94F9301053F821006C
:10896000002804D0012101FA02F271490A6031BCE9
:108970007047991891F948100906890F032905D104
:108980006F490968C140CA0702D503E0012901D136
:10899000022100E003214FF0A04202EB8000D0F85A
:1089A000002722F44032C0F80027D0F8002742EA1E
:1089B0000142C0F8002731BC704700002DE9F84F94
:1089C0004FEA000760A55F4EDFF86CA1DFF8509119
:1089D0004FF0010809F1500B04249BF9001011F12C
:1089E000010F3BD0C8B220F0C000C30800F007025E
:1089F000FB5C08FA02F21A4230D04FF0A04C0CEBAC
:108A0000800C5AF82030DCF800E72EF4403E0906CE
:108A10001B0CCCF800E7890F03F00303022BDCF8F2
:108A200000E70CBF032202224EEA0242CCF80027E4
:108A300008FA00F2326009EB000292F9302059F88E
:108A400022205AB1032908D0022B02D1012905D1D5
:108A500003E0032B08BF022900D19047641E0BF1ED
:108A6000010BBAD12A680092D2F820253A60009909
:108A7000C1F8202538680028ACD1BDE8F18F2DE978
:108A8000FC41002500954FF4807101220820284BFD
:108A90000CB204F1804404F5C0442668012E08D1CC
:108AA0001E68164205D000262660154324680194EE
:108AB000019E5200091D401EEAD11C48016801298F
:108AC0000BD1002202606A460068019000200199E3
:108AD0000121FFF731FE45F00045290618D0012697
:108AE000144FDFF83C8008242E420BD038683968D8
:108AF000D8F80020130005D0090C01F00301C0F3E1
:108B00000420904776003F1D641E08F10408EBD155
:108B1000002D44BF6846FFF751FFBDE8F381000018
:108B2000385C002006E400E000E100E07C610040E9
:108B3000046300401065004000070050FFE0FCFFA8
:108B400010050050200500500000005018B585B0F9
:108B50000A4601788DF80010436801938168104B34
:108B60008DF8081003EB8204C168039100698DF849
:108B70001000E16853F822206846904706B010BD07
:108B800030B40478064D45F8242005EB8405EB60ED
:108B900002B1044A234630BC001DF9F755BB000062
:108BA000D05E00204D8B020000000000000000009D
:108BB00028B10FF20C41800141F0010108477047D4
:108BC00010B5040005D04FF47A70FFF7F1FF641E72
:108BD000F9D110BD2DE9FF470746002F894603DD77
:108BE00040F2FF18C14505DB0720F7F7ADFA4FF05B
:108BF000FF3028E07C480FF2A02A07800021418046
:108C00008180C18000E07F1C474508BF01273946AD
:108C10005046F2F730FF10261025122402E00A20F9
:108C2000FFF7CEFF6846F4F74EFA0028F7D4462047
:108C3000FFF7BEFF641EF5D16D1EEED1761EEBD19F
:108C40004F45E0D1002004B0BDE8F08700002DE9D9
:108C5000F14F00288AB004DD40F2FF1081420591F7
:108C600005DB0720F7F770FA4FF0FF3071E00021C5
:108C70000A9F049100258A460391029100E07F1C1F
:108C80000498401C40F2FF1104908F4208BF012756
:108C90000FF204203946F2F7EEFEA84600244FEA10
:108CA000083000EB0740002600EB04294FF00E0BC4
:108CB0000BFB069B0E2206A95846F4F712FE46202F
:108CC000FFF776FF44EA0800304306D1BDF91810DB
:108CD0000FF2D0105A46F2F7CEFEBDF91800B84296
:108CE00004BFBDF91A00404508D1BDF91C00A042DF
:108CF00002BFBDF91E00B0426D1C01D00AF1010A8D
:108D0000761C122ED2DB641C102CC8DB08F1010883
:108D1000B8F1100FC2DB0FF2A81053462A463946AD
:108D2000F2F7A9FE03982D1802980395504402907B
:108D3000002505988742AA46A1D103990298059B70
:108D40000A9A0091019004990FF29C10F2F793FE99
:108D500000200BB0BDE8F08F4FF47A7030E72DE9BA
:108D6000F84187B010210FF2AC100FF2D0141F4D54
:108D70001F4EF2F780FE002740F6FC0840F6B830A0
:108D800097FBF0F040F6B83101FB1070F90703AA29
:108D90004CBF41464FF4FA61F5F764FCBDF818008A
:108DA000BDF81610039B3288029001917F1CBDF81C
:108DB0001400298800902046F2F75DFEFFF7CCFFF3
:108DC000B7F5FA6FDADB002008B0BDE8F08180B5B6
:108DD0000848817D0FF29010F2F74DFE0120FCF75C
:108DE0007BF9002002BD0000005F0020003500205C
:108DF000023500204432002038B50128144602D143
:108E00004FF0FF3032BD65680FF2701100F041F88D
:108E100040B9E068F3F7ECFD00F037F82946BDE80B
:108E20003440D7E60FF2601100F033F840B9E06843
:108E3000F3F7DEFD00F029F82946BDE8344006E7E7
:108E40000FF2501100F025F818B9BDE83140F3F7E2
:108E500069B90FF24C1100F01CF820B900F016F8B7
:108E6000F7F7A3FE0FE00FF2441100F012F810B96B
:108E7000BDE8314073E70FF23C1100F00AF810B979
:108E8000BDE83140A3E7002032BD0546A068F3F7F6
:108E9000AFBD2846F3F798BE626C6F636B20256404
:108EA0000D0A0000666C6173685F626C6F636B2013
:108EB0003A2025642C20253038580D0A0000000087
:108EC000626C6F636B2025303264203A2076616CCF
:108ED00069642025642C20696E76616C69642025A4
:108EE000640D0A0A00000000256420626C6F636B49
:108EF000732825642C202564292C2076616C6964F4
:108F00002025642C20696E76616C69642025640DCF
:108F10000A0000005374617274696E67207465738F
:108F2000745F7379735F626174746572795F6C6F7B
:108F30006728256429202E2E2E0D0A007379735F71
:108F4000626174746572795F6C6F67203A20256482
:108F50003A25642C203C25642C2025642C20256493
:108F60002C2025643E0D0A00747269676765725F84
:108F70006F6E203A2025640D0A000000736461744E
:108F8000615F77726974650073646174615F6368BF
:108F900065636B00626C655F74657374000000004C
:108FA0006661756C745F6C65640000006261745F7B
:108FB0006C6F6700666972650000000000000000C9
:108FC0000338FDD8704700000246136898680028EF
:108FD00000D1704770B586B06B460024002500268E
:108FE00070C370C3019190680590107910B1012889
:108FF0000AD011E001208DF8000011690291D068BB
:1090000003905069049007E002218DF80010D068A9
:109010000003029051690491684611688A6890477C
:1090200006B070BD1CB59D4C217A49B904F1B4015C
:1090300004F1A400FDF7B4FD606108B9606013BDE0
:10904000022063692072187910B1012813D024E03E
:1090500098695A69121AB2F5805F09D29208012AFA
:1090600098BF0122D9681B694118C01829DF06E0A2
:109070004FF48062F6E7D8681969081828DF10B144
:10908000112807D009E0207CB0B9BDE81C400021C0
:1090900002209FE00120207213BD60690321FFF7C9
:1090A00093FF00202072606004F1B40104F1A40079
:1090B000BDE81C40FDF79EBD13BD10B5774C201DCB
:1090C000FEF748FC002804BF607C002802D1BDE800
:1090D0001040A7E710BD000010B500BF71A16F4C94
:1090E00041602046FEF736FC50B9F8F755F8207479
:1090F0001C238C2204F1180104F1A400FDF7DEFC0E
:10910000002010BD10B5654C14212046F4F796FFE1
:1091100004F1A400FDF7EAFC002010BD2DE9FC4796
:1091200006460D46DFF878819246994669464046E4
:10913000FDF7FEFC040008BF042013D00A9F1C2189
:10914000FBF718FB002020712660A7602561C4F89A
:109150000CA0C4F8149069464046FDF711FDFFF7D6
:10916000ACFF0020BDE8F68780B510461A46F5F73B
:10917000C1F8002002BD2DE9F84381460F46DFF813
:10918000208115461E4669464046FDF7D1FC040085
:1091900008BF042011D01C21FBF7ECFA012020713C
:1091A000C4F80090A6603F0BE760656169464046E1
:1091B000FDF7E6FCFFF781FF0020BDE8F2830846DB
:1091C0007047002070473548017A481E8041C043EF
:1091D000C00F70471CB5022818BF032843D12F4C7D
:1091E000217A00293FD0022934D1022802D0032855
:1091F0001ED02FE060690021E160017959B1012999
:1092000028D10169491C01614069814222D10020B5
:109210002072002115E081694269531AB3F5805F1D
:1092200088BF4FF4805359189142816112D1EEE703
:10923000E068401C0928E0600CD30020E060207248
:109240000D216069FFF7C0FE04F1B40104F1A40030
:10925000FDF7D0FC607C10B9BDE81340E2E6BDE844
:109260001340F7F78EBF13BD0C4801214174007AFB
:10927000401E8041C00F7047012882B004D10749C9
:1092800000204874012004E0032805D10349002090
:109290004874087402B0C5E602B070471C5A00203A
:1092A000C05A00200010000004000000010000006F
:1092B000BFF34F8F7E497F480A6802F4E0620243A1
:1092C0000A60BFF34F8F00BFFDE7F8B57E487F4AC5
:1092D000016811F1010F08BF1178062905D17C49F9
:1092E0000B68C3F304217B4B19601378062B02BF74
:1092F0009168C1F30311032902D1774B77491960B3
:1093000003687749774C13F1010F08BF1378062BD8
:1093100003D12368C3F342334B601578724B062D9B
:1093200002BF9568C5F30315032D03D15D6F25F0CA
:1093300080755D67056815F1010F08BF1578062D6A
:1093400004D16A4D00262E606E600E601578062DE1
:1093500001BF9568C5F30315032D8D661578062D9D
:1093600002BF9568C5F30315032D08D1604D05268E
:109370002E600126AE670026AE603F266E6005684F
:1093800015F1010F03BF15789668C6F303164668FA
:10939000062D26D1F61E012E23D9564E564D37687E
:1093A0002F6077686F60B768AF60F768EF60376904
:1093B0002F6177696F61B7692F62F7696F62376AEA
:1093C000AF62776AEF62B76A2F63F76A6F63376BD2
:1093D0002F64776B6F64B76BAF64F76BEF64366CB9
:1093E0002E65056815F1010F08BF1578062D04D10B
:1093F0006469424D04F04F042C60046814F1010FBD
:1094000008BF1478062C06D13D4A1468E50744BF0E
:109410006FF0010515600268062A08D14468E41E51
:10942000022C04D9374A146844F4806414601A6822
:1094300042F470021A60BFF34F8FBFF36F8F03685F
:10944000314A062B05D14068C01E032884BF9068AE
:109450000862D068194B184CC10709D50121216059
:1094600018680028FCD0D5686D086D00D56011E043
:10947000116800295CBF5068002815D501212160C2
:1094800019680029FCD01520106018680028FCD04D
:109490001521516019680029FCD00020206018684F
:1094A0000028FCD0FFF704FF054806490160F1BD24
:1094B0000CED00E00400FA0504E5014000E4014081
:1094C000843300200090D00330010010E00F00F042
:1094D000240300104035014074C007400DF0ADBAC0
:1094E000380500404402001088ED00E00C01004007
:1094F000105600400404001020C50040E40E004057
:10950000000400403C170040001200102DE9F04F0D
:1095100089B0044600680293CDE9041200F0D7F840
:10952000049B5A1C00EB820650F822301E44A368AC
:109530000393236903EB82034FF0180853F8047C6C
:10954000039B304608FB073700F0CBF84FF00009CB
:1095500006900621304600F0D1F80546002800F0BC
:10956000AF800368994580F0AA8009F10109226A59
:1095700050F8293008FB03739968013100D19A60D3
:10958000DA60E6E7236A03F10108C4F820800A21C3
:10959000304600F0BCF810B133183058184405F1CB
:1095A000010A00EB8A0B50F82A309B440023082163
:1095B0005846079300F0A2F8079B002841D1129B60
:1095C000059A00935946029B204600F0A8F8002215
:1095D00006215846079200F091F8079A03460028A2
:1095E0003FD108215846079300F088F8079B0028D0
:1095F00044D1039A6369DDF808E0E06909FB0323BD
:10960000059A0EEB800CE64543D15546069B9D42DC
:10961000B8D100254FF018080821304600F06EF848
:10962000002850D003689D424DD20135226A50F87F
:10963000253008FB03739968013100D19A60DA6024
:10964000EAE702689342BAD2013350F8232009FBBB
:10965000027291680131AAD1C2F80880A7E70023FD
:10966000BFE701688A42FAD2013250F82230002B5B
:10967000AEDB09FB0373216AD960A9E70268934254
:10968000B7D20133216A50F8232009FB0272D1605E
:10969000A7E75068A8420DD190680499884209D183
:1096A0001068C3E9000E9868013008BFC3F808804D
:1096B000206AD86018330C320EF1040EA3E700259F
:1096C0004FF01809A2E7002009B0BDE8F08F10B5EF
:1096D0000821044600F01BF810B123182058184444
:1096E00010BD0368C31A1A880A2A05D95B89C218F3
:1096F00013B1C358D05870470020704710B50446C6
:1097000000F005F810B123182058184410BD036864
:10971000C01A03888B428CBF405A002070472DE945
:10972000F3470468DDF8289006460D4620460621DA
:1097300017469846FFF7EBFF00284CD02318205817
:1097400003EB000A04212846FFF7E1FF00B1285887
:10975000441C0AEB84005AF8243000220A211844E1
:1097600000F05AF877284DD0812836D0762843D19A
:10977000284600F05AF85C2849D1284600F05BF8EA
:10978000054600220421284600F046F8002204463F
:109790000621284600F040F8621C05460BD0336ACB
:1097A000013333623A46CDF80090434621463046B5
:1097B000FFF7ACFE08BB6B1C1ED0336A013333626B
:1097C0003A46434629463046CDF8289002B0BDE8D7
:1097D000F047FFF79BBE8246B4E7284600F025F825
:1097E00067280DD1284600F026F80421002200F059
:1097F00013F8411C04460CD1002002B0BDE8F087EC
:109800000020F2E7284600F010F85D28B4E70025B4
:10981000B7E74FF0FF35C2E738B505461446FFF706
:1098200076FF00B12C58204638BD08B500220A2129
:1098300000F00BF808BD10B50C210446FFF767FFD8
:1098400010B123182058184410BD38B505461446E9
:10985000FFF75DFF00B12C5C204638BD0000000022
:1098600001000100000000000100000000000000F5
:1098700002000500010000002200000000000000BE
:1098800000000000000000000000000000000000D8
:1098900001000100000000000100000000000000C5
:1098A000020005000100000042000000000000006E
:1098B00000000000000000000000000000000000A8
:1098C000010011000400FCFF040000000000000083
:1098D000020011000400FCFF040000000000000072
:1098E000030021000400FCFF040010000000000041
:1098F000040011000100FFFF010000000000000053
:10990000050011000200FEFF04000000000000003E
:10991000060011000400FCFF04000000000000002D
:10992000070011000400FCFF04000000000000001C
:10993000080017000200FEFF2400000060980200EB
:10994000090010000100FFFF010000005C98020008
:109950000A0027000200FEFF440003009098020066
:1099600000000000000000000000000000000000F7
:10997000010011000100FFFF0100000000000000D5
:10998000020017000200FEFF64010000C098020000
:1099900000000000000000000000000000000000C7
:1099A000010007000000000068010000709902003B
:1099B00002000100000000000100000000000000A3
:1099C000030005000100000042000000000000004C
:1099D0000000000000000000000000000000000087
:1099E000010017000400FCFF6801000070990200EC
:1099F000020017000400FCFFAC010000A099020067
:109A00000000000000000000000000000000000056
:109A10002DE9F04F06468BB04FF0000A06F17000BA
:109A200000F0D0F8504502DC4FF0000B59E03568EB
:109A30002846FFF74CFE0AF1010300EB830250F8C1
:109A400023300621D31828460093FFF760FE044612
:109A500010B12C582B181C44F06EC068C0460390FF
:109A60000098FFF73EFE4FEACA03049001930027D7
:109A7000049B9F4202D10AF1010ACFE700980A2114
:109A8000FFF745FE20B1009B009A0344105818448C
:109A9000013700EB870550F827301D440421284684
:109AA000FFF735FE00B128582368834240F28780D3
:109AB000013004EB800854F82030019A7168984412
:109AC000D6F880304FEA47199A58A9F120094A443C
:109AD0001C32404600F07CF8834630B1404600F02E
:109AE0009FF858460BB0BDE8F08FD6F88030019A49
:109AF0009B584B44DB69002B61D0D3F8148009904C
:109B0000B8F1200F4FF00E01284646D1FFF7FFFDB8
:109B100000283AD14FF0000BCDF808B006212846B6
:109B2000FFF7ECFDC046C046082105902846FFF728
:109B3000E5FDC046C046019AD6F8803006909B5895
:109B4000079303EB09081C220021404600F07EF831
:109B5000079B059A43F80920069BC8F80430099B27
:109B6000C8F81030029B1421C8E9053B2846FFF7CE
:109B7000C5FD00283FF47CAF0368002B3FF478AFAD
:109B8000C046C046C8F8080072E72B582A18D118FA
:109B9000043152F803B00291C0E7FFF7B8FD70B985
:109BA0007068036841469B68984740B1039A09ABC7
:109BB000294600F055F883460028ABD091E74FF0D6
:109BC000010B8EE708B58068FFF781FD006808BDCE
:109BD000002370B513600C460546164600F020F8C9
:109BE000CD2801461ADC202808D0236820461B68AF
:109BF00098473060B0FA80F0400970BD2B68EB1ACE
:109C00001A88062A0AD9DB88E9183BB1EB58226882
:109C100004335268194420469047EAE70120ECE7F4
:109C20000168411A02460B880A2B09D94B8903B1F6
:109C3000C358888800B110569842B8BF184670477C
:109C4000042B4FF00003F4D81846F5E710B504468E
:109C500010460A4601462046FCF7DCFF204610BDB0
:109C60002DE9F0410D46044616461F4600F008F85F
:109C70003B46014632462846A446BDE8F0416047CF
:109C8000044B1A681AB9044A044911601A6018682A
:109C9000704700BF2460002028600020C8BB02007D
:109CA0002DE9F04F9946436891B0CDE90713054679
:109CB0000023884681690F9307A8174600F0C9F86A
:109CC000044600285FD1059005A907A800F002F915
:109CD0000446002857D10646A7F1040A4046FFF77C
:109CE000F6FC0268059B96423ED33A46194607A801
:109CF00000F058F90446002845D1284600F0E5F95F
:109D00002146024600974B4607A8FFF7FFFB044693
:109D1000002838D16868036810211B6BDDE9097AD7
:109D2000984706466868036810229B683146984742
:109D30008046002800F08B80286903683246DB6982
:109D400041469847D5F810B03E46A146CA451ED1B7
:109D50006868D5F810B003685B6A984700268146AA
:109D600031464FF0FF3349E001362A6850F826109B
:109D7000146B5AF8362000EB860C61442846A04745
:109D800004460028AAD0204611B0BDE8F08F337DEC
:109D90001BB909F101091836D8E71021306800F025
:109DA00098F93269531C0146DBF8003008D19C68F1
:109DB0005846D6E90223A04704460028E9D0E2E746
:109DC0000092DC685846D6E90223A047F4E73A7DC2
:109DD00092B1DBF8002006939469039106AA5846D5
:109DE000A04704460028CED1069A786803994A44D1
:109DF000026001314FF0FF3301361837B245E6D12A
:109E000007A800F06DF9686803684146DB68984769
:109E1000686803685B69984704460028B3D168689E
:109E2000E96903681B6A984704460028ABD1286992
:109E300003681B6998472B6A834238BF28626868A9
:109E4000296A036810229B6A984704469BE701240D
:109E500099E72DE9F843044600688846FFF737FC88
:109E6000636801681A688900956818460422A84743
:109E70000746206160B30026D4F800903546484676
:109E8000FFF725FC03689E4212D36068C4F81C806B
:109E90000368C4E90555182145449B68E560042220
:109EA00069439847A060B0FA80F04009BDE8F883A4
:109EB00047F826504846FFF70AFC013600EB8602B9
:109EC00050F82600104400F019F903681D44D6E745
:109ED0000120EBE72DE9F04705680746884628464C
:109EE0001021FFF714FC10B90020BDE8F087DFF85F
:109EF000B090002610212846FFF709FC00284DD01D
:109F00002B582A18D118D3589E42EDD2013601EBB6
:109F1000860A51F826309A4404215046FFF7F7FB91
:109F20000028E7D00AEB00025AF80030D458D018C5
:109F3000172C2246494628BF17220430F1F7A9FC06
:109F40000028D7D1172CD5D10C212846FFF7DFFBED
:109F5000044610B12C582B181C4406215046FFF71C
:109F6000D6FB08B15AF80000431C04EB830254F8F6
:109F70002340144404212046FFF7C9FB60B1225856
:109F800023181344103353F8042CC8F80030BB696D
:109F90009A42AFD00120A8E7C368FFDE0368FCE760
:109FA0004CBB02002DE9F04F85B08368009300257B
:109FB000131F04460191AA4602934FF0FF3B20680D
:109FC000FFF785FB03689D4211D363690099E0693F
:109FD000182202FB0313012400224FF0FF319042AC
:109FE00003F1180369D1002005B0BDE8F08F0135F9
:109FF00000EB850850F825309844029B53F83560F3
:10A00000236903EB850332464146204653F8047C1E
:10A0100000F07EF80028E7D1009B182101FB0739EA
:10A020000746404600F06AF803689F42C7D2C9F865
:10A0300004604946304600F0A8F80028D4D13368BF
:10A04000C9E902BB013763BB4046039300F056F8F1
:10A0500000EB870C50F82700604400F0B0F8039B39
:10A0600020B9D9F80030003B18BF012389F814301B
:10A07000019BFBB153F82A30C9F8103040460393D6
:10A0800000F03CF800EB870C50F82700604400F02B
:10A0900096F8039B38B90AF1010A09F118090C3640
:10A0A000BFE70346E2E70133F5D04FF0010389F83B
:10A0B0001430F0E7C9F810B0EFE743E9041103F8F2
:10A0C000044C43F8081C013289E7C069042100F000
:10A0D00081B8431E0B44B3FBF1F301FB03F070475F
:10A0E00010B504464068A1680368DB68984760685B
:10A0F00021690368DB689847002010BD10B5042172
:10A100000446FFF704FB10B123182058184410BD73
:10A110002DE9F34708460C461646FFF7E2FA4FF0E2
:10A12000000805464FF0FF37A84501D1002029E07F
:10A130000A212046FFF7EBFA10B1231820581844E3
:10A1400008F1010800EB880950F828304FF0000AA8
:10A15000994414214846FFF7D1FA0028E4D0036857
:10A160009A45E1D20AF1010A01A950F82A30019773
:10A170000C2000FB036000F008F818B9019B002BCD
:10A18000E7D0012002B0BDE8F087436873B50D4603
:10A190009BB1196800220124914209DC007A01A9CF
:10A1A00000F01EF810B9019B63432B6002B070BD34
:10A1B00053F8046F01327443EEE70124EEE710B563
:10A1C0000E210446FFF7A3FA00B1205C003818BF47
:10A1D000012010BD4B1E1844B0FBF1F048437047FE
:10A1E000122804D8092804D8022824D858BB0120F2
:10A1F00070470A380828FAD801A353F820F000BFA6
:10A200002FA202004BA202004FA202004BA20200AA
:10A2100047A20200EFA1020047A20200EFA1020044
:10A2200043A2020012F4887F0FD10728DFD1022356
:10A230000B6000207047012303FA00F212F4127F32
:10A24000F0D00123F4E70423F2E70823F0E710231A
:10A25000EEE700BF2DE9F04F016887B00546C06EFC
:10A2600000F0CEF8014638B9012385F89130012479
:10A27000204607B0BDE8F08F05F170073846016150
:10A28000C0462846FFF7C4FB04460028F0D105F17C
:10A29000A006014630460161C046384600F0ECF8A1
:10A2A00004460028E4D1012130460161C046384609
:10A2B00000F013F904460028DAD10221304601618A
:10A2C000C046D5F880202968E86E05F1940300F0B7
:10A2D00034F904460028CBD1D5F8941030464161BA
:10A2E000C046EF6E28683B68D3F81C8000F041F947
:10A2F00081003846C047C5F898000028B7D0A3466B
:10A3000025E0D5F880201B68049238460393FFF7B8
:10A31000DEF94368043306211844FFF7EFF90134EE
:10A32000D5F898A0CDF800B050F82430049A3946FA
:10A330004846039FB8474FEA8408A8F10408D5F8B7
:10A3400098304AF8080053F80830002B8FD02F6857
:10A35000384600F00EF9D5F86C90A042D9F80030DC
:10A36000CFD83846DC6900F00FF981004846A04795
:10A37000C5F89C0000283FF47AAF0024A346D5F826
:10A380000080404600F000F9A0420ED8284600F0B8
:10A3900006F9044600287FF46BAF012385F890305E
:10A3A000032130460161C04662E7D5F86C90D5F8CC
:10A3B0008020D9F8003005921B6804934046FFF7CF
:10A3C00086F94368043308211844FFF797F90134EC
:10A3D000A700D5F89CA0CDF800B03B1F059A0393C9
:10A3E000049F50F8243041464846B847039B039ADF
:10A3F0004AF80300D5F89C309B58002BBFD136E7B4
:10A40000F8B5037D04460E4613B100252846F8BD75
:10A41000012303758068036804229B68082198471C
:10A42000A368144AC0E90023E060204600F0C4F8A5
:10A430000028EAD1A5682B6830469F68FFF747F9E6
:10A44000016804222846C900B84705460028DCD028
:10A4500023680246DB6A3146204698470028D4D15B
:10A4600023682A469B6A3146204698470028CDD06B
:10A47000CBE700BF6CBB02002DE9F047D0F8149089
:10A4800004460026E3691B689E4204D3C4F8149076
:10A490000020BDE8F087A0686661314600F09BF8B7
:10A4A0004FEAC60A80460027474501D10136E9E751
:10A4B000236953F80A5005EB4715D5E90410EB69F9
:10A4C0005A691B68202A06BFAA690146002213B1F7
:10A4D00060689847E8600137E6E72DE9F843D0F86F
:10A4E000148004460025E3691B689D4204D3C4F828
:10A4F00014800020BDE8F883A0686561294600F05B
:10A500006AF84FEAC50907460026B74201D101356E
:10A51000E9E7236953F8091001EB4611CB699B6801
:10A520002BB93146E06800F06AF80136EDE7606863
:10A5300098470028F5D00120DCE72DE9F0411D46C1
:10A54000037D04460E4617468BB1036882691B6C77
:10A550002946984748B923683A46D3F83C802B6887
:10A5600031462046C04700B92075BDE8F081012082
:10A57000FBE708B5FFF7ABF843680433062118443E
:10A58000FFF7BCF8006808BD08B5FFF7A0F84368FE
:10A59000043308211844FFF7B1F8006808BD10B56E
:10A5A00000F17004204600F04BF820B92046BDE8C9
:10A5B000104000F06FB810BD002310B50446836151
:10A5C0004068036804229B6990219847E061B0FAD3
:10A5D00080F0400910BD0368C31A1A88082A0CD9F4
:10A5E0001B89C2180BB1C3581344013103EB81001E
:10A5F00053F821301844FFF774B80023F5E70368D7
:10A6000070B55B6904460D469847C0B92046FFF710
:10A610005CFDA2690C235A438318984209D16068F3
:10A62000E1690368DD699032AC460423BDE87040FF
:10A6300060474168013108BF45600C30EDE770BDEF
:10A640002DE9F843D0F8148004460025E3691B681F
:10A650009D4204D3C4F814800020BDE8F883A068AC
:10A6600065612946FFF7B7FF4FEAC509074600268F
:10A67000BE4201D10135E9E7236953F8093003EB04
:10A680004613DA6922B1126912B1D968606890473D
:10A690000136EDE72DE9F04F054685B000264FF075
:10A6A0000C0BEB691A68964207D3A869002863D19E
:10A6B0000023184605B0BDE8F08F013603EB86088D
:10A6C00053F826304FEAC6099844A9F10809002733
:10A6D00004214046FFF71BF8002853D058F80030FB
:10A6E00008EB0002D118D3589F42DAD2013701EBB0
:10A6F000870451F827301C440E212046FFF707F845
:10A700000028E5D0235C002BE2D02B694B440BFBE7
:10A7100007FA5868AAF10C0A03A95044FFF735FD5F
:10A7200003460028C5D1019006212046FEF7EFFF21
:10A730000146A0B12256019B092A1BD10C212046BB
:10A74000FEF7E5FFA0B1231824581C440A21204637
:10A75000FEF7DDFF98B122582318134459682B697E
:10A76000039A4B445B6853F80A00FFF76FFAAFE7B0
:10A770000446EBE71946F2E700F006F898E743686D
:10A780008368FFDE0368FCE770B5054600241426E5
:10A79000AB68A34201DC002070BD2B6806FB0433CC
:10A7A0000134DA6893F910109868FFF74FFAEFE771
:10A7B0002DE9F04F85B01C460F9D80468A46934692
:10A7C000002120222846FFF741FA204600F0B4F885
:10A7D00005F11C0100F0B8F80746002850D12046CA
:10A7E000FFF7EDFC0E99A877204600F0B9F8002895
:10A7F00014BF0123022328616B7703AA05F1180116
:10A80000204600F0C7F80746002839D10421204629
:10A81000FEF77DFF002837D0221820581044C0468C
:10A82000C04668610C212046FEF771FF40B32358F3
:10A8300026181E44304600F0E0F8044600B30368D2
:10A84000F3B1304600F0E3F8D0B10368C3B16368F8
:10A85000AB60304600F0DBF84368EB60304600F058
:10A86000CCF8D0F80090BBF1000F0FD0DAF8003030
:10A8700004229B680C21504698470446E0B9012702
:10A88000384605B0BDE8F08F2A48CAE7D8F800304E
:10A8900004229B680C214046984704460028EED0CD
:10A8A000D8F800304846D3F808A0013080000422D0
:10A8B00001464046D0470AE0DAF800304846D3F86F
:10A8C000088001308000042201465046C047606085
:10A8D0000028D4D0304600F090F8C046C0466368E7
:10A8E00020609A46C3F800904FF0000BD9450ADC6F
:10A8F00010213046FEF70BFF00B13058A060012355
:10A900002B706C60BCE7304600F081F80268019261
:10A910008046304600F071F8019A03689A4208BFF9
:10A9200008EBCB080BF1010BD8F804304AF8043FD0
:10A93000DCE700BF78BD020010B506210446FEF733
:10A94000E6FE00B1205610BD38B504460D46FFF7AF
:10A9500097F9294602462046BDE8384000F061B824
:10A9600038B50D4608210446FEF7D1FE00B1205847
:10A97000013005EB800455F820301C4404212046AA
:10A98000FEF7C5FE28B123582218D118D05800B1BF
:10A99000081D38BDF7B514460268821A03461788A9
:10A9A000042F0D4626D99188461809B3405831180E
:10A9B0003058012601EB8000814214D1062F1AD9AC
:10A9C000D08800B118560DF10701FFF7BDFF40B95F
:10A9D0009DF807002146FFF703FC10B92368734375
:10A9E0002B6003B0F0BD51F804CF0CFB06F6E3E793
:10A9F0000126E3E701260020E5E710B5082104461B
:10AA0000FEF785FE10B123182058184410BD10B56C
:10AA10000A210446FEF77BFE10B123182058184483
:10AA200010BD11282DD8DFE800F0093012161A1ECB
:10AA3000200E22180C241C262814102A0123002082
:10AA400021E00B23FBE70723F9E71123F7E70223B4
:10AA5000F5E71023F3E70323F1E70923EFE70423E6
:10AA6000EDE70D23EBE70523E9E70623E7E70823F6
:10AA7000E5E70C23E3E70E23E1E70F23DFE71223EB
:10AA8000DDE7002301200B7070470A23D7E72DE98B
:10AA9000F04F90F8283085B004469BB385688DB39D
:10AAA000D0E90467002380F828301A46D4F808C09B
:10AAB0009C454FEA820E06EB820007EB820124DC04
:10AAC000ACEB020200F09EF801230022C4E9073239
:10AAD000A669D4F80C80D4F824B04FF0FF33B360EB
:10AAE0003B68736008EB0311B1464968013108BF48
:10AAF0004BF823205BF8233033604FF0010AA36842
:10AB0000534525DC05B0BDE8F08FD4F80C80D4F8AF
:10AB1000249008EB031C1801DCF8041058F800001E
:10AB2000B1F1FF3F1CBF46F80E0047F80E304FEA68
:10AB300083080BBF05F1FF35DCF8041046F825004B
:10AB4000013208BF47F8253049F808100133ADE756
:10AB500057F82A300093009A1B0108EB021158F8AD
:10AB600003300193D1E902234D6802936B1C19D184
:10AB70000020054601460390029B204600F05FF846
:10AB8000039949B14B6809684FEA031C58F80CC097
:10AB90008C446545B8BF654620B10168019B491BDF
:10ABA0008B42E7DC009B4BF82350E1690C234B43BD
:10ABB000F218F550009B53604B1CE361D9F800304C
:10ABC000AB4206DD236A936021620AF1010A9146D5
:10ABD00095E74846D0F808C0BCF1FF3F06D1816038
:10ABE000C2F808C04A46F0E77046F3E70C2303FBBF
:10ABF0000CF306EB030EF358AB42F5DDC2F808C0C8
